:100000000C94B5170C94EE170C94EE170C94EE1795
:100010000C94EE170C94EE170C94EE170C94EE174C
:100020000C94EE170C94EE170C94EE170C94EE173C
:100030000C94EE170C94E92B0C94EE170C94EE171D
:100040000C94EE170C94FD270C946AA10C94EE17F7
:100050000C94D4810C94CA810C94EE170C94EE1776
:100060000C94EE170C94EE170C94EE170C94EE17FC
:100070000C94EE170C94EE170C94EE170C94EE17EC
:100080000C94EE170C94EE170C94EE174E414E495B
:100090004E495459494E46CDCCCC3D0AD7233C1746
:1000A000B7D13877CC2B329595E6241FB14F0A0093
:1000B0000020410000C84200401C4620BCBE4CCA83
:1000C0001B0E5AAEC59D7400407A10F35A00A07200
:1000D0004E18090010A5D4E80000E8764817000083
:1000E000E40B54020000CA9A3B000000E1F5050051
:1000F0000080969800000040420F000000A086019A
:10010000000000102700000000E803000000006469
:1001100000000000000A00000000000100000000D4
:10012000002C76D888DC674F0823DFC1DFAE59E1A9
:10013000B1B796E5E3E453C63AE651997696E8E618
:10014000C28426EB898C9B62ED407C6FFCEFBC9CEB
:100150009F40F2BAA56FA5F490055A2AF75C936BFD
:100160006CF9676DC11BFCE0E40D47FEF520E6B5B8
:1001700000D0ED902E0300943577050080841E0892
:100180000000204E0A000000C80C333333330F98B0
:100190006E12831141EF8D2114893BE65516CFFE77
:1001A000E6DB18D1844B381BF77C1D901DA4BBE403
:1001B00024203284725E228100C9F124ECA1E53D45
:1001C000275045544700504C41005072696E7420CE
:1001D00041626F72746564004D3235005061757311
:1001E000696E672E2E2E004D323400454550524F19
:1001F0004D2056657273696F6E204572726F720082
:10020000454550524F4D20496E64657820457272C5
:100210006F7200454550524F4D2043524320457266
:10022000726F72003F0049676E6F726500526573AE
:10023000657400496E697469616C697A6520454529
:1002400050524F4D004D33303320553120452569F4
:100250002053256900504944204175746F74756EB0
:1002600065202A005049442D44202A005049442D3D
:1002700049202A005049442D50202A0020082046B9
:10028000616374002008204D6178002008204D69CA
:100290006E004F6666004F6E004175746F74656D39
:1002A0007000452073746570732F6D6D005A205374
:1002B000746570732F6D6D00592053746570732FC2
:1002C0006D6D00582053746570732F6D6D0041641F
:1002D00076616E6365642053657474696E6773003C
:1002E00054656D70657261747572650053746570E4
:1002F000732F6D6D00436F6E666967757261746907
:100300006F6E003F004E65787420436F726E6572A9
:1003100000446F6E65004E65787400486F6D696EBD
:10032000672058595A00526573746F72652044658E
:100330006661756C7473004C6F61642053657474EE
:10034000696E67730053746F7265205365747469C6
:100350006E677300416476616E63656420536574F3
:1003600074696E6773004D61696E0052756E6177D6
:1003700061792057617463683A204F4E004D61786F
:100380002054656D7000323630004D696E20546522
:100390006D7000350045313A204550434F532031B0
:1003A00030304B005053550047656E6572696300ED
:1003B00050726F746F636F6C00312E300042617544
:1003C0006400313135323030004D656C7A69202857
:1003D000437265616C69747929004578747275643B
:1003E0006572730031006769746875622E636F6DA2
:1003F0002F6B61642F4D61726C696E2F77696B6929
:10040000004D656761205A65726F00323032312DC0
:1004100030392D303300322E302E392E332D6B6192
:100420006431004D61726C696E00546865726D696B
:1004300073746F727300426F61726420496E666FED
:10044000005072696E74657220496E666F004D616E
:10045000696E003F004261636B0053746F70004D22
:10046000323200417474616368204D6564696100D3
:100470004D3231005072696E742066726F6D204D7E
:10048000656469610052656C65617365204D6564E2
:1004900069610041626F7574205072696E74657293
:1004A00000436F6E66696775726174696F6E0054A0
:1004B000656D7065726174757265004D6F74696FFA
:1004C0006E00526573756D65205072696E740054CC
:1004D000756E650053746F70205072696E740050B1
:1004E00061757365205072696E7400496E666F2085
:1004F00053637265656E003F0053746172742050DF
:1005000072696E740043616E63656C005072696E4F
:10051000740043616E6E6F7420656E746572207333
:1005200075626469723A200002202E2E0001526525
:100530006672657368004D61696E002100486F74D2
:10054000656E6420746F6F20636F6C64004261633A
:100550006B0050726F63656564004D6F74696F6EF8
:100560000044697361626C652053746570706572D4
:1005700073004D383400426564205472616D6D69BA
:100580006E67004732385A004732385900486F6D5D
:100590006520400047323858004175746F20486F1D
:1005A0006D6500473238004D61696E00C601C101BA
:1005B000436F6F6C646F776E00507265686561742D
:1005C00020240046616E205370656564004E6F7A8A
:1005D0007A6C65004D61696E004261627973746581
:1005E00070205A00466C6F770046616E205370652C
:1005F0006564004E6F7A7A6C6500537065656400BF
:100600004D61696E00486F6D696E67204661696C67
:100610006564006F70656E00545249474745524506
:1006200044003A20007A5F6D696E00795F6D696EF3
:1006300000785F6D696E005265706F7274696E67E5
:1006400020656E6473746F70207374617475730ABF
:10065000000000E0C0000000C00000000057617210
:100660006E696E673A20486F6D696E672042756DDE
:10067000702044697669736F72203C20310A000251
:100680000204000068430000634300007A43000056
:10069000A0400000A0400000004000000001000059
:1006A0000001000080005555550000004000333324
:1006B0003300AAAA2A004992240000002000C77132
:1006C0001C0099991900D1451700555515003BB1EB
:1006D00013002449120011111100000010000F0F27
:1006E0000F00E3380E0043790D00CCCC0C00C33072
:1006F0000C00E8A20B0064210B00AAAA0A00703DBE
:100700000A009DD80900427B090092240900DCD32D
:100710000800888808001042080000000800F0C1A6
:1007200007008787070075500700711C07003EEB24
:100730000600A1BC06006990060066660600703ED1
:1007400006006118060017F4050074D105005BB0BF
:100750000500B29005006272050055550500783914
:100760000500B81E0500050505004EEC040087D401
:100770000400A1BD040090A7040049920400C17DBB
:100780000400EE690400C7560400444404005C32CF
:1007900004000821040041100400000004003FF0A0
:1007A0000300F8E0030026D20300C3C30300CCB566
:1007B00003003AA803000A9B0300388E0300C0819F
:1007C00003009F750300D0690300505E03001D53B2
:1007D000030034480300913D03003333030016291E
:1007E0000300381F030097150300300C03000303B8
:1007F00003000BFA020049F10200BAE802005CE0D3
:1008000002002DD802002DD0020059C80200B0C04D
:10081000020031B90200DAB10200AAAA0200A0A3C4
:100820000200BC9C0200FA9502005C8F0200DF8887
:10083000020082820200457C0200277602002770B7
:100840000200436A02007C640200D05E02003F594D
:100850000200C8530200FFFDFCFAF8F6F4F2F0EED5
:10086000ECEAE9E7E5E3E1E0DEDCDAD9D7D5D4D29A
:10087000D0CFCDCBCAC8C7C5C3C2C0BFBDBCBAB933
:10088000B7B6B4B3B2B0AFADACAAA9A8A6A5A4A29E
:10089000A1A09E9D9C9A99989795949392908F8EE3
:1008A0008D8B8A8988878684838281807F7E7D7B09
:1008B0007A797877767574737271706F6E6D6C6B10
:1008C0006A696867666564636261605F5E5D5C5B00
:1008D0005A5958585756555453525150504F4E4DDF
:1008E0004C4B4A4A494847464645444342424140A8
:1008F0003F3E3E3D3C3B3B3A393838373635353460
:100900003332323130302F2E2E2D2C2B2B2A292909
:1009100028272726252524232322212120201F1EA6
:100920001E1D1C1C1B1B1A19191818171616151535
:1009300014131312121111100F0F0E0E0D0D0C0CBB
:100940000B0A0A0909080807070606050504040337
:100950000302020100000000614300006143000047
:100960007A430000E0C0000000C0000000005365B2
:100970007474696E67732053746F72656400290A1A
:10098000002062797465733B2063726320005365B5
:100990007474696E67732053746F726564202800E5
:1009A00048617264636F6465642044656661756C58
:1009B000742053657474696E6773204C6F6164654D
:1009C000640A0020286D6D29002046002048002080
:1009D000204D3134352053004D6174657269616C6E
:1009E0002068656174757020706172616D657465F1
:1009F00072730020204D3134392043203B20556E46
:100A000069747320696E2043656C736975730A009D
:100A100054656D706572617475726520556E697488
:100A200073002020473231203B004C696E656172B3
:100A300020556E69747300454550524F4D206461D6
:100A4000746173697A65206572726F722E0A00296B
:100A50000A002062797465733B2063726320002072
:100A600073746F7265642073657474696E67732044
:100A70007265747269657665642028002028636158
:100A80006C63756C6174656429210A0020213D2026
:100A900000454550524F4D20435243206D69736DC0
:100AA00061746368202D202873746F726564292037
:100AB000002053697A653A2000496E6465783A20CF
:100AC000000000FA430000FA430000A0400000C804
:100AD000410000A0420000A0420000C8430080C0C6
:100AE00043F4010000F401000064000000881300DA
:100AF00000204D61726C696E3D563836290A0045FA
:100B00004550524F4D2076657273696F6E206D6946
:100B1000736D617463682028454550524F4D3D0008
:100B200024F4D43050C38E20C2A24017828B70119F
:100B3000127A910D816CD90AA861E108C75866073D
:100B4000615143061E4B5D05C145A7041A411104BE
:100B5000093D9803713931034036DB026533910258
:100B6000D4305402802E1D02632CEE01752AC5017B
:100B7000B028A001102781018F2564012B244B018F
:100B8000E0223401AC211F018D200D01801FFC00EB
:100B9000841EED00971DDF00B81CD200E61BC600C6
:100BA000201BBC00641AB200B219A8000A19A000E8
:100BB0006A189900D117910040178B00B516840070
:100BC00031167E00B31579003A157300C7146F0013
:100BD00058146A00EE1366008813630025135E0044
:100BE000C7125B006C12570015125400C11151005E
:100BF00070114F0021114B00D61049008D10470095
:100C00004610440002104200C00F4000800F3E001A
:100C1000420F3C00060F3B00CB0E3800930E37000E
:100C20005C0E3500270E3400F30D3200C10D31008B
:100C3000900D3000600D2E00320D2D00050D2C00A2
:100C4000D90C2B00AE0C2900850C29005C0C270068
:100C5000350C27000E0C2600E80B2400C40B2400E2
:100C6000A00B23007D0B23005A0B2100390B210020
:100C7000180B2000F80A1F00D90A1E00BB0A1E002C
:100C80009D0A1D00800A1D00630A1C00470A1B0004
:100C90002C0A1B00110A1A00F7091A00DD091900B5
:100CA000C4091900AB091900920917007B09180043
:100CB000630917004C0916003609160020091600B2
:100CC0000A091500F5081500E0081400CC08140006
:100CD000B8081400A4081400900813007D0812003E
:100CE0006B0813005808120046081200340811005F
:100CF000230811001208110001081100F00710006C
:100D0000E0071000D0071000C0071000B0070F0068
:100D1000A107100091070E0083070F0074070F0052
:100D200065070E0057070E0049070E003B070D0030
:100D30002E070E0020070D0013070D0006070D00FB
:100D4000F9060C00ED060D00E0060C00D4060C00C0
:100D5000C8060C00BC060C00B0060C00A4060B0074
:100D600099060C008D060B0082060B0077060B001F
:100D70006C060B0061060A0057060B004C060A00C1
:100D800042060A0038060A002E060A0024060A0057
:100D90001A060A001006090007060A00FD050900E8
:100DA000F4050900EB050900E2050900D905090071
:100DB000D0050900C7050900BE050900B5050800F2
:100DC000AD050800A50509009C050800940508006C
:100DD0008C050800840508007C05080074050800DF
:100DE0006C050700650508005D050700560508004D
:100DF0004E050700470507004005080038050700B5
:100E0000310507002A050700230507001C05060019
:100E1000160507000F050700080506000205070074
:100E2000FB040600F5040700EE040600E8040600D3
:100E3000E2040700DB040600D5040600CF04060028
:100E4000C9040600C3040600BD040600B70406007A
:100E5000B1040500AC040600A6040600A0040500C9
:100E60009B04060095040500900406008A04050012
:100E700085040500800406007A0405007504050059
:100E8000700405006B04050066040500610405009C
:100E90005C04050057040500520405004D040500DC
:100EA00048040500430405003E0404003A0405001C
:100EB00035040500300404002C0405002704040058
:100EC000230405001E0404001A040400160405008F
:100ED000110404000D0404000904050004040400C6
:100EE00000040400FC030400F8030400F4030400FD
:100EF000F0030400EC030400E8030400E40304002E
:100F0000E0030400DC030400D8030400D40304005D
:100F1000D0030400CC030400C8030300C50303008E
:100F200024F404D9201BC40C5C0E9804C4095F028D
:100F300065077101F405F900FB04B300480487005C
:100F4000C10369005803550003034500BE023A007F
:100F50008402310053022A002902250004022000E5
:100F6000E4011C00C8011900AF011700980114002A
:100F700084011300710110006101100051010E0085
:100F800043010D0036010B002B010B0020010B006B
:100F9000150109000C01090003010800FB0008000D
:100FA000F3000800EB000700E4000600DE00060086
:100FB000D8000600D2000600CC000500C7000500DE
:100FC000C2000500BD000400B9000400B500040023
:100FD000B1000400AD000400A9000400A500030056
:100FE000A20003009F0004009B0003009800030080
:100FF0009500020093000300900003008D000200A2
:101000008B000300880002008600020084000300B9
:10101000810002007F0002007D0002007B000200D0
:1010200079000200770001007600020074000200DF
:1010300072000100710002006F0002006D000100EB
:101040006C0002006A0001006900020067000100F4
:1010500066000100650001006400020062000100FA
:1010600061000100600001005F0002005D000100FE
:101070005C0001005B0001005A0001005900010002
:101080005800010057000100560001005500010002
:101090005400010053000000530001005200010001
:1010A00051000100500001004F0001004E000000FF
:1010B0004E0001004D0001004C0001004B000000FB
:1010C0004B0001004A0001004900010048000000F7
:1010D00048000100470001004600000046000100F2
:1010E00045000000450001004400010043000000ED
:1010F00043000100420000004200010041000000E6
:1011000041000100400001003F0000003F000100DD
:101110003E0000003E0001003D0000003D000100D7
:101120003C0000003C0000003C0001003B000000CF
:101130003B0001003A0000003A00010039000000C5
:1011400039000100380000003800000038000100BC
:1011500037000000370001003600000036000000B4
:1011600036000100350000003500000035000100A8
:10117000340000003400000034000100330000009F
:101180003300000033000100320000003200000094
:101190003200010031000000310000003100010088
:1011A0003000000030000000300001002F0000007F
:1011B0002F0000002F0000002F0001002E00000073
:1011C0002E0000002E0001002D0000002D00000068
:1011D0002D0000002D0001002C0000002C0000005C
:1011E0002C0000002C0001002B0000002B00000050
:1011F0002B0000002B0001002A0000002A00000044
:101200002A0000002A000100290000002900000037
:10121000290000002900000029000100280000002A
:10122000280000002800000028000000280001001D
:101230002700000027000000270000002700000012
:101240002700010026000000260000002600000004
:1012500026000000260001002500000025000000F7
:1012600025000000250000002500000025000100E9
:1012700024000000240000002400000024000000DE
:1012800024000100230000002300000023000000D0
:1012900023000000230000002300000023000100C1
:1012A00022000000220000002200000022000000B6
:1012B00022000000220001002100000021000000A7
:1012C000210000002100000021000000210000009A
:1012D000210001002000000020000000200000008C
:1012E000200000002000000020000000200000007E
:1012F000200001001F0000001F0000001F00000070
:101300001F0000001F0000001F0000001F00010060
:101310001E0000001E0000001E0000001E00000055
:10132000393000003325000087190000B00F00009D
:10133000DB080000BD040000740200003F01000053
:1013400020436F756E7420583A0045310045002CDB
:101350002073797374656D2073746F707065642188
:10136000204865617465725F49443A2000544845DD
:10137000524D414C2052554E4157415900546865D9
:10138000726D616C2052756E61776179004865619C
:1013900074696E67204661696C65640048656174B4
:1013A000696E67206661696C6564004572723A20F7
:1013B0004D415854454D50004D415854454D5020D5
:1013C000747269676765726564004572723A204D90
:1013D000494E54454D50004D494E54454D50207492
:1013E000726967676572656400202F0020403A00CB
:1013F0007C3C3E5E2B3D3F2F5B5D3B2C2A225C00FC
:10140000434F4D4D554E49434154494F4E00445270
:101410005952554E004552524F525300494E464F75
:10142000004543484F00506C6561736520526573F9
:101430006574005052494E5445522048414C544521
:10144000440025533A202553004B494C4C45442E2B
:1014500020005072696E7465722068616C746564F6
:101460002E206B696C6C28292063616C6C6564218B
:101470000A006563686F3A004572726F723A002025
:10148000204D3230312058004D6178204163636532
:101490006C65726174696F6E2028756E6974732F44
:1014A0007332290020204D3230332058004D6178AE
:1014B000206665656472617465732028756E697451
:1014C000732F73290020520020204D3230342050D9
:1014D00000416363656C65726174696F6E20287585
:1014E0006E6974732F7332292028503C7072696EB4
:1014F000742D616363656C3E20523C726574726149
:1015000063742D616363656C3E20543C7472617634
:10151000656C2D616363656C3E2900204A00205490
:101520000020530020204D323035204200416476A7
:10153000616E6365642028423C6D696E5F73656708
:101540006D656E745F74696D655F75733E20533CA5
:101550006D696E5F66656564726174653E20543CBA
:101560006D696E5F74726176656C5F6665656472E5
:101570006174653E204A3C6A756E635F6465763EC1
:10158000290020440020490020204D3330312050D4
:1015900000486F74656E6420504944002E0A002094
:1015A0006E6F742064697361626C65642E20536889
:1015B0006172656420776974680020496E76616C99
:1015C0006964206578747275646572200020746F98
:1015D0006F206C6F6E6720657874727573696F6EBB
:1015E0002070726576656E7465640A0020636F6CA6
:1015F0006420657874727573696F6E207072657699
:10160000656E7465640A00536C6565702E2E2E003D
:10161000436C69636B20746F20526573756D652E22
:101620002E2E00616C736F20656E61626C6564299B
:101630000A004E6F204D6F76652E00456E64206661
:10164000696C65206C6973740A00426567696E2075
:1016500066696C65206C6973740A004E6F206D6555
:101660006469610A00286E6F2066696C6529004311
:10167000757272656E742066696C653A2000534419
:10168000207072696E74696E6720627974652000DB
:101690004E6F74205344207072696E74696E670ACD
:1016A000002E0A0044656C6574696F6E206661697E
:1016B0006C65642C2046696C653A200046696C654F
:1016C0002064656C657465643A002569730025695A
:1016D0006D20256973002569682025696D202569BD
:1016E0007300256964202569682025696D202569B6
:1016F000730025697920256964202569682025699A
:101700006D20256973005072696E742074696D656F
:101710003A20006F6B006F66660021141C141514CC
:101720000E14001444454255473A004D31313320E0
:1017300053004D656761205A65726F204F46462EF3
:1017400000434F4E4649475F4558504F5254004D55
:101750004541545041434B00434F4F4C45525F5419
:10176000454D5045524154555245004348414D4224
:1017700045525F54454D50455241545552450042E3
:101780004142595354455050494E470041524353EA
:10179000004D4F54494F4E5F4D4F44455300544800
:1017A00045524D414C5F50524F54454354494F4E62
:1017B00000455854454E4445445F4D3230004C4F2F
:1017C0004E475F46494C454E414D45004155544FAB
:1017D0005245504F52545F53445F535441545553F4
:1017E0000053445F575249544500524550454154B7
:1017F000005344434152440050524F4D50545F53A4
:101800005550504F525400484F53545F4143544930
:101810004F4E5F434F4D4D414E445300454D455251
:1018200047454E43595F504152534552004341533F
:10183000455F4C494748545F4252494748544E45DA
:10184000535300544F47474C455F4C494748545306
:1018500000534F4654574152455F504F5745520031
:101860004255494C445F50455243454E54004C4507
:1018700056454C494E475F44415441005A5F5052CF
:101880004F42450052554E4F5554004155544F4C10
:101890004556454C005052494E545F4A4F42005005
:1018A000524F4752455353004155544F5245504FA4
:1018B00052545F54454D50004155544F5245504F7E
:1018C00052545F504F5300564F4C554D455452495A
:1018D0004300454550524F4D0042494E4152595FD9
:1018E00046494C455F5452414E534645520053457C
:1018F0005249414C5F584F4E5F584F46460046494B
:10190000524D574152455F4E414D453A4D61726CC3
:10191000696E20322E302E392E332D6B61643120CA
:101920002844656320323720323032312031333A57
:1019300034363A33332920534F555243455F434F92
:1019400044455F55524C3A6769746875622E636FFF
:101950006D2F6B61642F4D61726C696E2050524F18
:10196000544F434F4C5F56455253494F4E3A312ED8
:1019700030204D414348494E455F545950453A4DFA
:10198000656761205A65726F204558545255444529
:10199000525F434F554E543A3120555549443A64AD
:1019A000626663636435352D656262612D3436315C
:1019B000352D616264372D313936616134333866D3
:1019C0003330340A002F2F004D31343520533C6919
:1019D0006E6465783E206F7574206F662072616E4C
:1019E00067652028302D31290A003F4A206F757421
:1019F000206F662072616E67652028302E3031209E
:101A0000746F20302E33290A002058004F464600BC
:101A10004F4E0020204D61783A2000200020204DBC
:101A2000696E3A2000203B200020204D32313120C9
:101A3000530046523A0020466C6F773A20006469A2
:101A40007300656E0043290A0061626C656420289A
:101A50006D696E2074656D702000436F6C64206545
:101A60007874727564657320617265200023646503
:101A700066696E652044454641554C545F004B6491
:101A800020004B6920004B702000504944204175D4
:101A9000746F74756E652066696E6973686564211C
:101AA0002050757420746865206C617374204B70CD
:101AB0002C204B6920616E64204B6420636F6E7331
:101AC00074616E74732066726F6D2062656C6F77DF
:101AD00020696E746F20436F6E66696775726174FA
:101AE000696F6E2E680A00504944204175746F7406
:101AF000756E65206661696C6564212074696D6529
:101B00006F75740A00504944204175746F74756E86
:101B100065206661696C6564212054656D7065722D
:101B2000617475726520746F6F20686967680A0058
:101B3000504944204379636C65730025532025691F
:101B40002F256900204B643A2000204B693A200081
:101B5000204B703A200020436C61737369632050FE
:101B60004944200A002054753A2000204B753A2041
:101B700000206D61783A2000206D696E3A200020C7
:101B8000643A200020626961733A200057616974E9
:101B900020666F7220686561742075702E2E2E008D
:101BA000504944204175746F74756E65207374617B
:101BB00072740A00504944204175746F74756E65E3
:101BC000206661696C6564212054656D7065726181
:101BD0007475726520746F6F20686967680A0050B9
:101BE0004944204175746F74756E65206661696C37
:101BF00065642120426164206865617465722069B2
:101C0000640A00504944204175746F74756E650014
:101C1000454550524F4D204F4B0A004D383400443B
:101C20006F6E65207072696E74696E672066696C8C
:101C3000650A004D3737004D333100496E76616CCF
:101C400069642065787472756465720A0043617016
:101C50003A0020573A00436F6F6C696E672E2E2E44
:101C60000048656174696E672E2E2E00453120256F
:101C700053004572723A207574663820666F6E7430
:101C8000206E6F7420696E697469616C697A65642D
:101C90002E004572723A207574663820666F6E7435
:101CA000206E6F7420696E697469616C697A65640D
:101CB0002E004572723A207574663820666F6E7415
:101CC000206E6F7420696E697469616C697A6564ED
:101CD0002E002568753A2530326875002530326847
:101CE000753A253032687500253032687527253001
:101CF00032687500256875642025303268753A258C
:101D0000303268750042656400456E636C6F7375B0
:101D1000726500202020202020200020202020008C
:101D2000453A00523A00657272001FE02010201000
:101D30002010102010202010201030300840048087
:101D400003001FE03FF03FF03FF01FE01FE03FF0D7
:101D50003FF03FF00FC0078003003FFFF0380070F6
:101D600030FC3020FC102078102030102C00D02EB9
:101D700031D02F7BD02F7BD02E31D02C00D02030F3
:101D80001020781020FC1030FC303800703FFFF03D
:101D90003FFFF03800703186302387102787902F5F
:101DA00087D02F03D02030102078102078102030DA
:101DB000102F03D02F87D0278790238710318630AC
:101DC0003800703FFFF0001DC43F0000000C861972
:101DD0008000000D0E198000000F0B198000000D0F
:101DE0009F198000000DD3998000001CFBFF0000AC
:101DF000000000000000000000000000F380001F51
:101E000080007700001980005B1CF6131DAE5B3567
:101E1000AB0635FB5B3DA70CBD9B4B30EB19B19B73
:101E2000E39D8E9F9D8E0001E000000000012000D8
:101E300000000001E0000000000C0F00FE0702257A
:101E400003BB017FFE08FE08FE05080806000040EF
:101E5000F0C88888987810050808060000C0F8883F
:101E600088888888F80505050600012030F83020AC
:101E70000508080600002070F820202020E0050951
:101E8000090600FF2070A8A8B888887020070505FB
:101E9000070001D86C366CD80509090600FFF8A8C0
:101EA0008888888888A8F8050A0A0600FE2050500D
:101EB000505088A8A8887003030306000340A04080
:101EC000FFFFFFFFFFFFFFFFFFFFFFFFFFFFFFFF22
:101ED000FFFFFFFFFFFF0000000605FF01070706E9
:101EE000020080808080800080030303060105A03B
:101EF000A0A005060606000050F85050F85005094D
:101F0000090600FF2070A8A07028A8702005070708
:101F1000060000C8C8102040989805070706000072
:101F200040A0A040A89068010303060205808080BD
:101F30000309090601FF20404080808040402003C3
:101F400009090601FF80404020202040408005070D
:101F50000706000020A8702070A8200505050600CF
:101F6000012020F820200203030601FFC040800565
:101F70000101060003F8020202060100C0C00507C5
:101F800007060000081010204040800507070600E3
:101F900000708898A8C8887003070706010040C031
:101FA00040404040E0050707060000708808102008
:101FB00040F8050707060000F8081030088870058B
:101FC000070706000010305090F8101005070706AC
:101FD0000000F880F0080888700507070600003048
:101FE0004080F0888870050707060000F808101088
:101FF00020202005070706000070888870888870F8
:10200000050707060000708888780810600205053B
:10201000060100C0C000C0C00206060601FFC0C025
:1020200000C04080030505060101204080402005D6
:102030000303060002F800F80305050601018040CD
:10204000204080050707060000708810202000202F
:102050000507070600007088B8A8B8807005070754
:10206000060000708888F888888805070706000041
:10207000F04848704848F00507070600007088805F
:1020800080808870050707060000F04848484848E7
:10209000F0050707060000F88080F08080F805074B
:1020A00007060000F88080F08080800507070600A2
:1020B000007088808098887005070706000088886F
:1020C00088F8888888030707060100E04040404000
:1020D00040E005070706000038101010109060055A
:1020E00007070600008890A0C0A090880507070693
:1020F0000000808080808080F80507070600008847
:10210000D8A8888888880507070600008888C8A896
:102110009888880507070600007088888888887076
:10212000050707060000F08888F080808005070713
:1021300006000070888888A89068050707060000D8
:10214000F08888F0A0908805070706000070888056
:1021500070088870050707060000F820202020205E
:10216000200507070600008888888888887005078A
:102170000706000088888888505020050707060059
:102180000088888888A8A850050707060000888866
:1021900050205088880507070600008888502020B6
:1021A0002020050707060000F80810204080F803EB
:1021B00009090601FFE080808080808080E00507BB
:1021C000070600008040402010100803090906019E
:1021D000FFE020202020202020E00503030600054A
:1021E0002050880501010600FEF8030303060105DF
:1021F00080402005050506000070087888780507EE
:10220000070600008080F0888888F0050505060034
:10221000007080808870050707060000080878882D
:102220008888780505050600007088F0807005072D
:1022300007060000304840E0404040050707060020
:10224000FE7088888878087005070706000080807F
:10225000F0888888880307070601004000C04040D6
:1022600040E00409090601FE100030101010109023
:102270006005070706000080808890E090880307CB
:1022800007060100C04040404040E005050506004B
:1022900000D0A8A8A8A8050505060000B0C8888831
:1022A0008805050506000070888888700507070600
:1022B00000FEF0888888F080800507070600FE7819
:1022C000888888780808050505060000B0C8808061
:1022D0008005050506000078807008F005070706F0
:1022E00000002020F82020201805050506000088A1
:1022F00088889868050505060000888888502005AC
:1023000005050600008888A8A850050505060000F8
:1023100088502050880507070600FE8888885020CE
:102320004080050505060000F8102040F803090963
:102330000601FF204040408040404020010909063E
:1023400002FF8080808080808080800309090601F0
:10235000FF804040402040404080050303060002CB
:1023600048A890FF43616E6E6F74206F70656E2099
:102370007375626469722000534420636172642043
:102380006F6B0A006F70656E526F6F7420666169C3
:102390006C65640A00766F6C756D652E696E697484
:1023A000206661696C65640A004E6F2053442063A7
:1023B0006172640A000A4D3234004D3233202573B5
:1023C000002E0A006F70656E206661696C65642C72
:1023D0002046696C653A200046696C652073656C1F
:1023E00065637465640A002053697A653A20004683
:1023F000696C65206F70656E65643A2000454E44D7
:1024000020535542524F5554494E450A00222070E0
:102410006F73002220706172656E743A220053550A
:1024200042524F5554494E452043414C4C20746113
:10243000726765743A220053756263616C6C204F59
:10244000766572666C6F7700457863656564656470
:10245000206D617820535542524F5554494E4520C6
:1024600064657074683A0057726974696E672074A5
:102470006F2066696C653A20006672657368006457
:102480006F696E67002066696C653A20004E6F7751
:1024900020002F6175746F25632E670000200000F7
:1024A00000000000000000000000000000DC000050
:1024B00000000000000000000000000000EF00002D
:1024C00000000000000000000000000001F7E00034
:1024D00000000000000000000000000003FBF0000E
:1024E00000000000000000000000000003FCFC00F1
:1024F00000000000000000000000000007FF7E0058
:1025000000000000000000000000000007FFBF0006
:10251000008080EE0E1B070E338303B00FFFDF80B9
:1025200000C0C0E71C7BC70E33C307B80FFFEFC066
:1025300001C0E0E73CFBC70E33E30F3C1FFFF7E0B1
:1025400000E078E338E0870E30E30C001FFFFBF07B
:1025500002E03CE071C0070E30E31C003FFFF430A6
:1025600002709EE0E1C0070E33C31C007FFFEFC086
:102570000770CFE0E1C0070E33C31C003FFFEFF050
:102580000638E7E0C1C0070E30231C001FFFDFE064
:102590000EF8E3E0C0E0070E30E31C001FFFBFC0F1
:1025A0000CFCE0E0C0F1C79C33E30F1C0FFF7F8001
:1025B0001C0CE060C07BC39C33C307BC07FF7F00DB
:1025C000180EE020C03B8190338303B007FEFE006D
:1025D00000000000000000000000000003FDFC00FF
:1025E00000000000000000000000000001FBF800F7
:1025F00000000000000000000000000001F7F000F3
:1026000000000000000000000000000000F7C00013
:10261000000000000000000000000000006E00004C
:10262000000000000000000000000000005000005A
:10263000000000000000000000000000000000009A
:10264000000000000000000000000000000000008A
:10265000000000000000000000000000000000007A
:10266000000FFF03C1FF0000000000000000000099
:102670000008610641018000000000000000000029
:10268000000CE704619CC000000000000000000096
:102690000004CC0C20964000000000000000000068
:1026A00000049809B09260000000000000000000E3
:1026B000000430199093200000000000000000008A
:1026C00000043013D891200000000000000000003A
:1026D0000004983008932000000000000000000073
:1026E0000004CC27EC926000000000000000000015
:1026F0000004E66424964000000000000000000092
:10270000000CF3CC379CC00000000000000000006B
:102710000008618423018000000000000000000028
:10272000000FFFFC3FFF0000000000000000000061
:102730000000000000000000000000000000000099
:102740000000000000000000000000000000FC7E0F
:10275000000000000FFE000000000000000086C224
:102760000000000008020000000000000000C38616
:102770000000000009F20000000000000000438497
:102780000001F0000B62000000000000000049247E
:102790007F1F17F80EC67F7FE3F800000000492472
:1027A000C1B07C0C018CC1C4360C000000004C652B
:1027B0009CE739E403199CE19CE6000000004C65AD
:1027C0003CCD9FE406313CA399B2000000004EE5E9
:1027D00001CD9C040C6F01A6F912000000004FE52A
:1027E0003FE779E408DB3FA409B200000000CC67B2
:1027F0009CB0E9C609F39CE60CE6000000008442A8
:10280000C1EF3C120802C1C2060C00000000FC7EB1
:102810007F4D97FE0FFE7F7E03F800000000000052
:102820000047100000000000000000000000000051
:1028300000707000000000000000000000000000B8
:10284000001FC00000000000000000006D61726CFD
:10285000696E66772E6F726700322E302E392E33F6
:102860002D6B616431001FFFFFFFFFFFFF60000061
:10287000000001FF400000000000FF800000000099
:10288000007F83CF00000C303F87FF80000C301F9B
:10289000867980000C000F8C30C7838C30E78C3039
:1028A000CFC7CC31F38C30DCECEC33B98C30D86C46
:1028B0006C33198C30D06C0C33198C30D86C0C33D1
:1028C000198C30DC6C0E3B198C30CF7C079F198C37
:1028D00030C77C038F194000000000000260000038
:1028E000000000061FFFFFFFFFFFF870012C0190A2
:1028F000012701B0012201C0011D01F001180110E2
:1029000002130130020E016002090190020401C0AD
:1029100002FF000003FA004003F5008003F000D03E
:1029200003EB002004E6007004E100E004DC00405A
:1029300005D700C005D2004006CD00D006C80080F3
:1029400007C3003008BE00F008B900C009B400B0E9
:102950000AAF00B00BAA00D00CA500000EA00050DA
:102960000F9B00C01096005012910000148C00C004
:10297000158700B0178200B0197D00D01B780000C9
:102980001E730040206E0090226900F02464004015
:10299000275F0090295A00E02B5500102E50002090
:1029A000304B0010324600E033410090353C0010BF
:1029B00037370070383200A0392D00B03A2800A017
:1029C0003B2300603C1E00103D1900903D14001098
:1029D0003E0F00703E0A00C03E0500003F00004070
:1029E0003FFBFF803FF6FFC03FF1FF2020506C61AE
:1029F0006E6E657242756666657242797465733A89
:102A000020002046726565204D656D6F72793A2011
:102A10000020436F6D70696C65643A2044656320E3
:102A2000323720323032310A00204C617374205525
:102A30007064617465643A20323032312D30392D42
:102A40003033207C20417574686F723A20286B61A6
:102A5000642C20416E796375626963204D656761FE
:102A6000205A65726F20313256290A004D61726C0E
:102A7000696E20322E302E392E332D6B6164310A6F
:102A80000020536F667477617265205265736574B8
:102A90000A00205761746368646F6720526573652C
:102AA000740A002042726F776E206F757420526531
:102AB0007365740A002045787465726E616C2052EB
:102AC000657365740A00506F77657255700A0073FC
:102AD000746172740A004732385859004D313030F1
:102AE00031006F6B006572726F7220777269746962
:102AF0006E6720746F2066696C650A00446F6E65AE
:102B000020736176696E672066696C652E0A0045E0
:102B10006E6473746F7073002553202563202563E2
:102B200020256320256300205A3A0020593A0020CE
:102B3000583A00656E6473746F7073206869743AF4
:102B40002000004D6F76652025736D6D004D6F760A
:102B50006520302E316D6D004D6F766520316D6DC5
:102B6000004D6F76652031306D6D004D6F766520BC
:102B700041786973004D6F7665204578747275648D
:102B80006572004D6F7665205A004D6F766520594D
:102B9000004D6F76652058005072696E7420667221
:102BA0006F6D204D6564696100FFFFFF4D656761D2
:102BB000205A65726F2052656164792E00507269E7
:102BC0006E74696E672E2E2E005072696E742050DE
:102BD000617573656400220A00556E6B6E6F776EC7
:102BE00020636F6D6D616E643A20220020450020E5
:102BF0005A0020590020204D393220580053746566
:102C000070732070657220756E6974003B200062DD
:102C10007573793A2070617573656420666F7220F0
:102C2000696E7075740A00627573793A2070617507
:102C300073656420666F7220757365720A00627531
:102C400073793A2070726F63657373696E670A00F7
:102C50004D6564696120496E736572746564000036
:102C60000000010200090A00000000040308070038
:102C70000000000000000000000000000000002133
:102C800021204B494C4C2063617573656420627947
:102C900020746F6F206D75636820696E616374695D
:102CA00076652074696D65202D2063757272656E7E
:102CB0007420636F6D6D616E643A20004D31313266
:102CC0002053687574646F776E0053544F505045AD
:102CD000442E20005072696E7465722073746F7098
:102CE0007065642064756520746F206572726F7200
:102CF000732E2046697820746865206572726F7241
:102D000020616E6420757365204D39393920746FE8
:102D100020726573746172742E202854656D70651D
:102D20007261747572652069732072657365742EA3
:102D30002053657420697420616674657220726521
:102D40007374617274696E67290A004E6F2043685C
:102D500065636B73756D2077697468206C696E6547
:102D6000206E756D6265722C204C617374204C6905
:102D70006E653A20004D3239004E6F20436865631E
:102D80006B73756D2077697468206C696E65206E51
:102D9000756D6265722C204C617374204C696E6590
:102DA0003A2000636865636B73756D206D69736DA0
:102DB000617463682C204C617374204C696E653AB1
:102DC00020004C696E65204E756D626572206973D6
:102DD000206E6F74204C617374204C696E65204EB8
:102DE000756D6265722B312C204C617374204C69B7
:102DF0006E653A20004D3131300053657269616C67
:102E000020737461747573206D69736D6174636888
:102E10000A0053442072656164206572726F720A01
:102E200000DB0FC93F45BCDA3F8FB30240FCF027FF
:102E30004056946140FE4B9B4084A5D840E0231847
:102E400041346A5641E859974164DBD5416E2717F2
:102E500042B4B75542CE1A9742C8AED542B5885A49
:102E600043D40684BFA65FA7BF7443E0BF10B11A66
:102E7000C01C2C58C0E8F697C0B849D6C04E4E17B3
:102E8000C124D355C1802497C1A0B5D5C1121A174A
:102E9000C244AE55C2781797C26CACD5C267885A87
:102EA000C320746F6F206C6F6E67206578747275C5
:102EB00073696F6E2070726576656E7465640A0062
:102EC00020636F6C6420657874727573696F6E200F
:102ED00070726576656E7465640A006F6B0A0052E5
:102EE0006573656E643A200020453A00205A3A0026
:102EF00020593A00583A0000002200250028002BF3
:102F00000000002100240027002A00020202020221
:102F1000020202040404040404040403030303037C
:102F20000303030101010101010101010204081071
:102F30002040800102040810204080010204081093
:102F400020408080402010080402014572726F7298
:102F50002077726974696E6720746F2045455052FE
:102F60004F4D210A000057C997CF11241FBECFEF44
:102F7000D0E4DEBFCDBF84B78093101414BE0FB66B
:102F8000F894A89580916000886180936000109209
:102F900060000FBE12E0A0E0B1E0EAEAFBEB01E066
:102FA0000BBF02C007900D92A635B107D9F724E1F7
:102FB000A6E5B2E001C01D92A031B207E1F717E12A
:102FC000C4EBD7E104C02197FE010E9425DBC33B7F
:102FD000D107C9F70E94FEC90C94C8DD0C9400000B
:102FE0000F931F93CF93DF93CDB7DEB760970FB6E4
:102FF000F894DEBF0FBECDBF8C01DC01ED91FC91DA
:103000000280F381E02DBE016F5F7F4F0995882319
:1030100009F464C08981807CC9F56F81637070E0B8
:10302000762F6627770F770F8885B4E08B9FC001D6
:103030001124682B792B89858295869586958370D6
:10304000682B6F5F7F4F90E080E02A852370220F0E
:103050003B8537FB332730F9232B3E813F70230F0D
:103060003327331F2750310904C0660F771F881F8D
:10307000991F2A95D2F760960FB6F894DEBF0FBE5F
:10308000CDBFDF91CF911F910F910895803419F535
:1030900068856695669570E090E080E0CB017727C3
:1030A00066272A85622B098510E0102F0027012E44
:1030B000000C220B330B602B712B822B932B6F5F39
:1030C0007F4F8F4F9F4F4AE0660F771F881F991FD2
:1030D0004A95D1F7D0CF8BE0F801848360E070E0AF
:1030E000CB01C9CF0895FC0182810895FC0190E1D4
:1030F000A4E6B3E001900D929A95E1F70895EF925E
:10310000FF920F931F93E0928B02F0928C02009338
:103110008D0210938E0260938F02709390028093C1
:1031200091029FEFFF27621B730B840B30F4809595
:1031300070956195790B890B99279093A003A6E070
:103140006A9F00929403512DEE277A9F500DE11D46
:103150008A9FE00D50939503E0939603AFE06A9F3A
:1031600000929803512DEE277A9F500DE11D8A9F02
:10317000E00D50939903E0939A03AAE06A9F0092AE
:103180009C03512DEE277A9F500DE11D8A9FE00D83
:1031900050939D03E0939E031F910F91FF90EF903A
:1031A00008959F92AF92BF92CF92DF92EF92FF92DB
:1031B0000F931F93CF93DF9300D000D01F92CDB712
:1031C000DEB7E6E5F8E00027BB27462F572FA82FEC
:1031D000AA2341F4A52F542FB85FAA2319F4A52FD1
:1031E0005527B85FA03138F45295A295452F4F70FE
:1031F000507FA42BBC5FA03428F4550FAA1F550F95
:10320000AA1FBE5FA03818F4550FAA1FB395550F1B
:10321000AA1FEA0FF01F449151E0AA27B85081F18C
:10322000C8F0B0FF02C0440F551FB1FF04C0440FE7
:10323000551F440F551FB2FF06C052954295142FDB
:103240001F70407F512BB3FF1BC0A52F542F442765
:103250000C944019B195B0FF02C055954795B1FF48
:1032600004C05595479555954795B2FF05C05295B1
:10327000407F4295452B5F70B3FF02C0452F552715
:10328000DD24CC24BB24B2E0649FD018C108B00A6E
:10329000B00B749FC018B108B00B849FB018B1096F
:1032A000659FC018B108B00B759FB018B109859F14
:1032B000B0196A9FB018B1097A9FB0194D9DA12C21
:1032C00099243327992722275D9DA00C911C301F3C
:1032D000901F201FAD9D900C311D901F201F4C9DF5
:1032E000A00C911C301F901F201F5C9D900C311D65
:1032F000901F201FAC9D300D911D201F4B9D900CE9
:10330000311D901F201F5B9D300D911D201FAB9D17
:10331000900D211D4B9F300D911D201F5B9F900D27
:10332000211DAB9F200DB1E0BB24CC24DD24639F85
:10333000D018C108B00AB00B739FC018B108B00B09
:10334000839FB018B109699FC018B108B00B799F6D
:10335000B018B109899FB019629FB018B109729F66
:10336000B019D61AC70AB80A20F0B1E03B0F901F77
:10337000201F1124792F632F90E0822F0F900F9040
:103380000F900F900F90DF91CF911F910F91FF90B1
:10339000EF90DF90CF90BF90AF909F900895FC0189
:1033A0007081472F50E0062E02C0559547950A942C
:1033B000E2F740FF14C040916F0250E0062E02C0B9
:1033C000559547950A94E2F740FF09C021E030E0A7
:1033D00001C0220F6A95EAF72095272320830895DC
:1033E0008F929F92AF92BF92CF92DF92EF92FF9215
:1033F000CF93FC01C080D180E280F38020E030E0F8
:1034000040E251E4C701B6010E94A6D420E030E0BA
:1034100048EC52E40E94A6D44B015C0120E030E06D
:10342000A901C701B6010E9440D420E030E040EA83
:1034300050E487FF04C020E030E040EA50ECC501D2
:10344000B4010E9449DB20E030E040E251E40E94F8
:10345000CCDB0E943EDC6B017C018BE2F7FE09C0F5
:10346000F094E094D094C094C11CD11CE11CF11CD8
:103470008DE280936302C701B60120E137E240E0AC
:1034800050E00E9406DB8AE0882E912CA12CB12C02
:10349000CA01B901A50194010E9406DB605D609339
:1034A0006402C701B60128EE33E040E050E00E941C
:1034B00006DBCA01B901A50194010E9406DB605D2B
:1034C00060936502C701B60124E630E040E050E0B9
:1034D0000E9406DBCA01B901A50194010E9406DB26
:1034E000605D609366028EE280936702C701B60159
:1034F000A50194010E9406DBC62FCA01B901A501EE
:1035000094010E9406DB605D60936802C05DC09319
:10351000690283E692E0CF91FF90EF90DF90CF9029
:10352000BF90AF909F908F9008958F929F92AF928F
:10353000BF92CF92DF92EF92FF92FC01C080D180C8
:10354000E280F38020E030E040E251E4C701B601C0
:103550000E94A6D420E030E040E251E40E94A6D4CC
:103560004B015C0120E030E0A901C701B6010E94D7
:1035700040D420E030E040EA50E487FF04C020E07F
:1035800030E040EA50ECC501B4010E9449DB20E084
:1035900030E040E251E40E94CCDB0E943EDC9B0123
:1035A0008BE237FF05C022273327261B370B8DE21E
:1035B00080936402C90168EE73E00E94F2DACB01E5
:1035C000EAE0F0E0BF010E94F2DA805D80936502DC
:1035D000C90164E670E00E94F2DACB01BF010E94EB
:1035E000F2DA805D80936602C901BF010E94F2DABF
:1035F000282FCB01BF010E94F2DA805D8093670221
:103600008EE280936802205D2093690284E692E056
:10361000FF90EF90DF90CF90BF90AF909F908F90F2
:1036200008958F929F92AF92BF92CF92DF92EF92C6
:10363000FF92CF93FC01C080D180E280F38020E034
:1036400030E040E251E4C701B6010E94A6D420E078
:1036500030E048EC52E40E94A6D44B015C0120E02B
:1036600030E040E251ECC701B6010E9440D4181688
:1036700054F420E030E048EC52E4C701B6010E9467
:10368000CCDC87FD86C020E030E0A901C701B6018F
:103690000E9440D487FF6EC060E070E080EA90EC4A
:1036A000A50194010E9449DB20E030E040E251E4B2
:1036B0000E94CCDB0E943EDC6B017C01F7FC5FC00A
:1036C00020E137E240E050E00E9406DBCA01B90188
:1036D0002AE030E040E050E00E9406DB605D60934D
:1036E0006402C701B60128EE33E040E050E00E94DA
:1036F00006DB9AE0892E912CA12CB12CCA01B901CC
:10370000A50194010E9406DB605D60936502C7011C
:10371000B60124E630E040E050E00E9406DBCA013A
:10372000B901A50194010E9406DB605D6093660209
:103730008EE280936702C701B601A50194010E9441
:1037400006DBC62FCA01B901A50194010E9406DB60
:10375000605D60936802C05DC093690284E692E098
:10376000CF91FF90EF90DF90CF90BF90AF909F9060
:103770008F90089560E070E080EA90E491CFF0943B
:10378000E094D094C094C11CD11CE11CF11C6DE2EA
:10379000A6CF20E030E0A901C701B6010E9440D4C5
:1037A00087FF6AC060E070E080EA90ECA5019401B8
:1037B0000E9449DB20E030E040E251E40E94CCDB93
:1037C0000E943EDC4B015C0120E030E0A901C70112
:1037D000B6010E94CCDC87FD0BC020E030E040E267
:1037E00051E4C701B6010E9440D460E287FD13C0D6
:1037F000B7FC47C0C501B40128EE33E040E050E01B
:103800000E9406DBCA01B9012AE030E040E050E046
:103810000E9406DB605D60936502C501B40124E689
:1038200030E040E050E00E9406DB8AE0C82ED12C58
:10383000E12CF12CCA01B901A70196010E9406DB17
:10384000605D609366028EE280936702C501B401F9
:10385000A70196010E9406DBC62FCA01B901A70184
:1038600096010E9406DB605D60936802C05DC093B4
:10387000690285E692E074CF60E070E080EA90E44F
:1038800095CFB094A09490948094811C911CA11C1D
:10389000B11C6DE2C0CF282F81E3243609F080E20D
:1038A0008093660290E22A3040F03AE0822F632F44
:1038B0000E94C4DA0E94C4DA905D90936702822F5E
:1038C0006AE00E94C4DA905D9093680285E280937A
:1038D000690286E692E008956091240170912501C5
:1038E000072E000C880B990B0E9447D42AE037ED75
:1038F00043E25CE30E94A6D460935E0170935F0193
:1039000080936001909361010895CF93DF93EC0160
:10391000CB01BA010E9447D429EC38EC48EC5EE3B5
:103920000E94CCDB20E030E040E05FE30E9449DB16
:103930000E9445DC6883DF91CF9108950E9447D4AF
:1039400029EC38EC48EC5EE30E94CCDB20E030E070
:1039500040E05FE30E9449DB0E9445DC24E6629F71
:10396000C001112481589F4F6FEF70E00E94F2DA7E
:10397000862F0C944B1C80919805811104C0809176
:10398000E8028093F90508958091EF128823C1F031
:1039900081508093EF12E4E5F1E1882351F08150EA
:1039A000990B2BE1289FF001299FF00D1124EF5175
:1039B000FE4E8BE1A9E3B1E101900D928A95E1F70A
:1039C0002091EF12211105C08091F912806480933B
:1039D000F91281E090E0A0E0B0E0211103C080E0A6
:1039E00090E0DC0180937F0590938005A093810592
:1039F000B09382051092790581E080938F0583E072
:103A000080934E010895CF92DF92EF92FF92CF9371
:103A1000DF9300D000D0CDB7DEB76B017C0120E092
:103A200030E0A9010E9440D487FD1BC06DEB77E315
:103A300086E095E3A70196010E9449DB69837A83BA
:103A40008B839C83CE0101960E94951A0F900F9054
:103A50000F900F90DF91CF91FF90EF90DF90CF907C
:103A600008956DEB77E386E095EBE4CF8F929F921C
:103A7000AF92BF92CF92DF92EF92FF92CF936B0102
:103A80007C0120E030E0A9010E9440D487FDAAC05B
:103A90006DEB77E386E095E3A70196010E9449DB91
:103AA0006B017C0120E030E0A9010E9440D487FF37
:103AB0009EC0C701B601905820E030E040E251E4DA
:103AC0000E94A6D420E030E040E251E40E94A6D457
:103AD00020E030E040EA50E40E9449DB20E030E0A2
:103AE00040E251E40E94CCDB0E943EDC6B017C0191
:103AF00080E28093630260E280E1C81687E2D80624
:103B0000E104F1048CF0C701B60120E137E240E0A6
:103B100050E00E9406DBCA01B9012AE030E040E033
:103B200050E00E9406DB605D6093640260E288EE14
:103B3000C81683E0D806E104F1048CF0C701B60191
:103B400028EE33E040E050E00E9406DBCA01B901F4
:103B50002AE030E040E050E00E9406DB605D6093C8
:103B6000650260E284E6C816D104E104F1048CF039
:103B7000C701B60124E630E040E050E00E9406DBD9
:103B8000CA01B9012AE030E040E050E00E9406DBC3
:103B9000605D609366028AE0882E912CA12CB12C86
:103BA000C701B601A50194010E9406DBC62FCA0118
:103BB000B901A50194010E9406DB605D6093670274
:103BC0008EE280936802C05DC093690283E692E052
:103BD000CF91FF90EF90DF90CF90BF90AF909F90EC
:103BE0008F9008956DEB77E386E095EB55CF20E05D
:103BF00030E040E251E4C701B60162CFCF93DF93DA
:103C0000EC01CB01BA010E9447D420E030E040E251
:103C100051E40E94CCDB688379838A839B83DF91A4
:103C2000CF910895CF93DF93EC01CB01BA010E94AD
:103C300047D420E030E040E251E40E94CCDB6883CE
:103C400079838A839B83DF91CF9108950E9447D423
:103C500020E030E040E251E40E94CCDB0C94361DC1
:103C6000CF93DF93EC01CB01BA010E9447D420E04F
:103C700030E048EC52E40E94CCDB688379838A838D
:103C80009B83DF91CF910895CF93DF93EC01CB011C
:103C9000BA010E9447D420E030E048EC52E40E9490
:103CA000CCDB688379838A839B83DF91CF910895EE
:103CB000CF92DF92EF92FF92CF93DF9300D000D0AC
:103CC000CDB7DEB70E9447D420E030E048EC52E4A4
:103CD0000E94CCDB6B017C0120E030E0A9010E9456
:103CE00040D42DEB37E346E055E387FF04C02DEBCE
:103CF00037E346E055EBC701B6010E9449DB698313
:103D00007A838B839C83CE0101960E94F0190F90D9
:103D10000F900F900F90DF91CF91FF90EF90DF9079
:103D2000CF9008950E9447D420E030E040E251E473
:103D30000E94CCDB0C94031DCF92DF92EF92FF9296
:103D4000CF93DF9300D000D0CDB7DEB70E9447D429
:103D500020E030E048EC52E40E94CCDB6B017C01B7
:103D600020E030E0A9010E9440D42DEB37E346E08B
:103D700055E387FF04C02DEB37E346E055EBC70161
:103D8000B6010E9449DB69837A838B839C83CE01D1
:103D900001960E94111B0F900F900F900F90DF91D2
:103DA000CF91FF90EF90DF90CF900895CF93DF9366
:103DB000EC01CB01BA010E9447D40E943EDC79831A
:103DC0006883DF91CF9108952CEA35EC47E25EE3FA
:103DD0006091DC027091DD028091DE029091DF0241
:103DE0000E94CCDB6093CC057093CD058093CE050B
:103DF0009093CF0508952CEA35EC47E25EE360919D
:103E0000E0027091E1028091E2029091E3020E944F
:103E1000A6D46093C8057093C9058093CA05909392
:103E2000CB05089580917B1190917C11891B8F7037
:103E300089F48091A805813069F09091F91292FB84
:103E4000882780F992FF07C097FB882780F991E0C7
:103E50008927089581E00895CF93DF93C091C1052C
:103E6000D091C205209729F16091BD057091BE05E2
:103E70008091BF059091C0050E943EDC6E5F7F4F30
:103E800024976C177D07ACF470938C0360938B03BD
:103E90000E943CA1605E714B8F4F9F4F60938D03DA
:103EA00070938E0380938F0390939003DF91CF9153
:103EB000089510928D0310928E0310928F0310922A
:103EC0009003F4CF0C942C1FCF93DF93EC018D81E2
:103ED0000E940A8260E08B81DF91CF910C9441A017
:103EE000DF92EF92FF920F931F93CF93DF938C019A
:103EF000C62FD22FF32EE42ED52E0E94641F0E94CF
:103F000048A18C2F80640E94FE818D2D0E94FE812D
:103F10008E2D0E94FE818F2D0E94FE818D2F0E948A
:103F2000FE8187E8C11101C085E90E94FE81CC3085
:103F300011F40E940382C0E00E940382F80186838C
:103F400087FF04C0CF3F11F0CF5FF6CFDF91CF9155
:103F50001F910F91FF90EF90DF90089561E0FC01B9
:103F600083810E9441A08FEF0C94FE810F931F93D9
:103F7000CF938C010E94641F0E9448A1C82F882300
:103F800071F08DEF0E94FE810E9448A1C82FC801E8
:103F90000E94AE1F8C2FCF911F910F91089582E147
:103FA000F8018483F4CF8F929F92AF92BF92CF9209
:103FB000DF92EF92FF920F931F93CF93DF93EC0169
:103FC0006A017B01590120E030E0A90167E30E940A
:103FD000701FA501980167E1CE010E94701F811139
:103FE00027C08F81833039F089E0CC0CDD1CEE1CBA
:103FF000FF1C8A95D1F7A701960169E1CE010E94C5
:10400000701F11E0882319F010E087E08C83CE0147
:104010000E94AE1F812FDF91CF911F910F91FF90D2
:10402000EF90DF90CF90BF90AF909F908F900895CA
:1040300089E08C8310E0EBCFCF93DF93EC016EBD72
:10404000FA01CA019E5F0DB407FEFDCF20812EBD8F
:104050000DB407FEFDCF21812EBD3296E817F9077A
:1040600091F70DB407FEFDCF8FEF0E94FE818FEF19
:104070000E94FE810E9403828E838F71853049F0F9
:1040800083E18C83CE010E94AE1F80E0DF91CF914F
:10409000089581E0FBCF0F931F93CF93DF93EC0143
:1040A0008B010E94641F0E9448A181110CC085E110
:1040B0008C8310E0CE010E94AE1F812FDF91CF9143
:1040C0001F910F910895A8016CEFCE010E941C2052
:1040D000182F882361F3EECF0F931F93CF93DF93B5
:1040E000EC0189018F81833039F089E0440F551F3D
:1040F000661F771F8A95D1F79A01AB0168E1CE015F
:104100000E94701F81112AC0A8016EEFCE010E948B
:104110001C20182F8823B1F00E9448A1182F882353
:10412000D1F020E030E0A9016DE0CE010E94701FC7
:10413000882321F086E18C8310E004C00E94038272
:104140008111F8CFCE010E94AE1F812FDF91CF9158
:104150001F910F91089587E18C83F4CF86E0EBCF18
:104160001F93CF93DF93EC010E94641F20E030E0A7
:10417000A9016CE0CE010E94701F11E0882319F0A4
:1041800010E083E08C83CE010E94AE1F812FDF916F
:10419000CF911F9108951F93CF93DF93EC018F81EF
:1041A000833039F089E0440F551F661F771F8A95C9
:1041B000D1F79A01AB0162E1CE010E94701F11E0BC
:1041C000882319F010E085E08C83CE010E94AE1F99
:1041D000812FDF91CF911F9108958F929F92AF927F
:1041E000BF92EF92FF920F931F93CF93DF938C01B7
:1041F000EB017A010E943CA14B015C012CE2820E92
:1042000021E0921EA11CB11C0E940382F80186834A
:104210008F3F69F40E943CA1681979098A099B09BA
:1042200097FDF2CF81E1F8018483C0E021C08E3F89
:1042300071F5F1E0EF1AF1088FEF8EBDFE012FEF5F
:104240000DB407FEFDCF8EB581932EBDCF018C1B23
:104250009D0B8E159F05A0F30DB407FEFDCF8EB507
:10426000CE0DDF1D88830E9403820E940382C1E07D
:10427000C8010E94AE1F8C2FDF91CF911F910F912B
:10428000FF90EF90BF90AF909F908F9008958FE038
:10429000CACF0F931F93CF93DF93EC018B010E9442
:1042A000641F40E052E0B801CE01DF91CF911F9131
:1042B0000F910C94ED200F931F93CF93DF93EC019C
:1042C00089018F81833039F089E0440F551F661FC3
:1042D000771F8A95D1F79A01AB0161E1CE010E9467
:1042E000701F81110AC040E052E0B801CE01DF9199
:1042F000CF911F910F910C94ED2084E08C83CE011F
:104300000E94AE1F80E0DF91CF911F910F91089521
:104310008F929F92AF92BF92CF92DF92EF92FF92D5
:104320000F931F93CF93DF93EC01162F1F821C82F4
:104330004B830E943CA16B017C0120EDC20E27E063
:10434000D21EE11CF11CA89561E08B810E9441A066
:104350008B810E942E9C249A2C9A279A2698259A23
:1043600081E00E940A8285E08D830E940A820AE031
:104370008FEF0E94FE810150D9F7A89520E030E030
:10438000A90160E0CE010E94701F8E83813081F010
:104390000E943CA16C197D098E099F0997FDEECF03
:1043A00081E08C83CE010E94AE1F1A8280E06AC039
:1043B000A8952AEA31E040E050E068E0CE010E9492
:1043C000701F853041F581E08F83A8958F81812C06
:1043D000912C5401823029F4812C912CA12C80E461
:1043E000B82E20E030E0A90167E3CE010E94701FE3
:1043F000A501940169E2CE010E94701F8E8388237B
:10440000F1F00E943CA16C197D098E099F0997FD6E
:10441000E8CF8AE0C6CF04E00E9403828E83015079
:10442000D9F78A3A11F482E0CFCF0E943CA16C19EF
:104430007D098E099F0997FDBCCF82E0B2CF8F81A5
:104440008230C1F420E030E0A9016AE3CE010E948D
:10445000701F882311F088E0A4CF0E940382807C23
:10446000803C11F483E08F830E9403820E940382C8
:104470000E940382CE010E94AE1F81E08A83173022
:1044800070F41D83DF91CF911F910F91FF90EF90FA
:10449000DF90CF90BF90AF909F908F90089588E16C
:1044A0008C8384CF0F931F93CF93DF93EC018B0109
:1044B00020E030E0A90169E00E94701F81110AC06C
:1044C00040E150E0B801CE01DF91CF911F910F91F3
:1044D0000C94ED2080E18C83CE010E94AE1F80E021
:1044E000DF91CF911F910F910895CF93C82FCB01EA
:1044F0000E94567D82E296E00E94567D83E196E01E
:10450000CC2311F088E196E00E94567D8AE0CF919D
:104510000C944F7D4091890221E042276CE070E0CD
:104520000C94F89B4091890221E0422764E070E0FE
:104530000C94F89B4091890221E0422761E070E0F1
:104540000C94F89B4091890221E0422761E070E0E1
:104550000C94F89B4091890221E0422768E070E0CA
:104560000C94F89B4091890221E042276CE070E0B6
:104570000C94F89B41E061E070E00C94F89B409152
:10458000890221E042270C94F89B6CE070E00C94C7
:10459000D0A061E070E00C94D0A06CE070E00C94CE
:1045A000D0A064E070E00C94D0A0BC0182E691E061
:1045B0000C94CCC680E090E0A0E8B0E480936A015F
:1045C00090936B01A0936C01B0936D018BEF91E020
:1045D0000E94D52280E090E0A0EFB1E480936201D8
:1045E00090936301A0936401B09365018093660189
:1045F00090936701A0936801B0936901E091E5028F
:10460000EE0FFF0BE552FE4F8081918183309105C3
:1046100049F184309105D9F1029761F480E090E08E
:10462000A3E4B3E48093620190936301A0936401D7
:10463000B093650183EE91E00E94D52210926A0149
:1046400010926B0110926C0110926D018BEF91E052
:104650000E94D5228091E5028F5F8430ECF4809334
:10466000E502089580E090E0A3E4B3E48093620162
:1046700090936301A0936401B093650180936601F8
:1046800090936701A0936801B0936901D3CF80E054
:1046900090E0A3E4B3E4F2CF1092E5020895CF9343
:1046A000DF93CDB7DEB720E24F8158856E818D81D3
:1046B0000E94029EDF91CF9108956EE672E582E03E
:1046C0000C94FAC663E772E581E00C94FAC668E7D9
:1046D00072E580E00C94FAC668E270E583E00C9421
:1046E000FAC6109279050C94F2AC80914E018823A1
:1046F00051F06091DA027091DB0230E020E041E09D
:1047000081E00C947C730895CF93DF93EC010E94B9
:104710003FA91B82DF91CF910895CF93DF93EC01E6
:10472000462F41706C857D858E859F850E942FA6C2
:10473000882351F0888920E2829FC0011124815F83
:10474000904FDF91CF91089590E080E0FACFCF9322
:10475000DF93EB01FC012381211104C080E0DF9194
:10476000CF9108952250223028F48FE28883198255
:1047700081E0F5CF60E00E948D23009779F3DC01A2
:1047800060E080E09EE22D91203299F0883031F493
:104790009E01260F311DF90190836F5F9E01260F48
:1047A000311DAD0141505109FA014081F9014083A9
:1047B0006F5F8F5F8B3039F7FE01E60FF11D1082BE
:1047C000D7CF3F924F925F926F927F928F929F923C
:1047D000AF92BF92CF92DF92EF92FF920F931F930F
:1047E000CF93DF93CDB7DEB72C970FB6F894DEBF2B
:1047F0000FBECDBF5C01DC0159968D909C90F401F9
:1048000081859285A385B4859C01AD012F5F3F4FC3
:104810004F4F5F4F29873A874B875C87D5011496A6
:104820004D905D906D907C901797411451046104F8
:10483000710409F459C0BFEF4B1A5B0A6B0A7B0A7B
:10484000312C730162011D821E821F821886F401C1
:1048500081859285A385B4852D813E814F815885C0
:10486000281739074A075B0708F056C089859A85DB
:10487000AB85BC858C159D05AE05BF0550F482E067
:10488000C82ED12CE12CF12C92E0492E512C612C18
:10489000712C9E012F5F3F4FB701A601C4010E94FA
:1048A00052A88823C9F189819A81AB81BC81892B67
:1048B0008A2B8B2B01F1260137019FEF491A590AE8
:1048C000690A790A2D813E814F8158852F5F3F4FBC
:1048D0004F4F5F4F2D833E834F8358873FEFC31A5F
:1048E000D30AE30AF30AB3CF408051806280738019
:1048F00033243394A6CFC414D504E604F70411F787
:104900000FEF1FEF2FEF3FE0B701A601C4010E9498
:10491000C0A7782E81111AC0712C872D2C960FB646
:10492000F894DEBF0FBECDBFDF91CF911F910F91E5
:10493000FF90EF90DF90CF90BF90AF909F908F90BF
:104940007F906F905F904F903F900895F501448164
:10495000558166817781411551056105710539F0F1
:1049600097018601C4010E94C0A78823A9F2D5013E
:104970001496CD92DD92ED92FC921797332051F070
:10498000D701C6010196A11DB11DF4018083918359
:10499000A283B383F50185899689A789B08D892B78
:1049A0008A2B8B2B09F0B9CFC58AD68AE78AF08E7D
:1049B000818180688183B1CF40E050E0BA010C94DE
:1049C0008BA94F925F926F927F92AF92BF92CF92DC
:1049D000DF92EF92FF920F931F93CF93DF931F927B
:1049E000CDB7DEB78C017B015A01C22EDB0159968F
:1049F0008D919C91F801928F818FCB010E94DC24D4
:104A0000712CF70180859185A285B38541895289F2
:104A10006389748984179507A607B70708F052C001
:104A200055E0B695A795979587955A95D1F7F82FA4
:104A3000FF70DF2ED70113968C91823010F480E046
:104A4000DBC041E050E0BE016F5F7F4FC7010E94B5
:104A5000B3AA0197A1F7F70180859185A285B38557
:104A60004F96A11DB11D80879187A287B387F0E281
:104A7000DF9EB0011124615F704F61157105F9F27D
:104A8000DB018C91882341F0853E09F04CC07720F2
:104A900029F077247394B5CF71100EC080910F1157
:104AA00090911011A0911111B0911211F801848709
:104AB0009587A687B787D08ADB018C918111E9CFD2
:104AC000772473948C2D8274823409F0B8CF7720C8
:104AD00009F4A2C0F801D08861E0C8010E948D23CA
:104AE000009709F4ACCF20E2DC011D922A95E9F78A
:104AF0002BE0F501DC0101900D922A95E1F721E20E
:104B000038E2FC01318B208B40E058E05787468724
:104B1000338B228B318F208F578B468B0E94E6A5DB
:104B2000811109C08CCF4BE050E0C5010E945EDDD1
:104B3000892B09F066CFF0E2DF9ED00111249D01A0
:104B4000215F304FF9018385817121F08C2D8271B5
:104B500009F001C1F801818D928D40910F115091A2
:104B60001011609111117091121144875587668759
:104B70007787D08AFD01E15FF04F44885588712C1A
:104B8000612C320155244424D80155964D925D92F2
:104B90006D927C925897428D538D70E060E044296D
:104BA00055296629772955964D935D936D937C938E
:104BB0005897D9011B962C91287109F0BEC0848D9D
:104BC000958DA68DB78DF801818B928BA38BB48BBD
:104BD00081E083838C2D8F70F8018183148215828C
:104BE00016821782108611861286138681E0C4FE13
:104BF00003C0C8010E941FAA0F90DF91CF911F919F
:104C00000F91FF90EF90DF90CF90BF90AF907F908B
:104C10006F905F904F900895D70113968C911397E2
:104C2000823009F40CCF51968D919D910D90BC91DD
:104C3000A02D803E9F4FAF41B10508F000CFC701C6
:104C40000E94E123882309F4FACE0E94E6A5882376
:104C500009F4F5CED7015996ED91FC915A97149627
:104C60004D905D906D907C901797B2E04B1A510873
:104C700061087108858504C0440C551C661C771CAE
:104C80008A95D2F786859785A089B189480E591EE5
:104C90006A1E7B1E81E08093131140920F11509287
:104CA00010116092111170921211EFE0FFE080E09C
:104CB00092E0DF019C011D9221503040E1F7DD249C
:104CC000D394D7015996ED91FC918481D816C0F404
:104CD0008091141190911511DC01ED91FC910288E5
:104CE000F389E02D2FE03FE0B301A2014D0D511DEE
:104CF000611D711D0995882309F4A1CED394E1CFDC
:104D0000258580E092E0A0E0B0E004C0880F991F04
:104D1000AA1FBB1F2A95D2F7F701418952896389DF
:104D20007489840F951FA61FB71F818B928BA38B4D
:104D3000B48B8FE09FE0D12CD6CE203161F4980166
:104D40002F5E3F4F0E94D5A8882329F084E0D80128
:104D500013968C933FCFD80113961C9270CEFC0112
:104D6000238121110C94842308952F923F924F9216
:104D70005F926F927F928F929F92AF92BF92CF92EB
:104D8000DF92EF92FF920F931F93CF93DF93CDB7F4
:104D9000DEB7C354D1090FB6F894DEBF0FBECDBF46
:104DA0004C015B016A01222E19821C821C8E1F8E0F
:104DB0006115710521F510E0CE014C960E94AF26D9
:104DC000CE0101960E94AF26812FCD5BDF4F0FB63B
:104DD000F894DEBF0FBECDBFDF91CF911F910F9131
:104DE000FF90EF90DF90CF90BF90AF909F908F900B
:104DF0007F906F905F904F903F902F900895FC01AF
:104E000083818111D8CFFA0180818F32A1F18B018A
:104E1000CE0101967C013C0180E2382E2E019CE1FE
:104E2000490E511C2396EFAE23972496FFAE24978C
:104E300022963FAE229721963FAE21973FAE3EAEDF
:104E40003DAE3CAE3BAE3AAE39AE38AE3FAA96016F
:104E500090E047E0D9018D91882309F447C08F3253
:104E600009F444C08E3209F54A3009F4A4CF98E021
:104E70004AE09D01EFCFFB01838182508B0182309C
:104E800060F0618D728DCE014C960E94A2AC8E01B5
:104E9000045E1F4F882309F48ECFC6016C01019672
:104EA000F60120812F32D1F3B3CFE0EFF3E124916B
:104EB000222321F031968213FACF7DCF491708F4CF
:104EC0007ACF813208F477CF8F3709F474CF3FE976
:104ED000380F3A3108F420EEE7E3F0E0EC0FFD1F65
:104EE000E90FF11D820F80839F5FC3CF8FA98032AE
:104EF00009F461CF6901F90180812F5F3F4F8F3243
:104F0000C9F3882301F121E0AE01495C5F4FB8018C
:104F1000C7010E94E124882309F44DCF0A151B051F
:104F200019F0C8010E948423942D852D6E147F04EE
:104F300031F023969FAD239724968FAD2497870158
:104F4000E92EF82E75CF222DAE01495C5F4FB801D6
:104F5000C4010E94E124182F2FCF8F929F92AF920D
:104F6000BF92CF92DF92EF92FF920F931F93CF9356
:104F7000C82F09EB15E0F80160857185072E000C3C
:104F8000880B990B0E9447D46B017C01F801848047
:104F90009580A680B78080E20E944F7D84E50E94C4
:104FA0004F7D8AE30E944F7DC501B4010E944D9C54
:104FB00089EE93E10E94567DC701B6010E944D9C87
:104FC00062E070E080E090E00E949DA087E1C8026E
:104FD000F0011124E754FA4F628570E08CEE93E102
:104FE000CF911F910F91FF90EF90DF90CF90BF90E6
:104FF000AF909F908F900C940C810F930FB70F93ED
:1050000000916E000B7F00936E0078940F930BB7A6
:105010000F930CB70F921F922F933F934F935F9371
:105020006F937F938F939F93AF93BF93EF93FF9370
:1050300011240E947663FF91EF91BF91AF919F91F0
:105040008F917F916F915F914F913F912F911F9021
:105050000F900CBF0F910BBF0F910460F894009359
:105060006E000F910FBF0F9118951092D005E9EBCC
:10507000F5E01186108610928D0310928E03109227
:105080008F031092900312865D980895EF92FF921D
:105090000F931F93CF93C82F7B018A018091DC056A
:1050A0008330E0F00E94637EC7010E94567D8FE44A
:1050B00093E10E94567DC7FD0EC08DE493E10E94EE
:1050C000567D6C2FCC0F770B880B990B0E94499B58
:1050D0008AE00E944F7D8AE00E944F7D0E94352821
:1050E000A89580917403811129C081E08093740395
:1050F00082E08093DC050E943528C5E1C150149AF6
:10510000B9F069E170E080E090E00E949DA0A89570
:10511000149868E270E080E090E00E949DA0A8955D
:1051200068E270E080E090E00E949DA0A895E6CF44
:1051300040E06AE473E1C8010E942881CF911F9189
:105140000F91FF90EF900895CF93DF93A8958091F2
:10515000BB059091BC050E94649B6093BD05709354
:10516000BE058093BF059093C005C091BB05D0914B
:10517000BC058091460190914701C817D9073CF4BE
:105180004BEA53E168EB73E180E00E94462880918E
:10519000C1059091C2051816190684F48091440146
:1051A000909145018C179D074CF44AEC53E167ED53
:1051B00073E180E0DF91CF910C944628DF91CF918D
:1051C00008952F923F924F925F926F927F928F92AB
:1051D0009F92AF92BF92CF92DF92EF92FF920F9386
:1051E0001F93CF93DF93CDB7DEB72F970FB6F89409
:1051F000DEBF0FBECDBF8091DC0581111AC0A8951E
:105200002F960FB6F894DEBF0FBECDBFDF91CF91C2
:105210001F910F91FF90EF90DF90CF90BF90AF90D4
:105220009F908F907F906F905F904F903F902F90C6
:10523000089580918A038111E3CF81E080938A03EE
:1052400080919302811103C010928A03D9CF0E94EA
:10525000A428109293020E943CA12B013C01609172
:105260004A0170914B01072E000C880B990B0E948C
:1052700047D49B01AC016091BD057091BE05809142
:10528000BF059091C0050E94CCDC18160CF4F2C149
:105290006091C1057091C205072E000C880B990B17
:1052A0000E9447D46B017C012091741130917511DB
:1052B00040917611509177110E9440D4811174C0B1
:1052C0002091731129835981523009F499C15330C7
:1052D00009F4C8C1513009F4D5C1C090BD05D090C2
:1052E000BE05E090BF05F090C00560914801709147
:1052F0004901072E000C880B990B0E9447D4A70187
:1053000096010E9440D487FF11C060914A017091BC
:105310004B01072E000C880B990B0E9447D4A70164
:1053200096010E94CCDC18160CF456C060E0609325
:10533000C30580918D0390918E03A0918F03B0914E
:1053400090030097A105B10509F47ECFA301920156
:10535000281B390B4A0B5B0BDA01C901B7FD74CF6F
:10536000C701B6010E943EDC20918B0330918C0373
:10537000621773070CF4B1C12091C1053091C205C9
:105380002115310541F06E5F7F4F245031096217BE
:1053900073070CF4AFC110928D0310928E0310921C
:1053A0008F031092900350CFC0927411D092751158
:1053B000E0927611F092771131E0398320E030E00D
:1053C000A901C701B6010E94CCDC18160CF01982A5
:1053D00049814093731177CF6091C1057091C205E7
:1053E0006115710509F481C1072E000C880B990B1A
:1053F0000E9447D4A70196010E9448DB4B015C0143
:1054000020E030E040E251EC0E9440D487FD6DC1C5
:1054100020E030E040E251E4C501B4010E94CCDC60
:1054200018160CF47AC18091890381117AC1809198
:10543000810390918203A0918303B09184038983B7
:105440009A83AB83BC83209185033091860340917E
:105450008703509188032D833E834F835887A7018C
:105460009601609175037091760380917703909116
:1054700078030E9448DB2091CC053091CD05409106
:10548000CE055091CF050E94A6D429813A814B8147
:105490005C810E9448DB20ED3CEC4CE45DE30E9423
:1054A000A6D429813A814B815C810E9449DB6983C2
:1054B0007A838B839C8360938103709382038093B0
:1054C0008303909384038091C8059091C905A091AE
:1054D000CA05B091CB0589879A87AB87BC872D8198
:1054E0003E814F815885C501B4010E9449DB8B0183
:1054F0008F879E8720E030E0A9010E9440D487FD7D
:105500001BC129853A854B855C8560E070E08FE79B
:1055100093E40E94CCDB6D837D871C0198014F854D
:105520005E850E9440D487FF04C00D811D852F86B3
:105530003E86C801AF85BE85809385039093860320
:10554000A0938703B09388032091C4053091C505CB
:105550004091C6055091C705C501B4010E94A6D46B
:105560004B015C018092790390927A03A0927B03B5
:10557000B0927C0398014F855E8569857A858B851D
:105580009C850E94A6D49B01AC0120937D0330939F
:105590007E0340937F0350938003C501B4010E94B2
:1055A00049DB29813A814B815C810E9449DB20E003
:1055B00030E0A9010E9449DB4B015C0120E030E0B2
:1055C000A9010E9440D487FD93C020E030E04FE75E
:1055D00053E4C501B4010E94CCDC181654F46FE703
:1055E000C0927503D0927603E0927703F09278032D
:1055F0009ECEC501B4010E943EDC75956795F0CF43
:10560000C090BD05D090BE05E090BF05F090C005EC
:105610008090741190907511A0907611B0907711D0
:1056200020E030E040E850E4C501B4010E9448DBCE
:10563000A70196010E9440D418160CF03FC00E94AA
:105640003CA1C0906F11D0907011E0907111F0905A
:1056500072116C197D098E099F0997FD3ECE83E07A
:10566000809373114DE653E16DE773E180E00E9492
:10567000462833CE4BEA53E168EB73E180E00E94A9
:10568000462806CEC090BD05D090BE05E090BF056F
:10569000F090C0058090741190907511A0907611D3
:1056A000B0907711A5019401C701B6010E9440D4C2
:1056B00087FD1BCE82E080937311B2CF0E943CA184
:1056C000605C73468F4F9F4F60936F1170937011A2
:1056D000809371119093721100CE4DE853E16CE903
:1056E00073E180E00E944628AFCD81E0809389037A
:1056F00060E076CF70938C0360938B030E943CA193
:10570000605E714B8F4F9F4F60938D0370938E033C
:1057100080938F039093900397CD81E080938903CA
:105720005ECF109289031D821E821F821886198205
:105730001A821B821C8293CE00E010E01F861E8618
:10574000F8CECF92DF92EF92FF92CF93DF93EC01EE
:10575000C880D980EA80FB8080E493E10E94567D76
:10576000C701B6010E94499BCC80DD80EE80FF809E
:1057700080EF9EE20E94567DC701B6010E94499BC0
:10578000C884D984EA84FB848CEE9EE20E94567D14
:10579000C701B6010E94499B8AE0DF91CF91FF903B
:1057A000EF90DF90CF900C944F7DBC01209155037A
:1057B00030915603409155035091560324173507F5
:1057C00031F481E02617370709F080E008959A0147
:1057D000F1CF0F930FB70F9300916E000F930B7FD4
:1057E00000936E0000916F000D7F00936F000F9388
:1057F0000BB70F930CB70F921F922F933F934F93BA
:105800005F936F937F938F939F93AF93BF93EF9328
:10581000FF9311240E945832FF91EF91BF91AF91F5
:105820009F918F917F916F915F914F913F912F91B8
:105830001F900F900CBF0F910BBF0F910260F89457
:1058400000936F000F9100936E000F910FBF0F91A7
:10585000189500C000C080912E0580FF1FC0459A9A
:105860008FEF80930E0380912E0581FF1AC0479A17
:105870008FEF80930F0380912E0582FF15C02A9829
:105880008FEF8093100380912E0583FF10C028981E
:105890008FEF8093110300C000C00895459881E008
:1058A000E0CF479881E0E5CF2A9A81E0EACF289AB5
:1058B00081E0EFCF80918A02982F977F90938A02A0
:1058C000982F937081E011F080E008955E9A08951A
:1058D0005E9880918A02886080938A020895E82FFA
:1058E000F0E021E030E0082E02C0220F331F0A94BE
:1058F000E2F72095309590918A02922390938A0244
:10590000E952FE4F2081922321E019F020E0822FFE
:105910000895813079F038F08230C9F7159A909166
:105920002D059B7F04C05E9A90912D059E7F9093DC
:105930002D05EDCF5E9A90912D059D7FF8CF80E0EB
:105940000E946F2C81E00E946F2C82E00E946F2CDD
:105950000C945A2C813079F070F0823071F021E093
:1059600030E001C0220F8A95EAF780918A02822BEB
:1059700080938A0208955E98F2CF1598F0CFCF9267
:10598000DF92EF92FF920F931F93CF93C82F6AE29B
:105990007AE00E948D9DC11102C00E94677E82E262
:1059A0009AE00E94567D83EC99E00E94567D8AE041
:1059B0000E944F7D60E17AE08C2F0E948D9DC11185
:1059C00002C00E94677E83EF99E00E94567D8C2F73
:1059D0000E94B19D8C2F0E94FF7D8C2F0E94297EFA
:1059E0008C2F0E94DD7D8C2F0E94A57D68ED79E0D3
:1059F0008C2F0E948D9D01E812E0C12CD12C7601E4
:105A0000C11102C00E94677E8FEC99E00E94567D12
:105A1000C701B6010E94DF9AF80160817181072EEB
:105A2000000C880B990B0E9447D4AB01BC018CEC95
:105A300099E00E94907DF8016281738189EC99E080
:105A40000E9419810C5F1F4FCA94CD28CE28CF2801
:105A500051F48C2FCF911F910F91FF90EF90DF9019
:105A6000CF900C94CA80C12CD12C7601C394C8CF9E
:105A7000853F910514F085EF90E09093C2058093E7
:105A8000C1050C942C1F8091E8029091E9020C94BE
:105A9000382DCF93DF9380918002811119C0C0917E
:105AA0000801D0910901219720E030E040E05FE358
:105AB0006091BD057091BE058091BF059091C005B4
:105AC0000E9449DB0E943EDC21E06C177D070CF050
:105AD00020E0822FDF91CF910895AF92BF92CF92B5
:105AE000DF92EF92FF920F931F93CF93DF93CDEB53
:105AF000DBE001EE15E08DECA82E8BE0B82EC12C7A
:105B0000D12C7601C39469917991899199910E94E0
:105B100045D4288939894A895B890E94A6D40E9484
:105B200045DCF80161937193819391938F01C616BF
:105B3000D706E806F90610F46B017C01AC16BD0629
:105B400011F76FEF7FEFCB01A70196010E9488DA72
:105B50002093F1053093F2054093F3055093F4053B
:105B6000DF91CF911F910F91FF90EF90DF90CF9039
:105B7000BF90AF9008950F931F93CF93DF9301EDE4
:105B80001BE0CAEFD5E0F80121913191419151918B
:105B90008F0160E070E080E89FE30E94CCDB6993B6
:105BA000799389939993F6E0CA30DF0761F70E94F1
:105BB0006D9DDF91CF911F910F910C946D2D0C94E1
:105BC000BB2D0C94BB2D0C94BB2D0C94BB2D909134
:105BD0007B1180917C11981306C080910A069091E8
:105BE0000B06892B19F00E9444B1F1CF08959091D2
:105BF0007B1180917C11981308C080910A069091C6
:105C00000B06892B11F40C949F2C0E9444B1EFCF0A
:105C10002F923F924F925F926F927F928F929F92BC
:105C2000AF92BF92CF92DF92EF92FF920F931F93AA
:105C3000CF93DF93CDB7DEB76C970FB6F894DEBF86
:105C40000FBECDBF8C015B015A834983FC01EA5B27
:105C5000FF4F208131814281538129873A874B87C9
:105C60005C87CA01B9010E9445D46B017C01D50152
:105C70002D913D914D915C910E94A6D40E94B5DB7F
:105C80002B013C01E981FA812081318142815381DC
:105C9000C701B6010E94A6D40E94B5DB4B015C018E
:105CA000C301B2010E9445DC698B7A8B8B8B9C8B84
:105CB000683771058105910540F428E730E040E040
:105CC00050E0298B3A8B4B8B5C8BC501B4010E9451
:105CD00045DC6D877E878F87988B683771058105D6
:105CE000910540F448E750E060E070E04D875E8742
:105CF0006F87788BF801EE5AFF4F408051806280A9
:105D00007380C301B2010E9447D469837A838B8375
:105D10009C8369897A898B899C890E9445D46D8B83
:105D20007E8B8F8B988F20E030E0A90169817A818A
:105D30008B819C810E9440D4882309F4E1C1A70192
:105D40009601C701B6010E94A6D44B015C012D89C2
:105D50003E894F89588DCA01B9010E94A6D49B0182
:105D6000AC01C501B4010E9448DB4B015C012981F3
:105D70003A814B815C81CA01B9010E9449DB9B01D8
:105D8000AC01C501B4010E94CCDB0E94B5DB0E94CE
:105D900045DC6D837E838F83988766277727CB01C9
:105DA00064197509860997090E9447D44B015C0163
:105DB0006D857E858F8598890E9445D42B013C0195
:105DC00020E030E0A901C501B4010E9440D488233D
:105DD00009F49AC1A3019201C301B2010E94A6D4A1
:105DE000698F7A8F8B8F9C8FA7019601C701B601AF
:105DF0000E94A6D49B01AC01698D7A8D8B8D9C8D00
:105E00000E9448DB6B017C01A5019401C501B4012E
:105E10000E9449DB9B01AC01C701B6010E94CCDBAB
:105E20000E9474DCD80195968D909D90AD90BC90A9
:105E30009897750164012D813E814F815885C21A62
:105E4000D30AE40AF50A0E9445DCC61AD70AE80A12
:105E5000F90AF7FE8EC02D893E894F89588DCA01F7
:105E6000B9010E94A6D46B017C0129813A814B8142
:105E70005C81CA01B9010E9449DB69877A878B87F7
:105E80009C8720E030E0A90169817A818B819C8127
:105E90000E9440D4882309F43BC1C501B4010E948B
:105EA00045D429853A854B855C850E94A6D4A701F7
:105EB00096010E9448DB6D837E838F839887A301C0
:105EC0009201C301B2010E94A6D49B01AC016D8175
:105ED0007E818F8198850E9449DB2B013C0120E067
:105EE00030E040E850E469817A818B819C810E9496
:105EF000A6D49B01AC01C301B2010E94CCDB0E947D
:105F0000B5DB2B013C0120E030E0A9010E94CCDC94
:105F100018161CF0412C512C3201C301B2010E9411
:105F200045DC6D837E838F83988786169706A80647
:105F3000B90620F48D829E82AF82B8866D817E8103
:105F40008F8198850E9445D429853A854B855C854B
:105F50000E94A6D4A70196010E9449DB0E940ADD97
:105F60000E9445DC69877A878B879C87C12CD12C5E
:105F7000760169857A858B859C8529893A894B8943
:105F80005C89621B730B840B950B0E9445D429819D
:105F90003A814B815C810E94CCDB20E034E244EF0B
:105FA00059E40E94A6D40E9445DC4B015C0169853E
:105FB0007A858B859C852D853E854F855889621B0A
:105FC000730B840B950B0E9445D429813A814B8138
:105FD0005C810E94CCDB20E034E244EF59E40E9473
:105FE000A6D40E9445DC2B013C013FE683169104B8
:105FF000A104B10408F090C0F401EE0FFF1FEE0FF2
:10600000FF1FE656F94F85919591A591B49189832B
:10601000292E3A2EBD8B4FE64416510461047104BB
:1060200008F083C0F201EE0FFF1FEE0FFF1FE656D0
:10603000F94F45915591659174919A01CB014D812C
:106040005E816F817885D80199964D935D936D93AC
:106050007C939C974C0D5D1D6E1D7F1DF80145A71F
:1060600056A767A770ABE65BFF4F49895A896B89D2
:106070007C894083518362837383D5968D929D92F0
:10608000AD92BC92D897F80141AE52AE63AE74AEF9
:10609000FD9649814083218232825D895383349603
:1060A000208331838283938369857A858B859C8560
:1060B000D1966D937D938D939C93D4973D962D852A
:1060C0003E854F85588920833183428353836C9664
:1060D0000FB6F894DEBF0FBECDBFDF91CF911F91F9
:1060E0000F91FF90EF90DF90CF90BF90AF909F9077
:1060F0008F907F906F905F904F903F902F9008957A
:1061000060E070E0CB0141CE60E070E0CB0188CE72
:1061100060E070E0CB01F3CEC501B4010E94D1185C
:106120006983272E382E9D8B76CFC301B2010E9442
:10613000D1189B0184CF90916F0081E091FD02C046
:1061400080E0089590916F009D7F90936F00089577
:10615000EFE6F0E08081826080830895CF93DF9343
:10616000CDB7DEB72C970FB6F894DEBF0FBECDBF0C
:106170000E949B309CE0E4E6F3E0DE011196019082
:106180000D929A95E1F781110E94A830CE010196F7
:106190000E94A12B2C960FB6F894DEBF0FBECDBF88
:1061A000DF91CF9108954F925F926F927F928F927D
:1061B0009F92AF92BF92CF92DF92EF92FF92409068
:1061C000620150906301609064017090650180905D
:1061D000660190906701A0906801B0906901C0903D
:1061E0006A01D0906B01E0906C01F0906D010E940B
:1061F0006D2D6091240170912501072E000C880BF4
:10620000990B0E9447D42AE037ED43E25CE30E94F9
:10621000A6D460935E0170935F01809360019093B8
:106220006101ACE0B1E090E080E0FC01EE59F64F96
:1062300045915591659174914D935D936D937D93C7
:10624000FC01EA5AF64F4591559165917491189663
:106250004D935D936D937C931B9704968C309105C1
:1062600021F70E94BB2DA301920160916201709100
:10627000630180916401909165010E9440D4811175
:106280001CC0A50194016091660170916701809125
:106290006801909169010E9440D481110EC0209143
:1062A0006A0130916B0140916C0150916D01C70101
:1062B000B6010E9440D4882381F00E94B09CFF90D8
:1062C000EF90DF90CF90BF90AF909F908F907F9096
:1062D0006F905F904F900C94AE30FF90EF90DF90F6
:1062E000CF90BF90AF909F908F907F906F905F9076
:1062F0004F900895CF93C82F0E949B3094E0C99F80
:1063000090011124F901E85AFC4F2C593C4FD90156
:106310004D915D916D917C91408351836283738334
:1063200091E090935703882319F0CF910C94A830F3
:10633000CF910895CF93DF938091F402329B4BC0AD
:1063400081608093F4028091F402339B46C08260A6
:106350008093F4028091F402349B41C08460809366
:10636000F402C0914803C0FF10C080912E0580FF49
:106370000CC08091F40280FF08C08091710581609B
:106380008093710580E00E947A31C1FF10C0809136
:106390002E0581FF0CC08091F40281FF08C080911E
:1063A000710582608093710581E00E947A31C2FF9D
:1063B00018C080912E0582FF14C08091F40282FFE4
:1063C00010C08091710584608093710582E0DF9137
:1063D000CF910C947A318E7FB4CF8D7FB9CF8B7FE4
:1063E000BECFDF91CF9108950E949B301092F505AA
:1063F0001092F6051092F7051092F80581110C9491
:10640000A83008950F931F9380917B1190917C1178
:10641000891B8F7009F449C090917811992361F01C
:10642000833040F48FEF890F29F08093781190E04A
:1064300080E038C01092781180917C112BE5829F0A
:10644000C0011124845F994FFC01208120FDEFCF12
:106450004091F5055091F6056091F7057091F805AA
:10646000E95AFF4F0081118122813381401B510B7A
:10647000620B730B4093F5055093F6056093F70597
:106480007093F80520917C112F5F2F702093791164
:1064900030917C1120917A11321304C0209179112E
:1064A00020937A111F910F9108950E94F431BFCF6C
:1064B0002F923F924F925F926F927F928F929F9214
:1064C000AF92BF92CF92DF92EF92FF920F931F9302
:1064D000CF93DF93CDB7DEB763970FB6F894DEBFE7
:1064E0000FBECDBF8FEF9FEF909389008093880000
:1064F0002AE02983312C212C7894809151039091AA
:106500005203A0915303B0915403892B8A2B8B2BF8
:1065100009F0C2C1809157038823D1F080915503BF
:106520009091560310925703892B91F010925603C5
:10653000109255031092480390917B1180917C1129
:10654000981731F080917C118F5F8F7080937C1150
:106550008091550390915603892B09F49DC1409178
:106560004D0350914E0360914F0370915003809101
:10657000490390914A03A0914B03B0914C030091C1
:106580003F0310E030E020E0841B950BA60BB70B17
:10659000081719072A073B0710F4D901C8018A8B8D
:1065A000840F951FA61FB71F80934D0390934E0332
:1065B000A0934F03B0935003E1E0C0901603D09036
:1065C0001703E0901803F09019038091260390912F
:1065D0002703A0912803B0912903C80ED91EEA1EF3
:1065E000FB1EC0922603D0922703E0922803F0926C
:1065F0002903F7FC33C040910E03042E000C550B09
:10660000660B770B8091640390916503A0916603FC
:10661000B0916703840F951FA61FB71F8093640373
:1066200090936503A0936603B09367038091120370
:1066300090911303A0911403B0911503B701A60123
:10664000481B590B6A0B7B0BDB01CA0180932603A5
:1066500090932703A0932803B093290300911A0372
:1066600010911B0320911C0330911D0380912A037C
:1066700090912B03A0912C03B0912D03080F191FAB
:106680002A1F3B1F00932A0310932B0320932C03F4
:1066900030932D0337FD33C040910F03042E000CBF
:1066A000550B660B770B8091680390916903A0915D
:1066B0006A03B0916B03840F951FA61FB71F8093C9
:1066C000680390936903A0936A03B0936B0380916E
:1066D000120390911303A0911403B09115032801A4
:1066E0003901481A590A6A0A7B0AD301C201809308
:1066F0002A0390932B03A0932C03B0932D03409176
:106700001E0350911F03609120037091210380911B
:106710002E0390912F03A0913003B0913103480FC5
:10672000591F6A1F7B1F40932E0350932F036093C2
:1067300030037093310377FD33C080901003082C31
:10674000000C9908AA08BB0880916C0390916D0316
:10675000A0916E03B0916F03880D991DAA1DBB1DFA
:1067600080936C0390936D03A0936E03B0936F03BB
:106770008091120390911303A0911403B09115031B
:106780003A014B01681A790A8A0A9B0AD401C301AB
:1067900080932E0390932F03A0933003B093310383
:1067A0008090220390902303A0902403B0902503AF
:1067B0008091320390913303A0913403B09135035B
:1067C000880D991DAA1DBB1D80933203909333033E
:1067D000A0933403B0933503B7FD33C04090110349
:1067E000042C000C55086608770880907003909080
:1067F0007103A0907203B0907303840C951CA61CC7
:10680000B71C8092700390927103A0927203B092B1
:1068100073038090120390901303A0901403B09020
:1068200015032C013D01481859086A087B085301DB
:1068300042018092320390923303A0923403B092CB
:106840003503E11104C0E0918400F0918500F7FE6A
:106850005F9A37FF469A77FF2B9AB7FF299AE09104
:106860008400F0918500E0918400F0918500F7FEAE
:106870005F9837FF469877FF2B98B7FF29985A887B
:10688000552021F080918400909185002A89215023
:106890002A8BE0E0211191CE809151039091520317
:1068A000A0915303B0915403892B8A2B8B2B11F0A9
:1068B0000C94123B40905503509056035B8A4A8AD1
:1068C000452811F40C94843B80914D0390914E0324
:1068D000A0914F03B09150034091490350914A0356
:1068E00060914B0370914C0384179507A607B70777
:1068F00008F44DC0109256031092550310924803AD
:1069000090917B1180917C11981711F40C94843B29
:1069100080917C118F5F8F7080937C1130EDC32E3E
:1069200037E0D32EE12CF12C809155039091560342
:10693000892B11F00C940A3B0E940232909356036B
:1069400080935503892B11F40C940A3B4090550316
:10695000509056035B8A4A8AD2018C9183FF09C505
:10696000C20145960E947618109256031092550364
:106970001092480390917B1180917C119817E1F25D
:1069800080917C118F5F8F7080937C11D5CF409167
:1069900044035091450360914603709147034817A3
:1069A00059076A077B0708F40FC2409140035091D2
:1069B00041036091420370914303EA89FB8985A9F1
:1069C00096A9A7A9B0AD481759076A077B0708F031
:1069D000D1C1411551056105710509F066C080906E
:1069E0008F0290909002A0909102B090920280E26B
:1069F00093E1A1E0FC0105911591259134910815D1
:106A000019052A053B0558F4B694A79497948794E2
:106A1000AA0F0496ECE3F3E1E817F90759F7A093FE
:106A20003F03F0E28F169104A104B10428F480E240
:106A3000882E912CA12CB12C20E2821A9108A10859
:106A4000B108811438E09306A104B10408F49BC195
:106A5000A4E09A9EC0011124805E904FFC01329602
:106A600025913491B82DEE27B39F8001B29F010D7F
:106A70001E1F06940E1F1E1F112430E020E0FC0193
:106A8000C590D490F12CE12CC01AD10AE20AF30A85
:106A90004C0D5D1D6E1D7F1D4093400350934103BF
:106AA00060934203709343033FCF10E00A81942F19
:106AB000852E862FBC81AD81FE81EF8138852985A9
:106AC0004B80E0918B02E99FA12DFF2730918C0232
:106AD000399FA00DF11D10908D02199EF00DE89DBB
:106AE000A00DF11D389DF00DE89FF00D4A2EBF2F2F
:106AF0004A9EE12D332722274F9EE00D311D211F95
:106B0000BA9FE00D311D211FBF9F300D211D432E67
:106B1000B22F4A9E012D332722274F9E000D311D93
:106B2000211FBA9F000D311D211FBF9F300D211D58
:106B3000432EB22FEE2790918F0280909002809189
:106B400091020090A003012A09F484C030919C03B3
:106B5000349DE119910B810A810B20919D03249DA5
:106B6000E0199109810A810B00919E03049D9019FF
:106B70008108810B3B9FE0199109810A810B2B9FB2
:106B800090198108810B0B9F801881094A9E012D65
:106B9000332722274F9E000D311D211FBA9F000D64
:106BA000311D211FBF9F300D211D432EB22F30916B
:106BB0009803349DE10D911F811E811F209199033F
:106BC000249DE00D911D811E811F00919A03049D5B
:106BD000900D811C811F3B9FE00D911D811E811F27
:106BE0002B9F900D811C811F0B9F800C811D4A9E45
:106BF000012D332722274F9E000D311D211FBA9FE3
:106C0000000D311D211FBF9F300D211D432EB22FBE
:106C100030919403349DE119910B810A810B2091ED
:106C20009503249DE0199109810A810B0091960337
:106C3000049D90198108810B3B9FE0199109810AFD
:106C4000810B2B9F90198108810B0B9F8018810964
:106C50000C94AC3630919C03349DE10D911F811E44
:106C6000811F20919D03249DE00D911D811E811F98
:106C700000919E03049D900D811C811F3B9FE00DA0
:106C8000911D811E811F2B9F900D811C811F0B9FC9
:106C9000800C811D4A9E012D332722274F9E000D17
:106CA000311D211FBA9F000D311D211FBF9F300DC7
:106CB000211D432EB22F30919803349DE119910B81
:106CC000810A810B20919903249DE0199109810A81
:106CD000810B00919A03049D90198108810B3B9FC1
:106CE000E0199109810A810B2B9F90198108810B72
:106CF0000B9F801881094A9E012D332722274F9E22
:106D0000000D311D211FBA9F000D311D211FBF9F96
:106D1000300D211D432EB22F30919403349DE10D8F
:106D2000911F811E811F20919503249DE00D911DCF
:106D3000811E811F00919603049D900D811C811F6F
:106D40003B9FE00D911D811E811F2B9F900D811C8B
:106D5000811F0B9F800C811D11244B820A83BC83F1
:106D6000AD83FE83EF8338872987982C892EB12C39
:106D7000A82E3DCEAA89BB89D1968D909D90AD90CD
:106D8000BC90D49734CED501C401B695A7959795FC
:106D900087958C7F805E944FFC01C590D490FC0158
:106DA000329625913491E82DE770E29FC001E39F70
:106DB000900D112403E0969587950A95E1F7C81A7E
:106DC000D90AF12CE12C64CE40913B0350913C0355
:106DD00060913D0370913E03481759076A077B078E
:106DE00008F031C28090360390903703A0903803AA
:106DF000B090390380913A03EA89FB8981117CC004
:106E0000EF5BFF4FE080F18002811381EA89FB890B
:106E1000E25BFF4F2081318142815381AA89BB8986
:106E2000D1966D917D918D919C91D4970E947F1800
:106E3000B1E0B0933A03EA89FB8941A952A963A959
:106E400074A980E293E1A1E0FC01059115912591DF
:106E50003491041715072607370758F47695679578
:106E600057954795AA0F0496ECE3F3E1E817F90765
:106E700059F7A0933F03403251056105710520F495
:106E800040E250E060E070E0405251096109710950
:106E90004115F8E05F076105710508F4B4C124E00D
:106EA000529FC0011124805E904FFC0132962591C3
:106EB0003491AA27439FF001429FE10DFA1F0694E7
:106EC000EA1FFA1F1124AF0170E060E0FC01C590D9
:106ED000D490F12CE12CC41AD50AE60AF70A8C0CDE
:106EE0009D1CAE1CBF1C8092360390923703A0926B
:106EF0003803B092390318CD81AD92ADA3ADB4ADD6
:106F000088169906AA06BB0608F073C1811491047D
:106F1000A104B10449F440918F0250919002609114
:106F20009102709192028DCFA0E0BA85982D492DE3
:106F30008A2DFB85EC857D856E855F85388929895D
:106F400050918B02599F712D662730918C02399F89
:106F5000700D611D10908D02199E600D549F700D73
:106F6000611D349F600D589F600DF72FE62FF79F2E
:106F7000512D33272227F69F500D311D2A1FE79FE1
:106F8000500D311D2A1FE69F300D211DF32FE22FDA
:106F9000F79FB12D33272227F69FB00D311D2A1FF1
:106FA000E79FB00D311D2A1FE69F300D211DF32FE5
:106FB000E22F552790918F0240919002809191028B
:106FC0000090A0030A2A09F484C030919C033F9FDB
:106FD00051199A0B4A0B8A0B20919D032F9F501930
:106FE00091094A0B8A0BB0919E03BF9F90194109EA
:106FF0008A0B3E9F501991094A0B8A0B2E9F9019BC
:1070000041098A0BBE9F40198109F79FB12D332793
:107010002227F69FB00D311D2A1FE79FB00D311DAD
:107020002A1FE69F300D211DF32FE22F3091980388
:107030003F9F510D9A1F4A1F8A1F209199032F9F2E
:10704000500D911D4A1F8A1FB0919A03BF9F900D4A
:10705000411D8A1F3E9F500D911D4A1F8A1F2E9F62
:10706000900D411D8A1FBE9F400D811DF79FB12DC0
:1070700033272227F69FB00D311D2A1FE79FB00D41
:10708000311D2A1FE69F300D211DF32FE22F309175
:1070900094033F9F51199A0B4A0B8A0B2091950339
:1070A0002F9F501991094A0B8A0BB0919603BF9FED
:1070B000901941098A0B3E9F501991094A0B8A0B7E
:1070C0002E9F901941098A0BBE9F401981090C948B
:1070D000EB3830919C033F9F510D9A1F4A1F8A1F26
:1070E00020919D032F9F500D911D4A1F8A1FB09123
:1070F0009E03BF9F900D411D8A1F3E9F500D911D05
:107100004A1F8A1F2E9F900D411D8A1FBE9F400D52
:10711000811DF79FB12D33272227F69FB00D311D1A
:107120002A1FE79FB00D311D2A1FE69F300D211D3C
:10713000F32FE22F309198033F9F51199A0B4A0B7E
:107140008A0B209199032F9F501991094A0B8A0BA2
:10715000B0919A03BF9F901941098A0B3E9F501925
:1071600091094A0B8A0B2E9F901941098A0BBE9FE9
:1071700040198109F79FB12D33272227F69FB00DC3
:10718000311D2A1FE79FB00D311D2A1FE69F300DCC
:10719000211DF32FE22F309194033F9F510D9A1F31
:1071A0004A1F8A1F209195032F9F500D911D4A1F42
:1071B0008A1FB0919603BF9F900D411D8A1F3E9F6D
:1071C000500D911D4A1F8A1F2E9F900D411D8A1F31
:1071D000BE9F400D811D1124BA87FB87EC877D87F8
:1071E0006E875F87388B298B542F492F70E0682F6B
:1071F00028CE2A893B89225B3F4FD9014D915D9171
:107200006D917C911ECEDB01CA01B695A79597952D
:1072100087958C7F805E944FFC01C590D490FC01D3
:107220003296259134914770429FC001439F900D43
:107230001124A3E096958795AA95E1F7C81AD90A73
:10724000F12CE12C4CCE8091260190912701A09148
:107250002801B0912901B7FF61C0EA89FB89EA5B87
:10726000FF4FC080D180E280F38080E293E121E093
:10727000FC0145915591659174914C155D056E0524
:107280007F0558F4F694E794D794C794220F049698
:107290004CE353E14817590759F720933F0350E255
:1072A000C516D104E104F10428F470E2C72ED12CF4
:1072B000E12CF12C60E2C61AD108E108F108C114F2
:1072C00078E0D706E104F10408F431C0A4E0DA9EC6
:1072D000C0011124805E904FFC01329625913491BB
:1072E000BC2D6627B39FA001B29F410D561F069487
:1072F000461F561F112470E060E0FC0185919491B7
:10730000B0E0A0E0841B950BA60BB70B8093260181
:1073100090932701A0932801B0932901C0902601E2
:10732000D0902701E0902801F0902901FDCAD701F3
:10733000C601B695A795979587958C7F805E944FEB
:10734000FC0125913491FC01329645915491EC2D2C
:10735000E770E49FC001E59F900D112463E09695CE
:1073600087956A95E1F7281B390BC901B0E0A0E0C9
:10737000CDCFEA89FB8985889688A788B08C81E083
:1073800081149104A104B10409F480E0AA89BB89A5
:107390005996CD90DD90ED90FC905C97C114D1048E
:1073A000E104F10409F08260EA89FB89458D568D7C
:1073B000678D70A1411551056105710509F0846063
:1073C00080934803109236031092370310923803CB
:1073D000109239031092400310924103109242031D
:1073E00010924303EA89FB8985A196A1A7A1B0A5C4
:1073F0008093490390934A03A0934B03B0934C03AB
:10740000442455243201481A590A6A0A7B0A4092D8
:10741000260350922703609228037092290340921A
:107420002A0350922B0360922C0370922D034092FA
:107430002E0350922F03609230037092310341A0CB
:1074400052A063A074A0440C551C661C771C880CC9
:10745000991CAA1CBB1C8092160390921703A09241
:107460001803B0921903CC0CDD1CEE1CFF1CC0925B
:107470001A03D0921B03E0921C03F0921D03440FE9
:10748000551F661F771F40931E0350931F03609381
:1074900020037093210340922203509223036092B1
:1074A000240370922503880F991FAA1FBB1F809386
:1074B000120390931303A0931403B0931503109237
:1074C0004D0310924E0310924F031092500381A56A
:1074D00092A5A3A5B4A58093440390934503A093DC
:1074E0004603B093470385A596A5A7A5B0A98093A9
:1074F0003B0390933C03A0933D03B0933E03EB5BAF
:10750000FF4F808190912E05891721F080932E05E1
:107510000E94292C80912C0581110E949A314424CB
:107520004A94542C320140922601509227016092D5
:10753000280170922901EA89FB89FD96E080F1809B
:1075400002811381AA89BB89D1962D913D914D91DC
:107550005C91D4976D01BAE4CB0ED11CF601608129
:107560007181828193810E947F1810923A03D60123
:107570004D915D916D917C9180E293E1A1E0FC01E0
:1075800005911591259134910417150726073707A2
:1075900058F47695679557954795AA0F0496ECE3AE
:1075A000F3E1E817F90759F7A0933F03403251057B
:1075B0006105710520F440E250E060E070E0405267
:1075C0005109610971094115F8E05F07610571050D
:1075D00008F478C024E0529FC0011124805E904FCF
:1075E000FC01329625913491AA27439FF001429FD6
:1075F000E10DFA1F0694EA1FFA1F1124AF0170E093
:1076000060E0FC01C590D490F12CE12CC41AD50A9D
:10761000E60AF70AC0925103D0925203E092530354
:10762000F09254038091510390915203A09153031F
:10763000B0915403AC01BD01009731E0A307B1053F
:1076400020F04FEF5FEF60E070E0841B950BA60B1E
:10765000B70B8093510390935203A0935303B093BD
:107660005403F89480918400909185004096A981FC
:10767000A150A983AA2309F445C0240E351E28165B
:10768000390610F40C947C323092890020928800E4
:10769000789463960FB6F894DEBF0FBECDBFDF912E
:1076A000CF911F910F91FF90EF90DF90CF90BF90FF
:1076B000AF909F908F907F906F905F904F903F9092
:1076C0002F900895DB01CA01B695A79597958795E8
:1076D0008C7F805E944FFC01C590D490FC01329663
:1076E000259134914770429FC001439F900D112412
:1076F00033E0969587953A95E1F7C81AD90AF12CA7
:10770000E12C88CF1C01C0CF80EDC82E87E0D82E99
:10771000E12CF12C0C949C34CF93DF9380917B115E
:1077200090917C11891B80958F7019F40E9444B14F
:10773000F5CF80917B118F5F8F70A0917B119BE5BE
:10774000A99FD0011124FD01E45FF94FEF011992C7
:107750009A95E9F798E09083AF5DB94F90E1EDE736
:10776000F1E101900D929A95E1F720917B119091B2
:107770007C11291303C094E69093781180937B11B8
:10778000DF91CF910C94A830FC012081318142819E
:1077900053816091DD0B7091DE0B8091DF0B909136
:1077A000E00B0E94A6D40E94D1DC609389117093F3
:1077B0008A1180938B1190938C1190917B11809101
:1077C0007C1198130C948C3B0E94E72D0E949B30F7
:1077D0004091891150918A1160918B1170918C1197
:1077E000409370035093710360937203709373031B
:1077F00081110C94A83008954F925F926F927F92FE
:107800008F929F92AF92BF92CF92DF92EF92FF92B0
:10781000CF93DF93EC012091DD0B3091DE0B409193
:10782000DF0B5091E00B6C857D858E859F850E94D6
:10783000A6D40E94D1DC6B017C012091D90B309140
:10784000DA0B4091DB0B5091DC0B688579858A85DA
:107850009B850E94A6D40E94D1DC4B015C01209143
:10786000D50B3091D60B4091D70B5091D80B6C8132
:107870007D818E819F810E94A6D40E94D1DC2B0144
:107880003C012091D10B3091D20B4091D30B509100
:10789000D40B688179818A819B810E94A6D40E9441
:1078A000D1DC60937D1170937E1180937F11909352
:1078B00080114092811150928211609283117092D6
:1078C00084118092851190928611A0928711B092B6
:1078D0008811C0928911D0928A11E0928B11F09296
:1078E0008C1190917B1180917C11981781F0DF9120
:1078F000CF91FF90EF90DF90CF90BF90AF909F908F
:107900008F907F906F905F904F900C948C3B0E9473
:10791000E72D0E949B30C82F8DE791E10E947618D9
:10792000CC2381F0DF91CF91FF90EF90DF90CF904B
:10793000BF90AF909F908F907F906F905F904F908F
:107940000C94A830DF91CF91FF90EF90DF90CF9013
:10795000BF90AF909F908F907F906F905F904F906F
:107960000895CF92DF92EF92FF92CF93DF93C82FCB
:107970000E949B3094E0C99FE0011124FE01EC5964
:10798000FC4FC080D180E280F38081110E94A8303A
:10799000C650DA4FC701B6010E9447D42881398109
:1079A0004A815B810E94A6D4DF91CF91FF90EF9036
:1079B000DF90CF900895CF92DF92EF92FF92CF9316
:1079C000DF93C82F0E949B3094E0C99FE0011124EF
:1079D000FE01E85AFC4FC080D180E280F380811123
:1079E0000E94A830C650DA4FC701B6010E9447D4A2
:1079F000288139814A815B810E94A6D4DF91CF9191
:107A0000FF90EF90DF90CF900895CF93DF931F9278
:107A1000CDB7DEB7898360E0CE0101960E94CF1911
:107A200061E0CE0101960E94CF1962E0CE0101967D
:107A30000E94CF1989810F90DF91CF9108954F92C5
:107A40005F926F927F928F929F92AF92BF92CF92EE
:107A5000DF92EF92FF920F931F93CF93DF93CDB7F7
:107A6000DEB72C970FB6F894DEBF0FBECDBF2B014B
:107A70003C0129873A874B875C8747015801F6010B
:107A8000E080F1800281138120E030E0A901B7019C
:107A9000C8010E9440D4882309F484C05E2D4F2D74
:107AA000302F212F852F942FA32FB22F89839A83D4
:107AB000AB83BC8320E030E0A901B701C8010E947C
:107AC00040D4811104C0E12CF12C00E810E4C7017E
:107AD000D8018D839E83AF83B887A50194016091FF
:107AE0006A0170916B0180916C0190916D010E940F
:107AF00040D487FF0CC080926A0190926B01A092E3
:107B00006C01B0926D01CE0105960E94D522409283
:107B100062015092630160926401709265018985EF
:107B20009A85AB85BC858093660190936701A0938D
:107B30006801B0936901CE0101960E94D522A5018A
:107B4000940160916A0170916B0180916C01909138
:107B50006D010E94CCDC181664F480926A01909248
:107B60006B01A0926C01B0926D01CE0105960E944E
:107B7000D5220E94E72D2C960FB6F894DEBF0FBEDB
:107B8000CDBFDF91CF911F910F91FF90EF90DF90CC
:107B9000CF90BF90AF909F908F907F906F905F90AD
:107BA0004F90089550E040E035E023E47BCF0C9403
:107BB0006D9D4F925F926F927F928F929F92AF9244
:107BC000BF92DF92EF92FF920F931F93CF93DF93B9
:107BD000D82EC82FD0E0FE01E755F44D6491062E53
:107BE000000C770B880B990B0E9447D42B013C01AA
:107BF0007E01EE0CFF1CEE0CFF1CF701E257F94F63
:107C00002591359145915491C301B2010E94A6D4AA
:107C10004B015C01F701EE57F94F65917591859124
:107C2000949120E030E040EC5FE30E94A6D4A301F1
:107C300092010E94A6D4AB01BC0100E010E09801C3
:107C40008D2D0E9417C620E030E0A901C501B401C6
:107C50000E9440D4882309F446C0B501A40170589D
:107C600000E010E098018D2D0E9417C6A501940137
:107C7000C501B4010E9449DB4B015C01C158D94FD9
:107C8000FE01C491C11107C00E94677E8DE596E098
:107C90000E94567DCAE0DD2039F0F1E060E070E03E
:107CA00080E793E4DF1204C060E070E88BE395E4C2
:107CB00020E030E040E752E40E94CCDB2B013C01A5
:107CC0006C2F70E090E080E00E9445D49B01AC01F5
:107CD000C301B2010E94CCDB8B019C01B501A40160
:107CE0008D2D0E9417C681E090E001C0880FDA94C4
:107CF000EAF790912D05982B90932D0590916F02A6
:107D0000892B80936F02F701EF5AF94F8591959176
:107D1000A591B491E701CE59DE4F88839983AA8358
:107D2000BB830E94D73DF701E059FD4F88819981BF
:107D3000AA81BB8180839183A283B383DF91CF919A
:107D40001F910F91FF90EF90DF90BF90AF909F90A9
:107D50008F907F906F905F904F9008954F925F92B9
:107D60006F927F928F929F92AF92BF92CF92DF924B
:107D7000EF92FF920E949B30F82E80917C118093AD
:107D80007B1180937A118093791184E68093781126
:107D90000E94F43180ED93E090930B0680930A06E5
:107DA000F1100E94A83081E0809357030E94E72DD4
:107DB00080E00E94B13C2B013C014092F5025092C0
:107DC000F6026092F7027092F80281E00E94B13CE4
:107DD0004B015C018092F9029092FA02A092FB02A0
:107DE000B092FC0282E00E94B13C6B017C01C09227
:107DF000FD02D092FE02E092FF02F092000383E0C7
:107E00000E94B13C40926201509263016092640111
:107E1000709265018092660190926701A09268015C
:107E2000B0926901C0926A01D0926B01E0926C013C
:107E3000F0926D0160936E0170936F0180937001F9
:107E400090937101FF90EF90DF90CF90BF90AF9033
:107E50009F908F907F906F905F904F900C94D73D44
:107E600087E396E00E94567D86B161E376E082FB6F
:107E7000882780F90E94752286B16BE276E083FB49
:107E8000882780F90E94752286B165E276E08295A6
:107E900081700C94752280912C05882331F062E06A
:107EA00070E080E090E00C94E8760895ADEBBBE0E4
:107EB00090E080E0FC01EF51F54F459155916591BF
:107EC00074914D935D936D937D93FC01EF52F54F4B
:107ED000459155916591749150964D935D936D9335
:107EE0007C935397FC01EF53F54F45915591659164
:107EF000749190964D935D936D937C9393970496B4
:107F000080319105B9F680E29EE4A0E0B0E0809374
:107F1000CD0B9093CE0BA093CF0BB093D00B80E002
:107F200090E0AAEFB3E48093F10B9093F20BA0934F
:107F3000F30BB093F40B8093F50B9093F60BA09397
:107F4000F70BB093F80B8093F90B9093FA0BA09377
:107F5000FB0BB093FC0B1092FD0B1092FE0B1092DA
:107F6000FF0B1092000C1092010C1092020C109258
:107F7000030C1092040C8AE097EDA3EABDE3809312
:107F8000DD059093DE05A093DF05B093E0058EEB51
:107F900090E090938202809381021092840210926A
:107FA000830286EE90E09093860280938502109281
:107FB0008802109287028FE892ECADE8B1E48093DA
:107FC000C4059093C505A093C605B093C7058CE979
:107FD00098EFA5E4BEE38093C8059093C905A093EC
:107FE000CA05B093CB0581E49CEBABECB3E4809382
:107FF000CC059093CD05A093CE05B093CF051092FC
:108000002C0510922B050E944B3F0E94D3300E94FA
:10801000677E80EA99E00C94567D809171058823F3
:1080200019F010927105089540E070E060E085E07D
:1080300096E00E9428810F931F938091A8058130BC
:1080400019F50E943CA10091F0021091F1022091DB
:10805000F2023091F302601B710B820B930B28EE3E
:1080600033E040E050E00E9488DA6091EC027091C9
:10807000ED028091EE029091EF02620F731F841F58
:10808000951F1F910F91089560916B0270916C0282
:1080900080916D0290916E02D6CF1092A805109239
:1080A000F0021092F1021092F2021092F30210927A
:1080B0006B0210926C0210926D0210926E0210927E
:1080C000EC021092ED021092EE021092EF0208956F
:1080D0008091A8058130F1F08230C9F40E941B40E4
:1080E0006093EC027093ED028093EE029093EF02A6
:1080F00081E08093A8050E943CA16093F0027093F8
:10810000F1028093F2029093F30281E008950E94BD
:108110004D40EECF80E008950E94DE9D0E940C77D6
:10812000882351F08091F91282FD06C087EE91E01C
:108130009093300580932F050C9468408091A8059A
:108140008150823070F41092A8050E943CA1609387
:108150006B0270936C0280936D0290936E0281E0CB
:10816000089580E008959C0197FF26C0EE27FF2721
:10817000E81BF90B2D398FEF38070CF05DC08DE24D
:1081800080936602CF0164E670E00E94F2DACB01D0
:108190002AE030E0B9010E94F2DA805D8093670244
:1081A000CF01B9010E94F2DACB01B9010E94F2DAE3
:1081B000805D809368022AC0283E83E03807B4F1CE
:1081C000C90168EE73E00E94F2DACB01EAE0F0E068
:1081D000BF010E94F2DA805D80936602C90164E605
:1081E00070E00E94F2DACB01BF010E94F2DA805DFA
:1081F00080936702C901BF010E94F2DACB01BF017F
:108200000E94F2DA805D80936802F901CF016AE092
:1082100070E00E94F2DA805D8093690286E692E067
:1082200008958DE237FDC5CF80E2C3CFF90180E22A
:10823000243631050CF0A4CF80E28093660280934F
:108240006702EA30F1056CF38DE237FF80E280933C
:108250006702CF016AE070E00E94F2DA605D60932D
:108260006802D4CF9C0197FD2DC080E224363105F1
:108270005CF0C90164E670E00E94F2DACB016AE0CA
:1082800070E00E94F2DA805D8093670280E22A301B
:1082900031055CF0EAE0F0E0C901BF010E94F2DACA
:1082A000CB01BF010E94F2DA805D80936802C901B0
:1082B0006AE070E00E94F2DA805D8093690287E6EE
:1082C00092E008953195219531098DE2DDCF0E942C
:1082D00047D40E943EDCCB010C9432410F931F9394
:1082E0000E943CA1009127051091280520912905A5
:1082F00030912A050115110521053105D9F5209187
:108300008F112223A1F1E0918D11215020938F1123
:1083100021E02E0F20938D1130919011231302C074
:1083200010928D1124E0E29FF0011124EF56FE4ED1
:10833000008111812281338100932305109324054C
:108340002093250530932605600F711F811D911D17
:1083500060932705709328058093290590932A053B
:108360008091250590912605892B09F0149A1F917B
:108370000F910895601B710B820B930B97FDF7CF44
:108380001498109227051092280510922905109232
:108390002A05EDCF0F931F93CF93DF938C01EB0151
:1083A00090918F1120919011921305C00E946E41FF
:1083B0000E94E128F5CF80918E1134E0839FF00177
:1083C0001124EF56FE4E11830083D383C2839F5F37
:1083D00090938F118F5F281739F080938E11DF9162
:1083E000CF911F910F91089510928E11F8CF63E9EC
:1083F00072E084E690E00E94CA416AEB72E084E693
:1084000090E00C94CA410E94563F0C94F7418111B0
:108410000C94F74168EB71E084E190E00C94CA4160
:108420004FE350E0BC0181E395E00C94AEDD8FE5B5
:1084300094E00C941042282F1092940580917F05AF
:1084400090918005A0918105B0918205B7FF08C089
:1084500010927F051092800510928105109282057E
:1084600080915F02882331F080917F0580937805A9
:1084700010928F05809172051816FCF4082E000CDE
:10848000990B821B910920917805022E000C330B69
:108490002817390794F097FF02C090E080E080939E
:1084A0007805092E000CAA0BBB0B80937F059093D7
:1084B0008005A0938105B09382058091780566239D
:1084C000A9F090917905891714F48093790520918A
:1084D0007905022E000C330B2C5F3F4F482F082EDE
:1084E000000C550B241735071CF484508093790534
:1084F00008958F929F92AF92BF92EF92FF920F9347
:108500001F93CF93DF93EC018B01E42EF22E809129
:10851000A1119091A2118C179D0709F443C02091DD
:108520005C0230915D0237FF04C010925D02109230
:108530005C0220E6C736D20709F03FC08A51974750
:1085400071F40E943CA16E517B4F8F4F9F4F6093FF
:10855000D6027093D7028093D8029093D902D09319
:10856000A211C093A11130E020E000937F05109389
:1085700080052093810530938205E0927905F09281
:108580007205CA51D74721F4109262021092D502A7
:1085900082E080934E0181E080938F0510925E020D
:1085A0001092E402DF91CF911F910F91FF90EF9015
:1085B000BF90AF909F908F90089527E7CA31D20760
:1085C00071F687569046D9F40E943CA18090D6025D
:1085D0009090D702A090D802B090D902681979097A
:1085E0008A099B0997FF0BC080912D058770873002
:1085F00031F40E94121FC2E0D3E48111B0CFCAE16E
:10860000D7E7ADCF20E040E070E060E08CE19FE490
:108610000E94794281E0809362021092610210927E
:108620006002089581E08093620280912D05877039
:10863000873051F010922D0510926F0283EA95E079
:108640009093300580932F0520E040E070E060E0DB
:1086500080EC93E40C94794220E040E070E060E02C
:108660008CE693E20C9479420E94492D882341F0D4
:1086700020E040E070E060E087E59DE40C94794202
:108680000C942C4321E020936202FC0180819181B3
:10869000A281B3818093020190930301A09304010E
:1086A000B093050120E040E070E060E080917A0541
:1086B00090917B050C947942CF93DF9300D000D04A
:1086C000CDB7DEB78DEC9CECACECBCE389839A8330
:1086D000AB83BC83CE0101960E9442430F900F9062
:1086E0000F900F90DF91CF910895CF93DF9300D03B
:1086F00000D0CDB7DEB78DEC9CECACECBDE389834C
:108700009A83AB83BC83CE0101960E9442430F90B3
:108710000F900F900F90DF91CF910895CF93DF933B
:1087200000D000D0CDB7DEB780E090E0A0E8BFE396
:1087300089839A83AB83BC83CE0101960E94424316
:108740000F900F900F900F90DF91CF910895CF93DE
:10875000DF9300D000D0CDB7DEB780E090E0A0E29C
:10876000B1E489839A83AB83BC83CE0101960E94D6
:1087700042430F900F900F900F90DF91CF9108958B
:1087800080914E01882341F030E020E041E06BE130
:1087900073E082E00E947C7380916F028770873063
:1087A00079F41092E50220E040E070E060E088EEAD
:1087B0009DE40E94794281E08093E4020C94DA22E5
:1087C000089520E040E070E060E08AE197E70C94D3
:1087D00079421092F9050E9435280C94E143CF9319
:1087E000DF93C091E802C7FD1FC084E0C802E0012A
:1087F0001124FE01EF57FD4F808191811816190653
:108800003CF4863F910514F085EF90E00E94382DEE
:10881000CF57DD4F8A819B818F3F910519F010F072
:108820008FEF90E08093F905DF91CF910C94E143B5
:108830008BE995E00E945BA50E94E1430C94DE9DCC
:108840000F931F93CF93DF93CDB7DEB76E970FB61D
:10885000F894DEBF0FBECDBF80919805282F082E5B
:10886000000C330BF901EE0FFF1FE050FF4F918119
:108870009F9390819F933F938F9385E492E09F9382
:108880008F938E010F5F1F4F1F930F930E94D7D3BB
:10889000C8010E9410420E94E1430FB6F894DEBF67
:1088A0000FBECDBF6E960FB6F894DEBF0FBECDBF24
:1088B000DF91CF911F910F910895CF93DF93E091B6
:1088C000D502EE2331F1E150E093D502AE2FB0E0B6
:1088D00099E0E99FF0011124E156FD4F278140E026
:1088E00070E060E0811103C046816281738189E09C
:1088F0008A9FE0018B9FD00D1124C156DD4F8881E6
:1089000099810E947942888580936202DF91CF919C
:108910000895DF91CF910C94E14381E00C945D4484
:108920002F923F924F925F926F927F928F929F927F
:10893000AF92BF92CF92DF92EF92FF920F931F936D
:10894000CF93DF9300D01F92CDB7DEB72090C10543
:108950003090C20561E081E00E941B4220917905C0
:108960002A83522E2B5F298382E085198B8381E035
:10897000782E7518452C419485E0682E65182A815B
:10898000211115C080917805882309F4D8C0809101
:108990004E01882309F46DC181E090917805911111
:1089A00080E024E044ED55E0642D0E94029E809119
:1089B000C1059091C2059093E9028093E8028A81F3
:1089C0008130F1F480917805813009F4DCC0809128
:1089D0004E01882309F443C011E08091780581306D
:1089E00009F010E08091E8029091E9020E94324182
:1089F00000E09C014DEC55E0672D812F0E948574AD
:108A00008091F9058093E8029A81923041F51092A5
:108A1000980580917805823009F4D0C080914E018C
:108A20008823E9F011E080917805823009F010E0A8
:108A30008091E80224E6829FC001112481589F4F53
:108A40006FEF70E00E94F2DA862F0E944B1C00E06C
:108A50009C0143EC55E06B81812F0E94857410E0EE
:108A600000E033E0F32EEA80E5180093E8028A8103
:108A70008F112CC0F801EE0FFF1FE455FA4F8591BE
:108A8000949190939A0580939905809178059A81A5
:108A9000891709F4CEC080914E018823B9F08FEE7A
:108AA00093E49F938F9389EB95E09F938F93EF923D
:108AB00081E0909178059F1180E08F930E944F2371
:108AC0000F900F900F900F900F900F908F2D0F5FC2
:108AD0001F4F94E0F92E843041F62114310409F43B
:108AE000C6C08A81853009F580917805853009F402
:108AF000AFC080914E018823C1F089EE93E49F932B
:108B00008F9380EB95E09F938F936F9281E090918C
:108B10007805953009F080E08F930E944F230F90E5
:108B20000F900F900F900F900F9086E09A819F5FAB
:108B30009A832981291323CF809372050EC08091D7
:108B4000730510927305882309F421CF0E948D4488
:108B500080918F05882309F41ACF0F900F900F9002
:108B6000DF91CF911F910F91FF90EF90DF90CF9009
:108B7000BF90AF909F908F907F906F905F904F903D
:108B80003F902F900895809173051092730588236C
:108B900009F41DCF0E94DF9E03E41DE225EF30E0C3
:108BA00050E040E068EE72E08DEC95E00E94A39FFB
:108BB00080918F05882309F40ACFCFCF8091730568
:108BC00010927305882309F429CF0E94DF9E6091DB
:108BD000E80270E090E080E00E9445D429EC38EC97
:108BE00048EC5EE30E94A6D420E030E040E05FE382
:108BF0000E9449DB0E9445DC4BEB842E4CE1942E15
:108C000053EFA52E5EE4B52E6B0114E6E12EF12C98
:108C100000E010E020E030E0A90168EE72E083ECB3
:108C200095E00E94EB9E80918F05882309F4F6CE93
:108C300094CF8091730510927305882309F42BCF8C
:108C40000E94EF4380918F05882309F424CF85CFBC
:108C50008091730510927305882309F44ACF0E940E
:108C6000E94380918F05882309F443CF76CF85E0CF
:108C70005DCF8091C1059091C2059093E9028093E8
:108C8000E802BECEEF92FF920F931F93CF93DF9334
:108C9000CDB7DEB765970FB6F894DEBF0FBECDBF78
:108CA0008091730510927305882379F00E948D449A
:108CB00065960FB6F894DEBF0FBECDBFDF91CF91A2
:108CC0001F910F91FF90EF90089560E085E00E9462
:108CD0001B420091790510E08AE3F82E90E2E92E1C
:108CE000011130C080914E01882341F030E020E036
:108CF00043E063E274E0812F0E947C73F982EA8290
:108D000042E150E064EE73E0CE0103960E94AED3E0
:108D10008C8987FD1C8A053069F480914E01882377
:108D200049F09E012F5F3F4F41E06AED73E0812FD4
:108D30000E947C730F5F1F5F153091F686E0809371
:108D40007205B6CF013051F480914E018823B1F203
:108D500030E020E041E066E174E0CDCF0230A9F4DC
:108D600080914E01882351F230E020E041E06BE039
:108D700074E0C1CF80914E01882309F4BFCF30E069
:108D800020E043E061E074E0B6CF033099F30430B3
:108D900009F0B4CF80914E01882309F4AFCF30E0C1
:108DA00020E041E066EE73E0A6CFEF92FF920F93D2
:108DB0001F93CF93DF93CDB7DEB765970FB6F894C7
:108DC000DEBF0FBECDBF809173051092730588235F
:108DD00079F00E948D4465960FB6F894DEBF0FBE01
:108DE000CDBFDF91CF911F910F91FF90EF9008952C
:108DF00060E085E00E941B420091790510E08AE363
:108E0000F82E90E2E92E01110CC080914E018823CA
:108E100041F030E020E043E069EC73E0812F0E94F4
:108E20007C73F982EA8242E150E062EC73E0CE01A9
:108E300003960E94AED38C8987FD1C8A013069F4A9
:108E400080914E01882349F09E012F5F3F4F41E002
:108E50006DEB73E0812F0E947C73F982EA8242E11C
:108E600050E069EB73E0CE0103960E94AED38C898B
:108E700087FD1C8A023069F480914E01882349F0F5
:108E80009E012F5F3F4F41E060EB73E0812F0E9416
:108E90007C73F982EA8242E150E068EA73E0CE0135
:108EA00003960E94AED38C8987FD1C8A033069F437
:108EB00080914E01882349F09E012F5F3F4F41E092
:108EC00064EA73E0812F0E947C730F5F1F5F15308F
:108ED00009F099CF84E0809372057DCFEF92FF92E5
:108EE0000F931F93CF93DF93CDB7DEB765970FB680
:108EF000F894DEBF0FBECDBF80917305109273054D
:108F0000882379F00E948D4465960FB6F894DEBFF1
:108F10000FBECDBFDF91CF911F910F91FF90EF90CA
:108F2000089560E085E00E941B420091790510E001
:108F30008AE3F82E90E2E92E01110CC080914E01D7
:108F4000882341F030E020E042E065E973E0812FC2
:108F50000E947C73F982EA8242E150E063E973E0A7
:108F6000CE0103960E94AED38C8987FD1C8A013006
:108F700069F480914E01882349F09E012F5F3F4F95
:108F800040E06AE873E0812F0E947C73F982EA82F4
:108F900042E150E066E873E0CE0103960E94AED352
:108FA0008C8987FD1C8A0230B1F480914E018823A0
:108FB00049F09E012F5F3F4F40E06DE773E0812F46
:108FC0000E947C730F5F1F5F153009F0B5CF84E0FE
:108FD0008093720599CF0330A9F780914E018823C1
:108FE00089F330E020E040E06BE673E0E8CFBF9229
:108FF000CF92DF92EF92FF920F931F93CF93DF9365
:1090000061E081E00E941B42C091790585E0C82E95
:10901000CC0ED4E0DC1B13E01C1B82E0F82EFC1A03
:1090200081E0E82EEC1ABC2EB194C11130C08091C1
:1090300078058823B1F080914E01882359F081E0B2
:1090400090917805911180E024E04EEC52E06B2D78
:109050000E94029ECF5FCC12E8CF85E0809372051C
:109060000CC08091730510927305882321F30E9430
:109070008D4480918F058823F1F2DF91CF911F916C
:109080000F91FF90EF90DF90CF90BF900895C13087
:10909000B9F5809178058130F1F080914E018823F7
:1090A000C9F2DD24D39480917805813009F0D12C68
:1090B0006091D10B7091D20B8091D30B9091D40B16
:1090C0000E94361D00E09C0143EC52E06E2D8D2D78
:1090D0000E948574BFCF8091730510927305882319
:1090E000E1F20E94DF9E45EE5DE261ED7BE083EC04
:1090F00092E00E945E9F80918F05882371F2BDCF20
:10910000C23009F07FC0809178058230E1F0809113
:109110004E01882309F49ECFDD24D39480917805F5
:10912000823009F0D12C6091D50B7091D60B8091D3
:10913000D70B9091D80B0E94361D00E09C0148EBA4
:1091400052E06F2DC4CF8091730510927305882370
:10915000F1F20E94DF9E43EE5DE265ED7BE088EB7D
:1091600092E00E945E9F80918F05882381F285CFD7
:10917000809178058330E1F080914E01882309F4D5
:1091800069CFDD24D39480917805833009F0D12C08
:109190006091D90B7091DA0B8091DB0B9091DC0B15
:1091A0000E94361D00E09C014DEA52E0612F8FCFF6
:1091B00080917305109273058823F1F20E94DF9E5F
:1091C00041EE5DE269ED7BE08DEA92E00E945E9FF8
:1091D00080918F05882381F250CF80917305109282
:1091E00073058823C9F00E94DF9E4FED5DE26DEDAF
:1091F0007BE082EA92E00E945E9F80918F05882347
:1092000059F03BCFC33009F4B3CFC43009F022CFBB
:1092100080917805843009F380914E01882309F408
:1092200019CFDD24D39480917805843009F0D12CB6
:109230006091DD0B7091DE0B8091DF0B9091E00B64
:109240000E94361D00E09C0142EA52E06D2F3FCFA4
:109250002F923F924F925F926F927F928F929F9246
:10926000AF92BF92CF92DF92EF92FF920F931F9334
:10927000CF93DF9300D000D000D0CDB7DEB761E050
:1092800081E00E941B4270907905672C85E0870D74
:109290008D8388E087198E8387E0582E571886E0E3
:1092A000482E471885E0382E371884E0282E2718D6
:1092B000711096C080917805882309F46AC0809166
:1092C0004E01882361F0662D619581E090917805CB
:1092D000911180E024E04EEC52E00E94029E2CEAC4
:1092E00035EC47E25EE36091C8057091C905809155
:1092F000CA059091CB050E94CCDB6093E00270938D
:10930000E1028093E2029093E3022CEA35EC47E21B
:109310005EE36091CC057091CD058091CE05909172
:10932000CF050E94A6D46093DC027093DD02809387
:10933000DE029093DF0285E07812AFC110929805AB
:1093400080917805853009F46CC180914E018823A5
:10935000C1F011E080917805853009F010E060914E
:10936000C4057091C5058091C6059091C7050E94FE
:10937000031D00E09C0144E752E0632D812F0E9411
:10938000857473948D81781293CF89E080937205F0
:109390000EC08091730510927305882309F48FCF56
:1093A0000E948D4480918F05882309F488CF2696EA
:1093B0000FB6F894DEBF0FBECDBFDF91CF911F91E6
:1093C0000F91FF90EF90DF90CF90BF90AF909F9064
:1093D0008F907F906F905F904F903F902F90089567
:1093E00081E0781230C0909178059130C9F0809179
:1093F0004E01882309F473CF61E0661981E0913052
:1094000009F080E09091D00526E932E0911102C088
:1094100022E932E001E049E952E00E9485745FCF21
:109420008091730510927305882309F38091D0050C
:1094300087258093D00583E080934E0180918F052E
:109440008823A9F2B4CF82E078121FC280917805F8
:10945000823009F466C080914E018823A9F011E0A2
:1094600080917805823009F010E08091560190914A
:1094700057010E94324162E0661900E09C014BE80E
:1094800052E0812F0E9485742CEA35EC47E25EE3BE
:109490006091C8057091C9058091CA059091CB056E
:1094A0000E94CCDB6093E0027093E1028093E202C1
:1094B0009093E3022CEA35EC47E25EE36091CC0541
:1094C0007091CD058091CE059091CF050E94A6D4D4
:1094D0006093DC027093DD028093DE029093DF02E2
:1094E00088E078124ECF10929805809178058830E8
:1094F00009F4B0C180914E01882309F442CF11E0F4
:1095000080917805883009F010E0809100019091F9
:1095100001010E94324100E09C0145E552E06E816C
:109520002DCF8091730510927305882309F493CF92
:1095300010E000E025EF30E050E040E066E571E04B
:109540008BE892E00E94A39F80918F05882309F405
:1095500082CF2DCF809178058330C9F080914E0164
:10956000882309F491CF11E080917805833009F0C8
:1095700010E080915001909151010E94324163E0CE
:10958000661900E09C0144E852E0812F46CF8091AB
:10959000730510927305882309F310E000E025EFAE
:1095A00030E050E040E060E571E084E892E00E9445
:1095B000A39F80918F05882389F2F9CE809173054E
:1095C00010927305882309F46CC120E030E048EC68
:1095D00052E4609152017091530180915401909135
:1095E00055010E94A6D40E9445DC912C812CABE051
:1095F000AA2EAFE4BA2E6B0118EEE12E13E0F12E85
:1096000000E010E020E030E0A90162E571E08CE7C5
:1096100092E00E94EB9E80918F05882309F441C15E
:10962000C6CE8091730510927305882309F48DCE00
:109630000E94DF9E20E030E040E251E46091C405EA
:109640007091C5058091C6059091C7050E94A6D46A
:1096500020E030E040E251E40E9448DB0E9445DC1B
:10966000912C812CE5E0AE2EEFE4BE2E6B0112E3CF
:10967000E12E16E8F12E01E010E02AE030E040E0B3
:1096800050E064EC75E084E792E00E94EB9E8091EC
:109690008F05882309F459CE8ACE86E0781279C0E6
:1096A00010929805809178058630B1F180914E0135
:1096B000882309F466CE11E080917805863009F0A0
:1096C00010E0C090E002D090E102E090E202F09061
:1096D000E30220E030E0A901C701B6010E9440D4B6
:1096E0002DEB37E346E055EB87FD04C02DEB37E368
:1096F00046E055E3C701B6010E9449DB69837A83DE
:109700008B839C83CE0101960E94F01900E09C019E
:109710004CE652E0642D32CE8091730510927305B1
:10972000882321F20E94DF9E20E030E048EC52E4E2
:109730006091E0027091E1028091E2029091E30277
:109740000E94A6D420E030E040E85FE30E9448DBBE
:109750000E9445DC3BEF832E3EE1932E4FEFA42E7B
:109760004EE4B42E6B0117E5E12E1EE3F12E0FE05F
:1097700010E021E030E040E050E060EE72E08CE686
:1097800092E00E94EB9E80918F05882309F48ECF92
:109790000ECE87E07812A4CE1092980580917805BD
:1097A0008730D9F080914E01882309F4EACD11E089
:1097B00080917805873009F010E06091DC027091AB
:1097C000DD028091DE029091DF020E94031D00E025
:1097D0009C0144E652E0652DD1CD80917305109235
:1097E00073058823F9F20E94DF9E20E030E040E21A
:1097F00051E46091DC027091DD028091DE02909173
:10980000DF020E94A6D420E030E040E251E40E9452
:1098100048DB0E9445DC84EE882E8EE1982E95E090
:10982000A92E9FE4B92E6B0112E3E12E16E8F12E6A
:1098300001E010E02AE030E040E050E06CED72E042
:1098400084E692E00E94EB9E80918F05882309F4C4
:10985000A9CFADCD8091730510927305882309F4CB
:1098600049CE0E94DF9E00E214E425EF30E046E995
:1098700050E060E071E085E592E00E94A39F809156
:109880008F05882309F436CE92CD83E0781609F44B
:1098900061CE84E0781223CD80917805843009F47C
:1098A0008DCE80914E01882309F4EECD11E0809198
:1098B0007805843009F010E0C0905201D090530137
:1098C000E0905401F090550120E030E0A901C7017B
:1098D000B6010E9440D42DEB37E346E055EB87FDFF
:1098E00004C02DEB37E346E055E3C701B6010E9403
:1098F00049DB69837A838B839C83CE0101960E9426
:10990000111B00E09C014CE752E0622D3ECE2F92ED
:109910003F924F925F926F927F928F929F92AF92FF
:10992000BF92CF92DF92EF92FF920F931F93CF934C
:10993000DF9300D01F92CDB7DEB74C013B015A0137
:10994000222E3B83280181E08093620240917F05B3
:1099500050918005609181057091820541155105F6
:109960006105710571F0141615060CF080E0809306
:10997000E40210927F0510928005109281051092EA
:1099800082051091E4023090730510927305311036
:1099900005C080914E01882309F46FC0C2010E9466
:1099A000906C082F80E0C114D10419F0C6010E9408
:1099B000906C1A821982E114F104B1F4402F50E046
:1099C000282F30E0CA01820F931F46976CF485E17F
:1099D00090E0841B950B821B930B97FD0196959548
:1099E00087958A8381E0898301E029E436E6A20134
:1099F000BE016F5F7F4FCE0102960E94166EE1148A
:109A0000F10491F08A81882321F01A8289818F5F85
:109A1000898300E02CE436E6A701BE016F5F7F4F2B
:109A2000CE0102960E94166EC114D10459F000E0D6
:109A300029E436E6A601BE016F5F7F4FCE01029694
:109A40000E94166E41E04127B30181E00E9492A37B
:109A5000C4010E94906C412FB40194E1981B892F9E
:109A60000E9492A3332049F0111102C0A22CBB80A6
:109A7000A114B104C1F0F50109950F900F900F905A
:109A8000DF91CF911F910F91FF90EF90DF90CF90DA
:109A9000BF90AF909F908F907F906F905F904F900E
:109AA0003F902F90089580E00E945D44E6CFCF92D2
:109AB000DF92EF92FF920F931F938BE3C82E85E006
:109AC000D82EF12CE12C0DE315E030E020E04CE243
:109AD00053E46DE475E082E595E00E94874C1F91A8
:109AE0000F91FF90EF90DF90CF900895AF92BF92CB
:109AF000CF92DF92EF92FF920F931F93CF93DF935A
:109B0000CDB7DEB7ADB6BEB68091760E6BE975E027
:109B1000882311F066E77EE0FB0101900020E9F761
:109B2000CF01861B970B01962DB73EB7281B390B2B
:109B30000FB6F8943EBF0FBE2DBF8DB79EB70196EE
:109B40007C0180E2EDB7FEB78183C70101960E94D8
:109B500099DD87EFC82E84E0D82E09EF14E030E0BD
:109B600020E048E154E465E075E08CE095E00E9477
:109B7000874C0FB6F894BEBE0FBEADBEDF91CF913D
:109B80001F910F91FF90EF90DF90CF90BF90AF901B
:109B90000895CF92DF92EF92FF920F931F9383E588
:109BA000C82E84E0D82EF12CE12C04ED14E030E036
:109BB00020E042E153E665E574E08AE594E00E9426
:109BC000874C1F910F91FF90EF90DF90CF900895F9
:109BD000CF92DF92EF92FF920F931F9383E0C82EF4
:109BE00083E0D82EF12CE12C05E013E02DE732E5DF
:109BF0004AED52E261E173E086E193E00E94874C16
:109C00001F910F91FF90EF90DF90CF900895AF924A
:109C1000BF92CF92DF92EF92FF920F931F93CF9359
:109C2000DF93CDB7DEB7ADB6BEB683E392E00E9458
:109C3000906C90E001962DB73EB7281B390B0FB6FC
:109C4000F8943EBF0FBE2DBF8DB79EB701967C0125
:109C500063E372E00E9486D38091E80200E012E0A4
:109C6000813031F00BEE11E0823011F003E112E0AF
:109C700084E2C82E82E0D82E21EE33E448E250E69A
:109C800066E272E08DE292E00E94874C0FB6F89493
:109C9000BEBE0FBEADBEDF91CF911F910F91FF9061
:109CA000EF90DF90CF90BF90AF9008950F931F93E8
:109CB000CF93DF93FC01EB0180917F0590918005AC
:109CC000A0918105B0918205B7FF08C010927F0571
:109CD0001092800510928105109282058091830573
:109CE00090918405A0918505B091860540917F05EE
:109CF00050918005609181057091820584179507C8
:109D0000A607B70744F480937F0590938005A0933E
:109D10008105B093820580914E018823E1F0609126
:109D20007F05709180058091810590918205009159
:109D30008705109188052091890530918A05600F6B
:109D4000711F821F931F0995BC0180918D05909111
:109D50008E050E94067480917305811108C0809160
:109D60007C058823D9F180914E018823B9F1809137
:109D70008B0590918C050097B1F040917F05509133
:109D80008005609181057091820500918705109191
:109D900088052091890530918A05400F511F621F67
:109DA000731FFE010995E0917D05F0917E053097C6
:109DB00041F080917C05811103C080917305811170
:109DC00009958091730510927305882339F080E01E
:109DD000DF91CF911F910F910C945D44DF91CF9152
:109DE0001F910F91089565E87CE18EE99CE10C9448
:109DF000564E62E17EE186E29EE10C94564E64E4AA
:109E00007EE188E59EE10C94564E6EEF7DE182E99D
:109E10009EE10C94564E60E37EE18CE99EE10C9449
:109E2000564E66ED7EE187E691E40C94564E109214
:109E3000620280E00C945D448F929F92AF92BF9239
:109E4000CF92DF92EF92FF92CF93809173051092A1
:109E50007305882359F0CF91FF90EF90DF90CF905A
:109E6000BF90AF909F908F900C94174FC0907F053C
:109E7000D0908005E0908105F0908205C114D10456
:109E8000E104F10441F110927F05109280051092D7
:109E900081051092820581E080934E0184E00E944A
:109EA000053D811118C0CC0CDD1CCC0CDD1C809153
:109EB0006002909161028C0D9D1D909361028093D0
:109EC00060028091940290919502C80ED91ED092A2
:109ED0009502C092940280914E01882309F4AEC08D
:109EE0006091600270916102072E000C880B990B43
:109EF0000E9447D420910206309103064091040647
:109F0000509105060E94A6D46B017C0120E030E050
:109F100040E251E40E94A6D420E030E04AE754E455
:109F20000E94A6D44B015C0120E030E0A901C701EA
:109F3000B6010E9440D420E030E040EA50E487FFC0
:109F400004C020E030E040EA50ECC501B4010E94BA
:109F500049DB20E030E040E251E40E94CCDB0E948B
:109F60003EDC6B017C018BE2F7FE09C0F094E094CB
:109F7000D094C094C11CD11CE11CF11C8DE28093D3
:109F80006302C701B60120E137E240E050E00E94E1
:109F900006DB8AE0882E912CA12CB12CCA01B901D4
:109FA000A50194010E9406DB605D60936402C70115
:109FB000B60128EE33E040E050E00E9406DBCA0123
:109FC000B901A50194010E9406DB605D6093650202
:109FD0008EE280936602C701B60124E630E040E0DD
:109FE00050E00E9406DBCA01B901A50194010E945C
:109FF00006DB605D60936702C701B601A5019401AD
:10A000000E9406DBC62FCA01B901A50194010E9476
:10A0100006DB605D60936802C05DC093690263E621
:10A0200072E089ED95E0CF91FF90EF90DF90CF90B7
:10A03000BF90AF909F908F900C940674CF91FF903B
:10A04000EF90DF90CF90BF90AF909F908F9008954A
:10A05000CF93DF9300D000D0CDB7DEB780917305EA
:10A0600010927305882349F00E94174F0F900F90AC
:10A070000F900F90DF91CF91089560917F057091BF
:10A08000800580918105909182056115710581059A
:10A09000910561F10E9447D42091020130910301A2
:10A0A00040910401509105010E94A6D420916E01B7
:10A0B00030916F0140917001509171010E9449DB14
:10A0C00060936E0170936F018093700190937101A2
:10A0D00083E00E94E86B81E080934E0110927F053F
:10A0E00010928005109281051092820580914E0198
:10A0F000882309F4BBCF20917405309175054091F8
:10A1000076055091770560916E0170916F01809195
:10A110007001909171010E9448DB69837A838B837F
:10A120009C83CE0101960E94951ABC0185E79BE2B3
:10A130000E9406749BCF3F924F925F926F927F92E4
:10A140008F929F92AF92BF92CF92DF92EF92FF9247
:10A150000F931F93CF93DF93CDB7DEB72C970FB636
:10A16000F894DEBF0FBECDBF9C878B87362E8091C3
:10A170007305109273058823D1F00E94174F2C9617
:10A180000FB6F894DEBF0FBECDBFDF91CF911F9108
:10A190000F91FF90EF90DF90CF90BF90AF909F9086
:10A1A0008F907F906F905F904F903F900895609157
:10A1B0007F057091800580918105909182056115E0
:10A1C00071058105910509F45CC020910A012223E3
:10A1D00009F4AEC020910B012111AAC021E0321672
:10A1E00009F484C0E2E03E1609F491C0C0900C016D
:10A1F000D0900D01E0900E01F0900F0140901801F9
:10A200005090190160901A0170901B010E9447D470
:10A210002091020130910301409104015091050108
:10A220000E94A6D46F83788789879A87F4E03F9E3F
:10A2300080011124C8018E599E4F9E838D83FC019D
:10A2400020813181428153816F81788589859A850A
:10A250000E9449DB4B015C01A3019201C701B601D9
:10A260000E9440D4811173C0F801EE59FE4F8082E4
:10A270009182A282B382832D0E94E86B81E0809359
:10A280004E0110927F051092800510928105109268
:10A29000820580914E01882309F471CF24E0329E1B
:10A2A000F0011124EE59FE4FC080D180E280F3808E
:10A2B000C982DA82EB82FC822DEC3CEC4CEC5DE353
:10A2C0006091020170910301809104019091050158
:10A2D0000E94CCDC87FD65C0CE0101960E94951AD4
:10A2E000BC018B859C850E94067449CFC0901001EB
:10A2F000D0901101E0901201F090130140901C01E8
:10A3000050901D0160901E0170901F017FCFC09082
:10A310001401D0901501E0901601F09017014090C3
:10A3200020015090210160902201709023016ECF96
:10A33000412C20E5522E23EC622E27E4722EC12CF4
:10A3400030E5D32E33ECE32E37ECF32E5FCF20E055
:10A3500030E0A9016F81788589859A850E9440D473
:10A3600087FF0FC0A7019601C501B4010E9440D428
:10A3700087FF7ACFED81FE81C082D182E282F382B3
:10A380007ACFA3019201C501B4010E94CCDC18165A
:10A390000CF06ACFED81FE8140825182628273822D
:10A3A0006ACF20E030E040E251E4C701B6010E94EC
:10A3B000A6D420E030E04AE754E40E94A6D44B0142
:10A3C0005C0120E030E0A901C701B6010E9440D441
:10A3D00020E030E040EA50E487FF04C020E030E0B5
:10A3E00040EA50ECC501B4010E9449DB20E030E0B6
:10A3F00040E251E40E94CCDB0E943EDC6B017C0118
:10A40000F7FC62C020EA36E841E050E00E9406DB3B
:10A41000CA01B9012AE030E040E050E00E9406DBCA
:10A42000605D60936302C701B60120E137E240E05E
:10A4300050E00E9406DB8AE0882E912CA12CB12CE2
:10A44000CA01B901A50194010E9406DB605D609319
:10A450006402C701B60128EE33E040E050E00E94FC
:10A4600006DBCA01B901A50194010E9406DB605D0B
:10A47000609365028EE280936602C701B60124E60E
:10A4800030E040E050E00E9406DBCA01B901A501BE
:10A4900094010E9406DB605D60936702C701B6010C
:10A4A000A50194010E9406DB162FCA01B901A5017E
:10A4B00094010E9406DB605D60936802105D10935A
:10A4C000690283E692E00CCFF094E094D094C094BB
:10A4D000C11CD11CE11CF11C6DE2A3CF62E083E83A
:10A4E0009BE20C949B5061E08AE89BE20C949B50A9
:10A4F00060E081E99BE20C949B5080E090E0A0E852
:10A50000B0E480936A0190936B01A0936C01B093C7
:10A510006D018BEF91E00E94D5220C94174F809330
:10A52000E80220E040E070E060E087E09EE40C9408
:10A5300079422F923F924F925F926F927F928F92C9
:10A540009F92AF92BF92CF92DF92EF92FF920F93C2
:10A550001F93CF93DF93CDB7DEB7C358D1090FB6A2
:10A56000F894DEBF0FBECDBF2DB73EB7CE57DF4F3D
:10A5700039832883C258D04041E064E070E0CE01C6
:10A5800087589F4F0E94F89B43E050E0BE016758F8
:10A590007F4F85E092E00E94A0DD892B09F453C033
:10A5A000ED968FADED97882339F08FE3EA968FAF64
:10A5B000EA97EB961FAEEB970E94677EBE01675845
:10A5C0007F4F8FEF9AE00E941B8281EF9AE00E94FA
:10A5D000567D82E00E948F5281E080930D0380912E
:10A5E0008902811107C08091DC05833018F080E07A
:10A5F0000E94BF2C90910D0381E08927CE57DF4F39
:10A6000028813981C258D0400FB6F8943EBF0FBEA2
:10A610002DBFCD57DF4F0FB6F894DEBF0FBECDBFB5
:10A62000DF91CF911F910F91FF90EF90DF90CF902E
:10A63000BF90AF909F908F907F906F905F904F9062
:10A640003F902F90089541E062E070E0CE01835882
:10A650009F4F0E94F89BE9961CAE1DAE1EAE1FAE2A
:10A66000E99710921D1110921C11CE0181589F4F35
:10A670000E94BA22CDB6DEB6C158DF4F0881CF574F
:10A68000D04010E00D5F1F4F000F111F000F111F72
:10A690008DB79EB7801B910B0FB6F8949EBF0FBE6F
:10A6A0008DBFEDB7FEB731965F012DB73EB7201BCA
:10A6B000310B0FB6F8943EBF0FBE2DBF8DB79EB7BE
:10A6C00001964C01EDB7FEB7E01BF10B0FB6F89405
:10A6D000FEBF0FBEEDBF2DB73EB72F5F3F4F7901D5
:10A6E000B801C5010E94BF224091890281E048273C
:10A6F00064E070E08DEC9BE00E94F89BB801C4011F
:10A700000E94BF22B801C7010E94BF221091890296
:10A7100011114DC0C158DF4F8881CF57D04090E014
:10A720000296ADEBBBE070E060E030E020E04DEE83
:10A730005AE0821793070CF49BC0F501E60FF71F50
:10A7400040805180628073804D925D926D927D92C7
:10A75000821793070CF492C0F401E60FF71F2080D4
:10A7600031800281E3812101602E7E2E50964D9230
:10A770005D926D927C925397821793070CF488C078
:10A78000F701E60FF71F208031800281E38121016C
:10A79000602E7E2E90964D925D926D927C92939754
:10A7A0002F5F3F4F6C5F7F4F2430310511F681EFF3
:10A7B0009BE00E94922285EF9BE00E94922289EF0B
:10A7C0009BE00E9492228DEF9BE00E94922281E00A
:10A7D0009CE00E949222CE018B589F4F0E949222B1
:10A7E000CE018B589F4F0E949222CE018B589F4FD3
:10A7F0000E949222CE018B589F4F0E9492228DED93
:10A8000095E00E9492220FB6F894DEBE0FBECDBE38
:10A81000CE0101967C010E94B222CE0183599F4F46
:10A820000E949A22C7010E949222CE018B589F4F0C
:10A830000E949222CE018B589F4F0E949222C70104
:10A840000E94BA22CE0183599F4F0E94BA22C9802A
:10A85000AE968FADAE97C89E6001112491E0C91AE3
:10A86000D10800F1CE018B589F4F0E949222F6CF63
:10A87000FA01459055906590749066CFEDEDFAE041
:10A8800045905590659074901201062DE72D6BCF81
:10A89000EDECFAE045905590659074901201062D0C
:10A8A000E72D75CFC7010E94B2220AE00150CE0108
:10A8B00029F08B589F4F0E949222F8CF80589F4FCB
:10A8C0000E94BA22CE018F579F4F0E94BA22C70121
:10A8D0000E94AA22CE0183599F4F0E94AA22C058EB
:10A8E000DF4FC880C058D040CF57DF4F8881C15854
:10A8F000D040C89E60011124F1E0CF1AD10830F099
:10A90000CE018B589F4F0E949222F6CFC7010E9422
:10A91000A222CE0183599F4F0E949A2201E0412F2B
:10A92000402760E170E0C7010E94F89BC7010E94C8
:10A93000A22240918902402768E070E081E892E01D
:10A940000E94F89B40918902402764E170E0C701B2
:10A950000E94F89B00918902011138C089809A8079
:10A96000AB80BC80A5019401C501B4010E944ADD01
:10A9700081112CC08092C4059092C505A092C60595
:10A98000B092C7052CEA35EC47E25EE36D817E812B
:10A990008F8198850E94A6D46093C8057093C905DD
:10A9A0008093CA059093CB052CEA35EC47E25EE331
:10A9B00069857A858B859C850E94CCDB6093CC056C
:10A9C0007093CD058093CE059093CF0511E0402F75
:10A9D000412762E070E0C7010E94F89BC7010E9416
:10A9E0008A22C7010E948A22C7010E949A22C701B7
:10A9F0000E949A22C7010E949A2285E0F7011192D3
:10AA00008A95E9F740918902412765E070E0C70126
:10AA10000E94F89BC7010E94A2224091890241270F
:10AA200060E270E0C7010E94F89BCE0183599F4FFE
:10AA30000E94A22240918902412769E070E0C7018B
:10AA40000E94F89B40918902412762E170E0C701B2
:10AA50000E94F89B40918902412764E270E0C7019F
:10AA60000E94F89B40918902412760E170E0C70194
:10AA70000E94F89B40918902412769E070E0C7017C
:10AA80000E94F89BC7010E949222409189024127AF
:10AA90006CE070E0C7010E94F89B40918902412759
:10AAA0006CE670E0C7010E94F89B19821A821B8233
:10AAB0001C821D821E821F82188619861A861B869A
:10AAC0001C86C7010E948A2240918902412768E0C2
:10AAD00070E0C7010E94F89BC7010E94B222CE011C
:10AAE00080589F4F0E949A22CE0183599F4F0E9407
:10AAF00092228091161190911711883D924041F158
:10AB00000E94637E87E39AE00E94567D10930D03B6
:10AB10000E94677E60911611709117116456710939
:10AB200089EB9AE00E940C8164E772E081EB9AE085
:10AB30000E94198181E00E948F52809189028111C7
:10AB40004ECD80910D0381114ACD0E94D33047CD67
:10AB500010920D0320911C1130911D11EF968EADB6
:10AB60009FADEF972817390721F110930D030E942D
:10AB7000637EEF960EAD1FADEF9781E99AE00E94DC
:10AB8000567DB80190E080E00E94DF9A00911C1190
:10AB900010911D118CE89AE00E94567DB80190E05A
:10ABA00080E00E94DF9A8CE79AE00E94567D80E068
:10ABB000C2CF809189028111C0CF0E94677E85E05B
:10ABC00092E00E9438A56091161170911711645699
:10ABD00071098FE59AE00E940C81C0901C11D09001
:10ABE0001D11F12CE12C82E59AE00E94567DC701EF
:10ABF000B6010E94DF9A8FE49AE00E94567D9DCFB5
:10AC000084E690E0909317118093161110921D1115
:10AC100010921C110C94995281E0809389020E9439
:10AC200000561092890281110C9400560E94563FE2
:10AC300080E008950E940C560C940742E091D502E2
:10AC4000E63028F581E08E0F8093D50240917F0594
:10AC50005091800560918105709182052091790560
:10AC6000909172058091620239E0E39FF001112416
:10AC7000E156FD4FA091A111B091A211B183A08323
:10AC800042835383648375832683978380870895E3
:10AC9000CF93DF93EC010E941E5620E040E070E06D
:10ACA00060E0CE01DF91CF910C9479422F923F92D8
:10ACB0004F925F926F927F928F929F92AF92BF92CC
:10ACC000CF92DF92EF92FF920F931F93CF93DF9378
:10ACD00000D000D0CDB7DEB761E081E00E941B421A
:10ACE000209179052B832B5F298385E0382E9B816A
:10ACF000391A84E0891B8A8366246A94712C23E0C4
:10AD0000291B2C8382E0582E591A81E0482E491ABB
:10AD1000292E21948B8181113BC080917805882355
:10AD2000A1F080914E01882359F081E0909178053F
:10AD3000911180E024E040E056E0622D0E94029EE6
:10AD40008091F9058093E80273C080917305109299
:10AD50007305882331F30E948D4480918F058823E9
:10AD600001F30F900F900F900F90DF91CF911F91F3
:10AD70000F91FF90EF90DF90CF90BF90AF909F909A
:10AD80008F907F906F905F904F903F902F9008959D
:10AD90009B81913009F06FC080917805813009F472
:10ADA00051C080914E01882359F211E080917805BD
:10ADB000813009F010E080910601909107010E9416
:10ADC000324100E09C014AEF55E0642D812F0E9442
:10ADD00085748091F9058093E8028B81833009F0B6
:10ADE000BDC01092980580917805833009F47BC02E
:10ADF00080914E018823E1F011E080917805833045
:10AE000009F010E08091E80224E6829FC00111243D
:10AE100081589F4FB3010E94F2DA862F0E944B1C8B
:10AE200000E09C0149EE55E06C81812F0E94857401
:10AE30002B812F5F2B83898128136CCF86E0809331
:10AE400072058FCF8091730510927305882309F4E2
:10AE5000A8CF10E000E027EE33E04AE050E066E0E3
:10AE600071E08AEF95E00E94A39F80918F0588236F
:10AE700009F497CF76CF2B81223009F0AACF8091A9
:10AE800078058230B9F080914E01882309F458CFBB
:10AE900011E080917805823009F010E08091C105C1
:10AEA0009091C2050E94324100E09C0143EF55E0C1
:10AEB000652D8CCF8091730510927305882319F34B
:10AEC0000E94DF9E02E61FE125EF30E050E040E007
:10AED00061EC75E083EF95E00E94A39F80918F0560
:10AEE000882389F23ECF80917305109273058823E1
:10AEF00009F47ECF0E94DF9E6091E80270E090E04E
:10AF000080E00E9445D429EC38EC48EC5EE30E94D6
:10AF1000A6D420E030E040E05FE30E9449DB0E94DD
:10AF200045DC8BEB882E8CE1982E93EFA92E9EE4C6
:10AF3000B92E6B0114E6E12EF12C00E010E020E0C8
:10AF400030E0A90168EE72E089EE95E00E94EB9E88
:10AF500080918F05882309F44BCF03CF8B818430F8
:10AF600091F5809178058430B9F080914E01882365
:10AF700009F45ECF11E080917805843009F010E08B
:10AF800080912401909125010E94324100E09C01B2
:10AF900044EE55E06A8149CF8091730510927305A4
:10AFA000882319F30CE61CE127EE33E04AE050E079
:10AFB00064E271E084EE95E00E94A39F80918F058A
:10AFC000882399F2CECE9B81953009F031CF8091C4
:10AFD0007805853091F080914E01882309F428CFBF
:10AFE00081E090917805953009F080E023E049ED0B
:10AFF00055E0632D0E94029E1BCF80917305109235
:10B000007305882341F382E093E40E9448568091BF
:10B010008F05882301F3A5CE7F928F929F92AF92E6
:10B02000BF92CF92DF92EF92FF920F931F93CF9335
:10B03000DF9361E081E00E941B42C0917905EC2E14
:10B0400085E0982E9C0E92E7C92E95E0D92ED7E088
:10B05000DC1BBB24B39416E01C1B22E0A22E05E0EF
:10B060000C1B84E0F82EFC1A8A2C8C1A7B2C7C1A80
:10B07000C11135C0809178058823B9F080914E01C7
:10B08000882361F06E2D619581E090917805911192
:10B0900080E024E047EA55E00E94029ECF5FC9119C
:10B0A000E7CF88E0809372050CC080917305109201
:10B0B0007305882319F30E948D4480918F0588239E
:10B0C000E9F2DF91CF911F910F91FF90EF90DF9008
:10B0D000CF90BF90AF909F908F907F900895C13098
:10B0E00011F580917805813079F080914E018823A7
:10B0F000A9F281E090917805913009F080E023E099
:10B100004BE65BE2672DC8CF809173051092730503
:10B11000882359F38BE799E50E94485680918F0563
:10B12000882319F3CECFC23009F0C5C090917805BD
:10B13000923071F080914E01882309F4AFCF81E005
:10B14000923009F080E020E249E955E0682DA4CF73
:10B150008091730510927305882361F323EA35E02B
:10B160003093300520932F0580918F05882311F3AC
:10B17000A8CF1092980590917805933079F080913E
:10B180004E01882309F48ACF63E06E1981E0933081
:10B1900009F080E020E24DE855E07ECF8091730514
:10B1A00010927305882359F324E935E03093300574
:10B1B00020932F0580918F05882309F382CFB092C9
:10B1C000980590917805943071F080914E01882314
:10B1D00009F464CF81E0943009F080E020E24DE88A
:10B1E00055E06F2D59CF8091730510927305882318
:10B1F00061F328E835E03093300520932F058091E6
:10B200008F05882311F35DCFA09298059091780562
:10B21000953071F080914E01882309F43FCF81E091
:10B22000953009F080E020E24DE855E0602F34CF02
:10B230008091730510927305882361F323E835E04C
:10B240003093300520932F0580918F05882311F3CB
:10B2500038CF80917805863081F080914E01882327
:10B2600009F41CCF81E090917805963009F080E0D8
:10B2700023E046E755E0612F0FCF809173051092D0
:10B280007305882351F382E193E40E94485680912C
:10B290008F05882311F315CF8091730510927305E4
:10B2A0008823D9F0D0923005C0922F0580918F0568
:10B2B000882399F006CFC33009F45BCFC43009F47A
:10B2C0007ECFC53009F4A0CFC63019F2C73009F0DF
:10B2D000E5CE909178059730F9F280914E01882360
:10B2E00009F4DCCE81E0973009F080E020E241E60D
:10B2F00055E06D2FD1CEDF92EF92FF920F931F9307
:10B30000CF93DF9361E081E00E941B42C0917905F9
:10B3100085E0E82EEC0ED4E0DC1B13E01C1B02E001
:10B320000C1B81E0F82EFC1ADC2ED194C1112EC02A
:10B33000809178058823B1F080914E01882359F0DF
:10B3400081E090917805911180E024E04AE555E094
:10B350006D2D0E94029ECF5FEC12E8CF85E08093B6
:10B3600072050CC08091730510927305882321F338
:10B370000E948D4480918F058823F1F2DF91CF9157
:10B380001F910F91FF90EF90DF900895C13011F55C
:10B3900080917805813079F080914E018823D9F22F
:10B3A00081E090917805913009F080E023E041E957
:10B3B0005BE26F2DCECF80917305109273058823C9
:10B3C00059F387E693E20E94485680918F058823BF
:10B3D00019F3D4CFC23009F055C08091780582307E
:10B3E00081F080914E01882309F4B5CF81E09091DE
:10B3F0007805923009F080E023E04AE85BE2602FB4
:10B40000A8CF8091730510927305882351F382E6CB
:10B4100093E20E94485680918F05882311F3AECFA6
:10B4200080917805833081F080914E01882309F462
:10B4300092CF81E090917805933009F080E023E08D
:10B4400043E85BE2612F85CF80917305109273050D
:10B45000882351F38DE593E20E94485680918F0531
:10B46000882311F38BCF8091730510927305882385
:10B4700091F084E393E40E94485680918F058823DD
:10B4800051F07CCFC33061F2C43009F064CF8091B9
:10B490007805843041F380914E01882309F45BCF15
:10B4A00081E090917805943009F080E023E045E751
:10B4B0005BE26D2F4ECFEF92FF920F931F93CF93CE
:10B4C000DF9361E081E00E941B42C091790585E035
:10B4D000F82EFC0ED3E0DC1B12E01C1B01E00C1B61
:10B4E000EC2EE194C1112DC0809178058823B1F034
:10B4F00080914E01882359F081E090917805911157
:10B5000080E024E04EE454E06E2D0E94029ECF5F66
:10B51000FC12E8CF84E0809372050CC08091730523
:10B5200010927305882321F30E948D4480918F052A
:10B530008823F1F2DF91CF911F910F91FF90EF904F
:10B540000895C13011F580917805813079F08091AE
:10B550004E018823E1F281E090917805913009F065
:10B5600080E023E041E454E0602FCFCF8091730569
:10B5700010927305882359F382E496E40E9448569A
:10B5800080918F05882319F3D5CFC23091F5809132
:10B590007805823081F080914E01882309F4B7CF7D
:10B5A00081E090917805923009F080E023E046E355
:10B5B00054E0612FAACF8091730510927305882300
:10B5C00051F385ED96E40E94485680918F058823BB
:10B5D00011F3B0CF8091730510927305882381F029
:10B5E0008EE697E40E94485680918F05882341F0AB
:10B5F000A1CFC33009F08BCF80917805833051F310
:10B6000080914E01882309F482CF81E090917805E2
:10B61000933009F080E023E04AE254E06D2F75CFCB
:10B62000DF92EF92FF920F931F93CF93DF930E94CD
:10B63000121F082F61E081E00E941B42C091790532
:10B64000FC2E85E0E82EEC0E11E01C1BDC2ED194C4
:10B65000C11114C0809178058823F9F080914E01C2
:10B66000882309F477C081E090917805911180E0FA
:10B6700024E045EF52E06D2D0E94029E01113DC075
:10B68000D2E0C130D9F5809178058130D1F0809138
:10B690004E01811125C0D2E047C080917305109200
:10B6A00073058823D9F20E948D4480918F058823E9
:10B6B000A9F2DF91CF911F910F91FF90EF90DF9052
:10B6C00008958091730510927305882301F387EF25
:10B6D00097E40E94485680918F058823C1F2E9CFF4
:10B6E00081E090917805913009F080E023E04CEE04
:10B6F00052E0612F0E94029ECECFD1E0DC1314C035
:10B70000809178058D17B9F080914E01882361F002
:10B710006C2F6F1981E0909178059C1380E023E0F5
:10B7200040EE52E00E94029ECF5FCE1191CFDF5FCC
:10B73000D0937205BECF8091730510927305882354
:10B7400019F388E299E40E94485680918F05882376
:10B75000D9F2AFCFD1E0002309F49DCFE5CFCF934D
:10B76000DF93C0915C02D0915D02DF77209759F59D
:10B770008091F91283FD2BC00E940C77882319F168
:10B780008091F1129091F212A091F312B091F41203
:10B790000097A105B105B9F0BC01CD01615F784DFD
:10B7A0008F4F9F4F20E137E240E050E00E9488DA5F
:10B7B0006091F5127091F6128091F7129091F81243
:10B7C0000E9488DAE901CE01DF91CF910895C0E1AE
:10B7D000D7E2F9CFCF93DF93CDB7DEB78D819091CC
:10B7E0000E0F891778F080930E0F9E01285F3F4F50
:10B7F0004E815F8164E570E089EB9EE00E9407D492
:10B800001092B80EDF91CF9108950F931F93CF93AD
:10B81000DF936F3F11F410920E0F20910E0F211144
:10B820001EC08C010E948DD3800F911FEC01C01BA4
:10B83000D10BC535D1053CF00197FC012491207C4A
:10B840002038D1F3F3CFDD27AE01B80189EB9EE0BC
:10B850000E94AED3C754D14F18821092B80EDF9118
:10B86000CF911F910F9108958F929F92AF92BF92A7
:10B87000DF92EF92FF920F931F93CF93DF93CDB799
:10B88000DEB7C658D1090FB6F894DEBF0FBECDBFE4
:10B89000C358DF4F188219821A821B82CD57D040BD
:10B8A0008091510290915202A0915302B0915402A2
:10B8B000CF57DF4F88839983AA83BB83C158D04079
:10B8C00084E690E0909317118093161110921D1149
:10B8D00010921C1110920D0364E070E0CE018F579E
:10B8E0009F4F0E94D0A0809116119091171102963F
:10B8F000909317118093161110921D1110921C1124
:10B9000081E0CA57DF4F8883C658D040CE018A579E
:10B910009F4F0E94C92268E470E08DEB9BE00E947B
:10B92000D0A080E1E2E7F1E08E010F5F1F4FD80168
:10B9300001900D928A95E1F760E170E0C8010E94E4
:10B94000D0A08DED95E00E94D1228CE0F8011192FB
:10B950008A95E9F7C8010E94CD227E01FDE6EF0E2F
:10B96000F11C8FEFF7018083C7010E94C922198261
:10B970001A821B821C82C8010E94D12219821A825B
:10B980001B821C82C8010E94D122C358DF4F18823B
:10B9900019821A821B82CD57D04083E0F701808341
:10B9A0008983CE0183589F4F0E94D122C7010E94F4
:10B9B000C922C8010E94C9224AE0D42EDA94DD20AF
:10B9C00031F0CE0183589F4F0E94D122F7CF8CE0F7
:10B9D000F80111928A95E9F7C8010E94CD22C35857
:10B9E000DF4F188219821A821B82CD57D0403AE06D
:10B9F000D32EDA94DD2031F0CE0183589F4F0E9480
:10BA0000D122F7CF88E0F701982F11929A95E9F7A4
:10BA1000F80111928A95E9F783E0CB57DF4F8883CD
:10BA2000C558D040EA968FAFEA97CE018B579F4F0B
:10BA30000E94C922CE0187589F4F0E94C92268E008
:10BA400070E0C8010E94D0A068E070E0C7010E94C9
:10BA5000D0A0C358DF4F188219821A821B82CD579B
:10BA6000D0402AE0A22EB12CF1E0AF1AB10831F09B
:10BA7000CE0183589F4F0E94D122F6CF1982BB245A
:10BA8000BA94F701B082C8010E9438A1C7010E9490
:10BA9000C92280E1D82EF8018D2D11928A95E9F7FF
:10BAA00060E170E0C8010E94D0A01982C8010E9424
:10BAB00038A168E070E081E892E00E94D0A0198A85
:10BAC0001A8A1B8A1C8A80E090E0A0E8BFE38D8779
:10BAD0009E87AF87B88B8091C4059091C505A091D2
:10BAE000C605B091C70589839A83AB83BC832CEAD2
:10BAF00035EC47E25EE36091C8057091C90580911D
:10BB0000CA059091CB050E94CCDB6D837E838F8329
:10BB100098872CEA35EC47E25EE36091CC057091A2
:10BB2000CD058091CE059091CF050E94A6D469875E
:10BB30007A878B879C8764E170E0C8010E94D0A05F
:10BB400084E190E09A83898362E070E0C8010E94FA
:10BB5000D0A08CE0E2E8F1E0D80101900D928A9546
:10BB6000E1F7C8010E94C5228CE0E2E8F1E0D801CB
:10BB700001900D928A95E1F7C8010E94C5221982B1
:10BB8000C8010E94C9228FE78983C8010E94C92287
:10BB9000B982C8010E94C92285E0EEE8F1E0D8012F
:10BBA00001900D928A95E1F765E070E0C8010E946E
:10BBB000D0A01982C8010E9438A180E2E3E9F1E037
:10BBC000D80101900D928A95E1F760E270E0C8011A
:10BBD0000E94D0A0F7011082C7010E9438A11982EB
:10BBE000C8010E9438A180E090E0A0EEBFE3C358F6
:10BBF000DF4F88839983AA83BB83CD57D040CE0182
:10BC000083589F4F0E94D122C358DF4F1882198258
:10BC10001A821B82CD57D040CE0183589F4F0E947D
:10BC2000D12282E1F80111928A95E9F762E170E090
:10BC3000C8010E94D0A084E2E3EBF1E0D8010190BA
:10BC40000D928A95E1F764E270E0C8010E94D0A0ED
:10BC5000F8011192DA94E9F760E170E0C8010E94FE
:10BC6000D0A089E0F80111928A95E9F769E070E0C7
:10BC7000C8010E94D0A0C358DF4F188219821A82CF
:10BC80001B82CD57D040CE0183589F4F0E94D122B6
:10BC90009CE0D92EF8018D2D11928A95E9F76CE080
:10BCA00070E0C8010E94D0A08CE6F80111928A953C
:10BCB000E9F76CE670E0C8010E94D0A081E093E053
:10BCC0000E94C522F701108211821282138214820F
:10BCD00015821682178268E070E0C7010E94D0A02A
:10BCE000F7011192DA94E9F7CB57DF4F1882C55864
:10BCF000D04080E090E0A0E4B0E4ED968CAF9DAF42
:10BD0000AEAFBFAFED97C7010E94CD22CE018B57DA
:10BD10009F4F0E94C922CE0187589F4F0E94D12277
:10BD2000D0900D03D1104AC0009116111091171137
:10BD30000456110980911C1190911D11F7019183F6
:10BD4000808384E690E0909317118093161164E04D
:10BD500070E085E092E00E94D0A062E070E0C70150
:10BD60000E94D0A00E94677E8EE899E00E94567DD6
:10BD7000B80190E080E00E94DF9AF7018080918016
:10BD8000B12CA12C81E899E00E94567DC501B40137
:10BD90000E94DF9A8EE799E00E94567D0437124098
:10BDA00041F00E94637E87E39AE00E94567DDD2485
:10BDB000D39480910D038D2980930D0380910D0301
:10BDC000811105C060E08EE699E00E94055C9091CB
:10BDD0000D0381E08927CA57DF4F0FB6F894DEBF05
:10BDE0000FBECDBFDF91CF911F910F91FF90EF90CC
:10BDF000DF90BF90AF909F908F9008950E94345C29
:10BE00000C9407422F923F924F925F926F927F92D3
:10BE10008F929F92AF92BF92CF92DF92EF92FF925A
:10BE20000F931F93CF93DF930E94121FD82F61E0CF
:10BE300081E00E941B42C09179052C2E85E0382EAE
:10BE40003C0E03E012E496E2E92E93E0F92E84E042
:10BE5000782E7C1A2AE1C22E26E5D22E37E3A32EB5
:10BE600033E0B32E83E0682E6C1A4EEF842E4EE53D
:10BE7000942E82E0582E5C1A81E0482E4C1AC11193
:10BE800037C0809178058823A1F080914E018823E6
:10BE900061F0622D619581E090917805911180E0CB
:10BEA00024E046E653E00E94029EDD2309F4ACC084
:10BEB000C8C08091730510927305882331F30E94E6
:10BEC0008D4480918F05882301F3DF91CF911F91DD
:10BED0000F91FF90EF90DF90CF90BF90AF909F9029
:10BEE0008F907F906F905F904F903F902F9008952C
:10BEF000C13019F580917805813081F080914E0133
:10BF0000882309F49CC081E090917805913009F074
:10BF100080E023E044E553E0642DC5CF80917305B4
:10BF200010927305882351F380E19BE50E944856E7
:10BF300080918F05882311F3C8CFC23009F066C005
:10BF4000809178058230E1F080914E01882309F4D8
:10BF500076C09F928F9285E493E09F938F935F9238
:10BF600081E090917805923009F080E08F930E94F3
:10BF70004F230F900F900F900F900F900F9095CF31
:10BF800080917305109273058823F1F20E94FE5E82
:10BF900080918F058823C1F298CF8091730510920C
:10BFA00073058823E1F10E941A5680918F0588233A
:10BFB000B1F18BCF8091730510927305882369F0DE
:10BFC0000E94034280918F05882339F07ECFC430D0
:10BFD000D9F480917805843069F380914E018823EB
:10BFE00099F01F930F93FF92EF927F9281E09091CF
:10BFF0007805943011F58F930E944F230F900F9086
:10C000000F900F900F900F9085E01CC0D11119C0B8
:10C01000C330E9F680917805833009F4BECF809172
:10C020004E01882389F3DF92CF92BF92AF926F9235
:10C0300081E0909178059330F1F280E0DCCFDD2350
:10C0400031F283E0CF5F3C121ACF809372053DCF6F
:10C05000CF930E94563F0E94345CC82F882319F06A
:10C0600080E00E94BF2C8C2F0E940742CF910C943D
:10C07000E143CF9380919702811109C08CED91E04B
:10C080009093DB028093DA0281E0809397020E9412
:10C090001E5620E040E070E060E085E793E20E94F9
:10C0A0007942C1E0C09362020E94E72D0E94174FBF
:10C0B000C093620260E089EC9BE20E94055C88ED1F
:10C0C00091E09093300580932F05CF9108952F92A2
:10C0D0003F924F925F926F927F928F929F92AF9218
:10C0E000BF92CF92DF92EF92FF920F931F93CF9365
:10C0F000DF9300D000D01F92CDB7DEB79091A80596
:10C100008091F91244244394913051F082FB4424ED
:10C1100040F882FF05C087FB442440F891E049269F
:10C1200084FB662460F8212C84FF03C00E940C77F6
:10C13000282E61E081E00E941B42209179052C832A
:10C14000522E2B5F298380E002EC14E091E0392E1F
:10C150003518752C719499E3E92E90E6F92E2FEDA0
:10C16000C22E24E0D22E92E095199A8393E095197D
:10C170009B8330E7832E34E0932E45E8A42E44E0E1
:10C18000B42E9C812981921709F449C2992349F15F
:10C1900041107EC00E942D7D882309F4ADC19C8191
:10C1A000913009F477C122E02D832C818D812813F1
:10C1B00092C180917805281709F4A1C180914E01A0
:10C1C000882309F488C16C81651981E09091780514
:10C1D0002C81921380E023E04BEB54E00E94029EFE
:10C1E0007AC180917805882379F180914E01882366
:10C1F00079F281E090917805911180E024E04BEE96
:10C2000054E0672D0E94029E442021F224E02D83F9
:10C210009C812D8192135FC080917805981709F455
:10C220007FC180914E01882309F455C06C81651946
:10C2300081E0909178052C81921380E023E04FEA11
:10C2400054E00E94029E47C08091730510927305CE
:10C25000882359F20E948D4480918F05882329F20A
:10C260000F900F900F900F900F90DF91CF911F9133
:10C270000F91FF90EF90DF90CF90BF90AF909F9085
:10C280008F907F906F905F904F903F902F90089588
:10C290008C81813009F49DC0823009F4C5C09C8135
:10C2A000933009F0B3CF80917805833009F4E1C071
:10C2B00080914E01882309F4A9CF81E090917805FF
:10C2C000933009F080E023E04FEC54E06B810E9452
:10C2D000029E84E08D838D818F5F9C81981316C0B0
:10C2E00080917805981709F42CC180914E0188231C
:10C2F00069F06C81651981E0909178052C81921329
:10C3000080E023E041EA54E00E94029E8D818E5F2E
:10C310009C81981316C080917805981709F422C162
:10C3200080914E01882369F06C81651981E09091BC
:10C3300078052C81921380E023E043E954E00E94C9
:10C34000029E8D818D5F662009F440C121103DC0A1
:10C350009C8198131DC080917805981709F413C12A
:10C3600080914E018823A1F01F92BF92AF928C81E1
:10C3700085198F9381E0909178052C81921380E04C
:10C380008F930E944F230F900F900F900F900F905C
:10C390008D818C5F9C81981316C0809178059817C9
:10C3A00009F403C180914E01882369F06C816519FD
:10C3B00081E0909178052C81921380E023E044E79E
:10C3C00054E00E94029E8D818B5F9C819F5F9C83C5
:10C3D000D8CE809178058130D1F080914E018823AC
:10C3E00009F414CFFF92EF92DF92CF923F9281E057
:10C3F00090917805913009F080E08F930E944F234F
:10C400000F900F900F900F900F900F90FFCE809194
:10C41000730510927305882301F30E94396080919F
:10C420008F058823D1F21CCF80917805823091F05E
:10C4300080914E01882309F4E9CE81E0909178053E
:10C44000923009F080E023E044ED54E06A810E94DC
:10C45000029EDCCE8091730510927305882341F310
:10C4600089EC9DE40E94485680918F05882301F352
:10C47000F7CE8091730510927305882309F418CFC5
:10C4800086E596E50E94485680918F05882309F439
:10C490000FCFE6CE80917805813009F180914E0171
:10C4A000882309F480CE8CE890E49F938F931F93A8
:10C4B0000F933F9281E090917805913009F080E0F0
:10C4C0008F930E944F230F900F900F900F900F901B
:10C4D0000F9082E08D838D818F5F8D8399CE8091C7
:10C4E0007305109273058823C9F20E948C408091D5
:10C4F0008F05882399F2B4CE91E09D8356CE80912A
:10C50000730510927305882309F458CE8CE098E5E2
:10C510000E94485680918F05882309F44FCEA0CE03
:10C520008091730510927305882309F47ACE80E90F
:10C5300094E40E94485680918F05882309F471CEB7
:10C540008FCE8091730510927305882309F4CDCEA8
:10C5500082E09FE50E94485680918F05882309F468
:10C56000C4CE7ECE8091730510927305882309F4A2
:10C57000D7CE8BE59AE50E94485680918F05882397
:10C5800009F4CECE6DCE8091730510927305882389
:10C5900009F4E6CE8FE594E00E94104280918F0569
:10C5A000882309F4DDCE8C8110CF80917305109221
:10C5B0007305882309F4F6CE8DE494E60E9448566C
:10C5C00080918F05882309F4EDCEEDCF9C819813DF
:10C5D00014C0909178052C81291791F080914E011B
:10C5E000882359F06C81651981E02C81291380E042
:10C5F00020E243E654E00E94029E8D818C5FE5CEEE
:10C600008091730510927305882341F39092300551
:10C6100080922F0580918F05882301F3C4CF8093EA
:10C6200072051ECE1092D305109259010E940C770C
:10C630009091F91280FB97F99093F91260E08AECDF
:10C6400091E00E94055C0C94E1430F931F930E94BC
:10C650003CA1009158021091590220915A02309148
:10C660005B02601B710B820B930B97FD0CC089B1B1
:10C6700083FB882780F991E089274A9B8260309B61
:10C680008460809357028091570281709091570285
:10C6900091FD826090919602981749F0813009F1DE
:10C6A00048F0823079F0833091F0809396021F91A8
:10C6B0000F910895913079F09230B9F79091560228
:10C6C00091500CC0992339F09330C1F3EECF9130E3
:10C6D000A9F3923051F7909156029F5F90935602C2
:10C6E000E4CF992359F3933001F7F5CF1F93CF93FC
:10C6F000DF9380912C018F3708F46EC08F57909193
:10C70000C30590939303992309F46BC05D9A8F5FDF
:10C7100080932C018091920391E08927809392036A
:10C7200081110E94256380912B0191E0980F833045
:10C730000CF090E0813009F48AC00CF054C08823DA
:10C7400009F467C090932B01C0919402D091950297
:10C75000209709F42DC0F89413B1147082E00E9460
:10C76000AA2C00C000C01C161D060CF090C02A9A0E
:10C7700000C000C02B9A00C0000082E090E001974A
:10C78000F0F72B9800C000C0112309F482C02A9A48
:10C7900000C000C0789480919402909195021C167C
:10C7A0001D060CF078C00197909395028093940237
:10C7B00080912C0581110E949A3180910A069091F6
:10C7C0000B06009729F0019790930B0680930A06B9
:10C7D000DF91CF911F91089590919303891708F4E9
:10C7E00096CF5D9894CF8230E9F1833009F0AACFDB
:10C7F00080919103811103C087E080939103809120
:10C800009103815080939103882309F49BCF93E097
:10C8100099CF80912A018F5F80311CF480932A0187
:10C8200091CF10922A018091930281110BC0209127
:10C83000B9053091BA053093BC052093BB0581E062
:10C84000809393021092BA051092B9057BCF109293
:10C850007B0087E480937C0080917A0080648093E1
:10C860007A0070CF80917A0086FD0FC040917800E9
:10C87000509179002091B9053091BA05240F351FE8
:10C880003093BA052093B9055DCF92E05BCF2A982B
:10C890006FCF2A987DCF019687CF2F923F924F92EC
:10C8A0005F926F927F928F929F92AF92BF92CF9240
:10C8B000DF92EF92FF920F931F93CF93DF93CDB749
:10C8C000DEB7EC970FB6F894DEBF0FBECDBF8091F8
:10C8D0005F02882369F18091F91200E010E084FF83
:10C8E00023C089E391E10E94DC248BE1E9E3F1E1DB
:10C8F000DE01919601900D928A95E1F710E000E03B
:10C90000BE016F5F7F4FCE0181960E94ACAB1816BF
:10C910003CF4CE0101960E94B5A5080F111DF0CF81
:10C92000CE0181960E94AF260093E6021093E702A3
:10C9300061E081E00E941B4210917905312E85E073
:10C94000810F8CAF212E219484ECA82E8CE1B82E7F
:10C9500098E2892E95E0992E01E0011B2DE2622ECE
:10C9600025E0722E111113C080917805882391F172
:10C9700080914E01882359F081E0909178059111C2
:10C9800080E024E046E355E0622D0E94029E809103
:10C99000F91286FF55C01130D9F4809178058130A5
:10C9A000F1F180914E01882309F455C11F927F92C5
:10C9B0006F920F9381E090917805913009F080E0BB
:10C9C0008F930E944F230F900F900F900F900F9016
:10C9D00082E066C08091730510927305882341F24E
:10C9E0000E948D4480918F05882311F2EC960FB63A
:10C9F000F894DEBF0FBECDBFDF91CF911F910F9195
:10CA0000FF90EF90DF90CF90BF90AF909F908F906E
:10CA10007F906F905F904F903F902F9008958091FE
:10CA2000730510927305882309F4BBCF1092790522
:10CA30000E94F2AC80918F05882309F4B2CFD6CF43
:10CA400084FF2DC0113021F6809178058130D1F01E
:10CA500080914E01882309F4FEC0BF92AF929F924D
:10CA60008F920F9381E090917805913009F080E0EA
:10CA70008F930E944F230F900F900F900F900F9065
:10CA80000F90A6CF8091730510927305882301F350
:10CA90000E94C41C80918F058823D1F2A7CF81E02A
:10CAA00090914E01992309F4D7C0582ED12CC12C56
:10CAB000412E4318852DE090E602F090E702CE1457
:10CAC000DF0408F0C9C05112A5C091E0E91AF108CD
:10CAD000EC18FD0889E391E10E94DC248BE1E9E395
:10CAE000F1E1DE01919601900D928A95E1F7F12C2A
:10CAF000BE016F5F7F4FCE0181960E94ACAB1816CE
:10CB00007CF4CE0101960E94B5A5882389F3EF102D
:10CB10006BC0BE016F5F7F4F8BE995E00E94D0A58F
:10CB2000CE0181960E94AF268091F91290917805EE
:10CB300085FF75C0911363C08091730510927305D2
:10CB4000882309F45CC019821C8280913C1164E541
:10CB500071E1882311F069E371E121E04BE955E0CF
:10CB6000CE0101960E94B526882309F43FC08BE1CF
:10CB7000FE013196A9E3B1E101900D928A95E1F7AA
:10CB80008091F9128F7B8093F912A091EF12AA3055
:10CB900080F481E08A0F8093EF128BE18A9FD001AD
:10CBA0001124AF51BE4EE9E3F1E101900D928A9557
:10CBB000E1F7CE0101960E94AF261092790582E03E
:10CBC00090E0A0E0B0E080937F0590938005A09373
:10CBD0008105B093820581E080938F0510925E02FB
:10CBE00083E080934E0102CFF39482CF0E94677E50
:10CBF0006BE975E082E195E00E94DAAEDACF8091D0
:10CC00004E01882339F081E0911380E041E0642DEA
:10CC10000E94439E8FEFC81AD80A53944BCF9117A6
:10CC200059F080914E018823A9F381E09091780515
:10CC3000911380E040E0EBCF809173051092730573
:10CC4000882379F386E79DE40E94485680918F05FA
:10CC5000882339F3CBCE82E01F5F9CAD911382CE47
:10CC600080937205C3CEFC01A081B1811C92A28188
:10CC7000B3818C918F5F8C930280F381E02D908142
:10CC80008CE0989F800D1124E3EAF1E113AE84AFAC
:10CC90000895FC0184910895FC0180810895119804
:10CCA00000C087FD43C0419800C0119A00C000C079
:10CCB000119800C086FD46C0419800C0119A00C07E
:10CCC00000C0119800C085FD3BC0419800C0119A7A
:10CCD00000C000C0119800C084FD30C0419800C061
:10CCE000119A00C000C0119800C083FD25C0419872
:10CCF00000C0119A00C000C0119800C082FD1AC087
:10CD0000419800C0119A00C000C0119800C081FD78
:10CD10000FC0419800C0119A00C000C0119800C017
:10CD2000419800C0119A00C000C00895419ABCCF3C
:10CD3000419AF0CF419AE5CF419ADACF419ACFCFCD
:10CD4000419AC4CF419AB9CF90E080E0089590E035
:10CD500080E008952091AC04833021F425FD0CC0BF
:10CD600024FD0CC030E0A90102C0559547958A9575
:10CD7000E2F7CA018170089581E0089580E0089586
:10CD80008091C70484FD0BC08091C90487FD07C052
:10CD90009091CA04937081E019F480E0089581E0D5
:10CDA00008952FEB280F2A3108F047C0E22FF0E05A
:10CDB0008091C7049091C804A091C904B091CA049D
:10CDC00004C0B695A795979587952A95D2F780FDCB
:10CDD00002C081700895E355FB4FE081EE2341F1DD
:10CDE0008091D1059091D205E80FF92FF11D808136
:10CDF00090ED980F9A3030F08E3251F4818180534B
:10CE00008A3098F4F093A504E093A40481E0089597
:10CE10008D3211F08B3249F4818190ED980F9A3068
:10CE200088F38E3211F48281EACFF0E0E0E0EACFBD
:10CE30001092A5041092A404E9CF80E00895CF9346
:10CE4000DF9385E40E94D166882309F188E0409150
:10CE5000C7045091C8046091C9047091CA04972F07
:10CE60009170C92F90E0D92FCC0FDD1F71FB2227C5
:10CE700020F930E0220F331F220F331FC22B67FB34
:10CE8000442740F9C42B8C2BDF91CF91089580E08B
:10CE9000DECF0E94D166882341F081E02091A40476
:10CEA0003091A504232B09F480E00895BF92CF921E
:10CEB000DF92EF92FF920F931F93CF93DF936B015B
:10CEC000E9014A3009F4E1C0453109F089C0DB01CC
:10CED0001296ED91FC911281C681D781139A00C000
:10CEE000000086E290E00197F0F7012F0295007FA5
:10CEF00020E1B22EB10E88EF0E944F6600C0000004
:10CF000086E290E00197F0F7103208F0A8C0812F78
:10CF1000807780680E944F66802F0E944F6600C015
:10CF2000000086E290E00197F0F780E80E944F66EB
:10CF300080E00E944F6600C0000086E290E001970A
:10CF4000F0F78AEF0E944F6600C0000086E290E092
:10CF50000197F0F77E01B0E1EB0EF11C8881807F34
:10CF60000E944F6689918295807F0E944F66CE1500
:10CF7000DF05A1F700C0000086E290E00197F0F71E
:10CF80001F5F005F1B11B7CF1398D6011296ED916A
:10CF9000FC9180819281980F92832181921708F0F1
:10CFA000BAC194819F5F94839381890F821710F097
:10CFB0008FEF820F8383458150E0440F551F70E04F
:10CFC00060E0868197810E9474DD81E0DF91CF91DE
:10CFD0001F910F91FF90EF90DF90CF90BF90089539
:10CFE000FB0102811381423309F497C108F49FC108
:10CFF000463409F48CC1473409F494C14B3329F702
:10D0000089812B81D80112967C91129713963C91BD
:10D01000213009F4D1C1233009F0B2C148EF480FE3
:10D02000582F91E0341708F490E031E0541708F0DD
:10D0300030E0492F432B61E0571708F460E04623A6
:10D0400019F4932309F4C1CFFA8030E0F901EF5EBF
:10D05000FD4FD080235F3D4FF901E080AAC180EEF3
:10D06000810F8068807F0E944F66812F8295807F2C
:10D070000E944F6600C0000086E290E00197F0F742
:10D0800080E80E944F6680E854CF0B9A1398399A33
:10D090004198099A119A139A00C0000086E290E024
:10D0A0000197F0F788E790E0CEE9DFE0FE013197E5
:10D0B000F1F70197D9F788EF0E944F6600C0000092
:10D0C00086E290E00197F0F780E20E944F6680E0F0
:10D0D0000E944F6600C0000086E290E00197F0F7E2
:10D0E00080E00E944F6680E80E944F6600C000000A
:10D0F00086E290E00197F0F780E00E944F6680E1C1
:10D100000E944F6600C0000086E290E00197F0F7B1
:10D11000CE010197F1F7CE010197F1F7CE0101970A
:10D12000F1F7CE010197F1F7CE010197F1F7CE01AA
:10D130000197F1F7CE010197F1F7CE010197F1F7D1
:10D14000CE010197F1F7CE010197F1F7CE010197DA
:10D15000F1F7CE010197F1F7CE010197F1F7CE017A
:10D160000197F1F72197F1F780E20E944F6680E482
:10D170000E944F6600C0000086E290E00197F0F741
:10D1800080E20E944F6680E60E944F6600C0000069
:10D1900086E290E00197F0F7D0E0C0E08C2F807736
:10D1A00080680E944F668D2F0E944F6600C000006D
:10D1B00086E290E00197F0F780E80E944F6680E0F9
:10D1C0000E944F6600C0000086E290E00197F0F7F1
:10D1D0008AEF0E944F6600C0000086E290E001974F
:10D1E000F0F780E2119800C0419800C0119A00C089
:10D1F00000C0119800C0419800C0119A00C000C042
:10D20000119800C0419800C0119A00C000C0119848
:10D2100000C0419800C0119A00C000C0119800C021
:10D22000419800C0119A00C000C0119800C04198F8
:10D2300000C0119A00C000C0119800C0419800C001
:10D24000119A00C000C0119800C0419800C0119A06
:10D2500000C000C0119800C0419800C0119A00C0E1
:10D2600000C0119800C0419800C0119A00C000C0D1
:10D27000119800C0419800C0119A00C000C01198D8
:10D2800000C0419800C0119A00C000C0119800C0B1
:10D29000419800C0119A00C000C0119800C0419888
:10D2A00000C0119A00C000C0119800C0419800C091
:10D2B000119A00C000C0119800C0419800C0119A96
:10D2C00000C000C000C00000E6E2F0E03197F0F7D7
:10D2D000815009F087CF88EF0E944F6600C00000A0
:10D2E00086E290E00197F0F7CF5FD05FC03209F09F
:10D2F00055CF80E00E944F6680EC0E944F6600C0D0
:10D30000000086E290E00197F0F713985ECEF801F6
:10D31000858188835ACE80E059CEB901C8010E9428
:10D32000B4A153CED80111968C9188834ECE44314E
:10D3300091F0473109F049CE1882D80112968C91AC
:10D340001297898315968C91159781508A8313962D
:10D350008C918B833ACED80115964C91159750E05D
:10D36000440F551F70E060E016968D919C910E94CD
:10D3700074DDF8011282808181508383148225CE6E
:10D38000381708F422CE871708F41FCEFA80E12C54
:10D39000D12C243070F459CEBE01C8010E94B4A132
:10D3A000898198819D0D98838E0D8983FF0C09F4E6
:10D3B0000CCEF7FEF6CFF0CF58E0580F482F31CE05
:10D3C000EF92FF920F931F93CF93DF93EC018B01AA
:10D3D0007A018A859B858617970731F08881998124
:10D3E0000E94FDA31B870A87B701888199810E944B
:10D3F000AB9E2E813F81820F932F911D9F838E8341
:10D4000090E080E0DF91CF911F910F91FF90EF901E
:10D4100008959F92AF92BF92CF92DF92EF92FF92C8
:10D420000F931F93CF93DF93EC018B01942EA52EC6
:10D430008A859B858617970731F0888199810E949C
:10D44000FDA31B870A8788859985019649F5BC80CD
:10D450000A818E81080FC880D980D6015596ED913A
:10D46000FC91C6010995B80EE92CFA2C10E0F701E1
:10D4700021917F01211127C08E819F81810F911DF4
:10D480009F838E8390E080E0DF91CF911F910F9179
:10D49000FF90EF90DF90CF90BF90AF909F90089556
:10D4A0000E811F81692D7A2D888199810E94AB9E02
:10D4B000800F912F911D288539852817390738F657
:10D4C00081E090E0E1CF4B2D602FC6010E9455A472
:10D4D000080F180FCCCFDF92EF92FF920F931F939C
:10D4E000CF93DF93EC01D62E1CAD0BAD7C0184E015
:10D4F000E80EF11CE98DFA8DC7010995412F480FFF
:10D500002D2D602FC7010E9455A49BAD890F8BAFB5
:10D5100081E090E0DF91CF911F910F91FF90EF900C
:10D52000DF9008952F923F924F925F926F927F9279
:10D530008F929F92AF92BF92CF92DF92EF92FF9223
:10D540000F931F93CF93DF93162F072F242EFC01E9
:10D5500080809180A280B380C501B40120E13EE0CB
:10D5600040E050E00E9488DAE22ED32EC22FD32F63
:10D570008CE3482E512C612C712CC501B401A30100
:10D5800092010E9488DAC62E372ECA01B901A30182
:10D5900092010E9488DAF62E772E222059F1C501D9
:10D5A000B40120E831E541E050E00E9488DA6901E9
:10D5B0007F92FF92CE0168E170E00E94DEDA9F93D5
:10D5C0008F933F932F9384EF9CE19F938F930F93BF
:10D5D0001F930E94D7D3EDB7FEB73A960FB6F894D3
:10D5E000FEBF0FBEEDBF88E0FAE0CF16D104C8F051
:10D5F00089E017C0209741F53F92CF927F936F93B8
:10D6000088EE9CE19F938F930F931F930E94D7D333
:10D610008DB79EB708960FB6F8949EBF0FBE8DBF0C
:10D6200085E0DF91CF911F910F91FF90EF90DF90F8
:10D63000CF90BF90AF909F908F907F906F905F90B2
:10D640004F903F902F900895C436D105A8F47F9352
:10D650006F93DF92EF928CED9CE19F938F930F93EA
:10D660001F930E94D7D3EDB7FEB738960FB6F89444
:10D67000FEBF0FBEEDBFD4CF7F936F93DF92EF92CB
:10D6800082ED9CE19F938F930F931F930E94D7D3BA
:10D690008DB79EB708960FB6F8949EBF0FBE8DBF8C
:10D6A00086E0BFCF8091A4049091A504009731F04B
:10D6B0004AE050E070E060E00C942DD160E070E052
:10D6C000CB0108950E94526B97FD0CC00E94526BD3
:10D6D0006F3F71058105910509F034F40E94526B8A
:10D6E000862F089580E008958FEF08958091A40417
:10D6F0009091A504892B41F00E94626B91E0811109
:10D7000001C090E0892F089591E0FCCFCF93DF9383
:10D71000C82FD62F0E944967882321F0DF91CF912F
:10D720000C94766B8C2F0E94D166811101C08D2FD5
:10D73000DF91CF9108950E94526BCB010895CF9352
:10D74000DF93EB010E944967882321F0DF91CF919D
:10D750000C949B6BCE01DF91CF9108958091A4042E
:10D760009091A504009731F04AE050E070E060E04D
:10D770000C945BD260E070E0CB0108950F931F938F
:10D78000CF938091A4049091A5040097E9F0FC0147
:10D790008F01C1912C2F2F7D81F0C53411F0C5363A
:10D7A000B9F7F801108270E060E00E94CFCFF80175
:10D7B000C083CF911F910F91089570E060E0CF91E9
:10D7C0001F910F910C94CFCF60E070E0CB01F1CFAF
:10D7D000CF92DF92EF92FF92CF93C82F0E943CA18D
:10D7E0006B017C0124EA30E74DE75FE360910201C1
:10D7F0007091030180910401909105010E9440D431
:10D8000087FD18C08AEF90E0A0E0B0E08C0D9D1D70
:10D81000AE1DBF1D8093160590931705A0931805A4
:10D82000B0931905C0934301CF91FF90EF90DF9023
:10D83000CF90089580E090E0DC01E8CFCF93809115
:10D84000D304811154C01092DE111092DF11109296
:10D85000E0111092AC111092AB111092AE11109217
:10D86000AD111092B01181E08093AF1182E28093EC
:10D87000B1111092B6111092B511EAECF1E128ED58
:10D8800031E18FEF81932E173F07E1F7C1E0C0939D
:10D89000C71125EC38E93093BD112093BC11C0931A
:10D8A000BE111092BF111092C01190E49093C1115B
:10D8B0001092C21124EC38E93093D9112093D81179
:10D8C0002BE331E03093AA112093A9119EE19093AC
:10D8D000CE1191E19093CF119CE19093CC11809364
:10D8E000CB118093CA110E94F2A1C093D30481E0AE
:10D8F0008093D20483E19DE19093191180931811D4
:10D9000010921B1110921A1153985B9A52985A9ABE
:10D910003898409A0E94256310925602CF9108953C
:10D92000FC0180E0309749F09491992331F0907C8C
:10D93000903809F08F5F3196F7CF0895009751F036
:10D94000FC0180E09191992331F0907C9038D1F3E3
:10D950008F5FF8CF80E00895AF92BF92CF92DF92B1
:10D96000EF92FF920F931F93CF93DF93EC015B0134
:10D970008A01FB01099587FD16C0C82ED12CF12C18
:10D98000E12C2196F801C082D182E282F382CE019D
:10D99000DF91CF911F910F91FF90EF90DF90CF908B
:10D9A000BF90AF900895982F907E903CA9F48F710E
:10D9B00090E0B0E0A0E06C017D0156E0CC0CDD1CF5
:10D9C000EE1CFF1C5A95D1F7CE010196F501099581
:10D9D0008F73C82A2296D6CF982F907F903E11F54C
:10D9E0008F7090E0B0E0A0E06C017D0136E0CC0CDF
:10D9F000DD1CEE1CFF1C3A95D1F7CE010196F50116
:10DA000009958F73C82A46E0CC0CDD1CEE1CFF1C68
:10DA10004A95D1F7CE010296F50109958F73C82A70
:10DA20002396B0CF982F987F903F79F5877090E03C
:10DA3000B0E0A0E06C017D0186E0CC0CDD1CEE1CAA
:10DA4000FF1C8A95D1F7CE010196F50109958F73D8
:10DA5000C82A96E0CC0CDD1CEE1CFF1C9A95D1F771
:10DA6000CE010296F50109958F73C82A26E0CC0CE9
:10DA7000DD1CEE1CFF1C2A95D1F7CE010396F501A3
:10DA800009958F73C82A24967DCF982F907C903863
:10DA900041F4807C803869F42196CE01F501099526
:10DAA000F8CF8E7F8D3F28F02196CE01F5010995A4
:10DAB000F8CFC12CD12C760165CF9CE0899F802DB9
:10DAC000112491E0980F9093D1042CE0280F20931B
:10DAD000970530E02E5F3F4F4091DB114217130650
:10DAE00019F014F080E008952091DD119217D0F71D
:10DAF000662341F08E5F0E941DA3809197058E5F83
:10DB00000E941DA3809197059091DB11891750F316
:10DB10002091DD119091D104291720F31092DE118C
:10DB20008093DF1181E008952091D004022E000C33
:10DB3000330B8217130641F08093D00468E37EE133
:10DB400087EA91E10C94FDA30895CF92DF92EF92C2
:10DB5000FF920F931F93CF93DF93CDB7DEB72C9730
:10DB60000FB6F894DEBF0FBECDBF6F3F71058105C4
:10DB7000910509F0D0F483EA91E10E946B6AE0918B
:10DB8000AB11F091AC113196849190E02C960FB6C8
:10DB9000F894DEBF0FBECDBFDF91CF911F910F91E3
:10DBA000FF90EF90DF90CF900895F090DE11E0901D
:10DBB000DF112091D20421110FC042EB5CE16E2DE8
:10DBC0008F2D0E94C1A490E080E0F80EF092DE114B
:10DBD000E092DF119927DACFC090AB11D090AC1151
:10DBE00027EA31E13A8329832F2D30E03C832B83D0
:10DBF0002E2D30E03E832D8318861F822FEF3FEFBE
:10DC00003A8729871C861B8609E01AE69E012F5F4A
:10DC10003F4FAB01BC01C6010E94D699B60187EA0D
:10DC200091E10E94FDA38F819885CFCF4F925F92A3
:10DC30006F927F928F929F92BF92CF92DF92EF92DC
:10DC4000FF920F931F93CF93DF93CDB7DEB7289743
:10DC50000FB6F894DEBF0FBECDBF7C016A0149014B
:10DC6000FB0190818CE0989F800D1124982FF70183
:10DC70002081822F880F820F880F8093DE1190936E
:10DC8000DF114115510571F1FA82E9827C836B83C2
:10DC9000011121C0AE014B5F5F4FB401C6010E946C
:10DCA000AC6C6C016D817E818F81988561157105E9
:10DCB00081059105B9F00E94A56DF70180818F5F04
:10DCC0008083853138F3CE0101960E943366E2CF1E
:10DCD000B12C860129C08A01B12C26C045284628CE
:10DCE0004728B1F728960FB6F894DEBF0FBECDBF18
:10DCF000DF91CF911F910F91FF90EF90DF90CF9028
:10DD0000BF909F908F907F906F905F904F900895FD
:10DD1000B39407C0B1102EC001151105C9F20F5FF1
:10DD20001F4F01151105A9F2AE014B5F5F4FB40102
:10DD3000C6010E94AC6C6C014D805E806F8078845F
:10DD40004114510461047104A9F0F0E24F1651042A
:10DD500061047104F9F2D301C2018D97A109B109DF
:10DD60000297A105B10530F04BE24416510461045D
:10DD7000710471F6F7018081482F4B0D5527551F0F
:10DD80004631510534F0853020F0CE0101960E94D5
:10DD9000336681E0411451046104710409F480E0A8
:10DDA000B80EF70180818B0D8083BB2009F496CFDC
:10DDB000BA94AE014B5F5F4FB401C8010E94AC6CD6
:10DDC0008C016D817E818F8198850E94A56DEDCF3C
:10DDD000CF93DF93FC0125AD211104C021E025AFD5
:10DDE0000E94F2A1C091A911D091AA11E091D8117D
:10DDF000F091D91182E00995E091D811F091D911F3
:10DE000081E0099530E020E044E1BE0187EA91E13C
:10DE10000E94EEA12AED31E147E1BE0187EA91E1DE
:10DE20000E94EEA1E091D811F091D91180E0DF912C
:10DE3000CF9109944F925F926F927F928F929F92AF
:10DE4000AF92BF92CF92DF92EF92FF921F93CF9348
:10DE5000DF9300D000D0CDB7DEB70E943CA16B01AC
:10DE60007C01809143018F3FC1F10E943CA18090D1
:10DE7000160590901705A0901805B090190568191F
:10DE800079098A099B0997FD28C080917B1190919F
:10DE90007C118F5F8F70891701F1E091430180E061
:10DEA00090E0A5E0B3E4E53050F424E0E29FF00117
:10DEB0001124EB5EFD4F80819181A281B381898322
:10DEC0009A83AB83BC83BE016F5F7F4F82E691E094
:10DED0000E94CCC68FEF809343010E9425638091FE
:10DEE000570282FF33C080912105811131C091E03A
:10DEF000909321058091D305892780937305109213
:10DF0000D30583E080934E01109257020E943CA1FA
:10DF10006C507E4F8F4F9F4F609358027093590201
:10DF200080935A0290935B0268E873E182E090E08C
:10DF30000E94CA4116E0115059F00E946E4162E001
:10DF400070E080E090E00E949DA0F5CF1092210546
:10DF50008091B5059091B605A091B705B091B8052F
:10DF6000A7019601281B390B4A0B5B0BDA01C9018B
:10DF7000B7FF05C080915E02882309F4ECC1D70188
:10DF8000C6018C599F4FAF4FBF4F8093B5059093FB
:10DF9000B605A093B705B093B80560915602062E5A
:10DFA000000C770B77FF03C0719561957109909113
:10DFB000560280912005981367C0633008F064C052
:10DFC000109256028091560280932005643008F02A
:10DFD0006BC0809173058111E9C08091A11190916E
:10DFE000A21137E78A31930709F004C180914C01EF
:10DFF000882309F4EDC0815080934C010E949B302E
:10E000008090F5059090F605A090F705B090F80582
:10E0100081110E94A830D501C4013AE0B695A795B8
:10E02000979587953A95D1F7009751E0A507B105E7
:10E0300020F08FEF9FEFA0E0B0E0969587952091BC
:10E040004E01211106C130915E023111B1C18091A2
:10E05000A1119091A2118A51974709F490C1809122
:10E06000620281118CC180911C0590911D05A091C7
:10E070001E05B0911F05C81AD90AEA0AFB0AF7FC67
:10E080008CC10E94E14389C1633009F09BCF80912C
:10E09000560287FD07C081E0880F880F80935602E3
:10E0A00064E090CF8FEFF8CF8091940521E030E0CD
:10E0B00040E050E0882309F456C08090900590908D
:10E0C0009105A0909205B090930581149104A1044C
:10E0D000B104E9F170E090E080E00E9445D420E0D6
:10E0E00030E040E85EE30E94A6D42B013C01C7016A
:10E0F000B601681979098A099B090E9445D49B01D8
:10E10000AC01C301B2010E94CCDB20E030E04AE761
:10E1100054E40E94A6D44B015C0120E030E040EAC8
:10E1200052E40E94CCDC24E630E040E050E087FF7F
:10E1300012C020E030E040EF51E4C501B4010E947C
:10E14000CCDC2AE030E040E050E087FF04C021E072
:10E1500030E040E050E0C0929005D0929105E0920E
:10E160009205F0929305A09156020A2E000CBB0B6B
:10E170000E9440DB24E030E040E050E00E9406DBFB
:10E1800080917F0590918005A0918105B0918205D5
:10E19000820F931FA41FB51F80937F059093800566
:10E1A000A0938105B093820510925602D701C60153
:10E1B0008856954CAF4FBF4F80931C0590931D051B
:10E1C000A0931E05B0931F0581E080934E0105CFFB
:10E1D0008CE080934C0180911A0590911B0500976B
:10E1E00029F0019790931B0580931A0581E0809395
:10E1F0004E0104CF8D54944609F000CF80914C011C
:10E200009FEF980F90934C018111F8CE8091950566
:10E210008F5F809395059091960524E0891708F00B
:10E220002CE020934C01981710F41092950581E092
:10E2300080934E01D701C6018856954CAF4FBF4F12
:10E2400080931C0590931D05A0931E05B0931F0598
:10E25000D5CE009741F040911A0550911B05481703
:10E26000590708F0F4CE80915E02811112C022306D
:10E2700038F0243008F441C0243011F410924E01DB
:10E2800083EA91E10E94E86E81E080935F028093CF
:10E290005E0283E00E94946D81E08093C711E0915B
:10E2A000A111F091A211099510925F0280915E0276
:10E2B000811127C0109273058091A1119091A21134
:10E2C0008A51974709F0CBCE0E943CA1DC01CB01DB
:10E2D0008C199D09AE09BF0980901A0590901B0505
:10E2E000B12CA12C88169906AA06BB0608F0AFCE61
:10E2F00090931B0580931A05AACE81E080934E016E
:10E30000BFCF87EA91E10E94CBA391E0811101C0C8
:10E3100090E090935E02882369F28091A111909120
:10E32000A2118A519747B9F40E943CA1DC01CB01AC
:10E330008C199D09AE09BF09C0901A05D0901B0524
:10E34000F12CE12CC816D906EA06FB0620F49093BE
:10E350001B0580931A050F900F900F900F90DF917F
:10E36000CF911F91FF90EF90DF90CF90BF90AF9033
:10E370009F908F907F906F905F904F90089558E995
:10E38000C50E5AE3D51EE11CF11CC0921C05D092AB
:10E390001D05E0921E05F0921F0580915E0281111D
:10E3A000DACF80914E018130B1F610924E01D3CF79
:10E3B000009709F46ECF4FCFCF92DF92EF92FF928A
:10E3C0000F931F93CF93DF93CDB7DEB72C970FB684
:10E3D000F894DEBF0FBECDBFF090DE11E090DF11EC
:10E3E0002091D20421111DC042E95CE16E2D8F2DD8
:10E3F0000E94C1A490E080E0F80EF092DE11E0925D
:10E40000DF1199272C960FB6F894DEBF0FBECDBF53
:10E41000DF91CF911F910F91FF90EF90DF90CF9000
:10E420000895C090AB11D090AC1127EA31E13A8346
:10E4300029832F2D30E03C832B832E2D30E03E832B
:10E440002D8318861F827A8769871C861B8609E0C0
:10E450001AE69E012F5F3F4F49E456E6BC01C60114
:10E460000E949A9AB60187EA91E10E94FDA38F81EA
:10E470009885C2CF8F929F92AF92BF92CF92DF9238
:10E48000EF92FF920F931F93CF93DF9300D000D0B2
:10E49000CDB7DEB77C01062F5A01122F862F660FEB
:10E4A000990B9C01275F3D4F690186E0882E912CD6
:10E4B00011160CF040C0AE014F5F5F4F69E476E685
:10E4C000C7010E94AC6C7C0169817A818B819C813F
:10E4D000611571058105910571F16D337105810536
:10E4E000910509F462C06E3771058105910509F443
:10E4F0005CC06A3271058105910579F507FF12C08C
:10E5000089E09DE10E3F11F085E09DE136E01302C8
:10E51000B00111240E94DC7166E070E00E94F2DA22
:10E52000161B73C065E470E080E090E00E94A56D6A
:10E530001150E9F510E0812F0F900F900F900F9080
:10E54000DF91CF911F910F91FF90EF90DF90CF90CF
:10E55000BF90AF909F908F900895643271058105B0
:10E56000910579F4A114B104E1F0E6E01E02B001D6
:10E570001124C5010E94DC71B4010E94F2DA161B5D
:10E5800097CF603471058105910559F41150F6015A
:10E590006081062E000C770B880B990B0E94A56DED
:10E5A00087CF0E94A56D115083CF07FDA9CF61E0F1
:10E5B00089819A81AB81BC81CD97A105B10509F410
:10E5C00060E0600F6A30ACF01150862F6AE00E9464
:10E5D000D0DA092F682F880F770B605D7F4F072EE9
:10E5E000000C880B990B0E94A56D112309F4A2CF92
:10E5F000602F062E000C770B605D7F4F072E000CFE
:10E60000880B990B0E94A56D1150112309F492CF2C
:10E6100086E01802B0011124C7010E94DC7166E097
:10E6200070E00E94F2DA161B86CFE3EAF1E183AFD5
:10E6300064AF6FEF7FEFCA010C94DC71CF92DF9271
:10E64000EF92FF920F931F93CF93DF93CDB7DEB777
:10E650002C970FB6F894DEBF0FBECDBFF090DE1141
:10E66000E090DF112091D20421111DC042E75CE14E
:10E670006E2D8F2D0E94C1A490E080E0F80EF092E4
:10E68000DE11E092DF1199272C960FB6F894DEBFC9
:10E690000FBECDBFDF91CF911F910F91FF90EF90F3
:10E6A000DF90CF900895C090AB11D090AC1127EAC5
:10E6B00031E13A8329832F2D30E03C832B832E2DAB
:10E6C00030E03E832D8318861F827A8769871C86F7
:10E6D0001B8609E01AE69E012F5F3F4F4CE456E689
:10E6E000BC01C6010E949A9AB60187EA91E10E9494
:10E6F000FDA38F819885C2CF8F929F92AF92BF92D8
:10E70000CF92DF92EF92FF920F931F93CF93DF93FD
:10E710005B01C42F790141FB662760F90E945D6DA2
:10E72000882309F462C0D12CC12CA114B10439F0A2
:10E73000C5010E94906C96E0899F6001112410E051
:10E7400000E0E114F10429F0C7010E949E6C082F3B
:10E7500010E0C0FF21C080E890E08C199D094AEFCD
:10E7600040039001419F300D1124820F931F6CE0F4
:10E7700070E00E94F2DA4B01C0E8D0E081E0881A34
:10E78000910897FC0BC060E270E080E090E00E948E
:10E79000A56DC81BD90BF2CFC0E8D0E0CD2899F009
:10E7A000CE0166E070E00E94DEDA262F40919905E6
:10E7B00050919A0560919805C5010E943A7296E0C1
:10E7C000899FE0011124012B31F0BE01C7010E9495
:10E7D0001E73C81BD90BC730D10538F060E270E05A
:10E7E00080E090E00E94A56DF4CFDF91CF911F9162
:10E7F0000F91FF90EF90DF90CF90BF90AF909F90E0
:10E800008F9008956FEF7FEF0C941E73AF92BF92BD
:10E81000CF92DF92EF92FF920F931F93CF93DF93EC
:10E820005C016B010E94906CE82EC6010E949E6CF8
:10E83000F12C03E110E0081B1109C5E20E151F05BC
:10E840000CF4CFE18C2F90E09C012E5F3F4F409164
:10E85000DB114217130609F0CCF509972091DD1161
:10E86000281719069CF14091990550919A056091DD
:10E8700098051092DE11C093DF1125E1C5010E94B9
:10E880003A72D1E0C114D104B1F06AE370E080E0E3
:10E8900090E00E94A56D0E151F05D4F4C45F809111
:10E8A000DB11C81740F02091DD114C2F4950550B5A
:10E8B000241715067CF4DF91CF911F910F91FF90E3
:10E8C000EF90DF90CF90BF90AF900895D0E0DACF77
:10E8D000DD2389F3802F880F080F000F0093DE11CE
:10E8E000C093DF1160E270E080E090E00E94A56DCF
:10E8F000C601DF91CF911F910F91FF90EF90DF90B4
:10E90000CF90BF90AF900C9402748F929F92AF9271
:10E91000BF92CF92DF92EF92FF920F931F93CF930C
:10E92000DF93CDB7DEB72C970FB6F894DEBF0FBEDE
:10E93000CDBF982F862F5A017901D02E692F0E94C2
:10E940005D6D882309F489C01091D204C7010023AA
:10E9500081F10E94906CC82E8090AB119090AC1108
:10E96000111143C01FEF23E12C19409199055091DB
:10E970009A0560919805C5010E943A72CC2009F46D
:10E980006CC0B6E08B9F500111246AE370E080E018
:10E9900090E00E94A56D57E0A516B10408F442C0AE
:10E9A00060E270E080E090E00E94A56DA81AB90ACC
:10E9B000F2CF0E949E6CC82E8090AB119090AC114B
:10E9C000112381F2FE0133968AE0DF011D928A95C0
:10E9D000E9F787EA91E19A83898300EE19E69E01BF
:10E9E0002F5F3F4F4CE456E612C0FE0133968AE09B
:10E9F000DF011D928A95E9F787EA91E19A8389837D
:10EA000000EE19E69E012F5F3F4F49E456E6B7013D
:10EA1000C4010E949A9AB40187EA91E10E94FDA381
:10EA20001F81A1CF40919705212F30E0A6E0CA9E1B
:10EA3000C00111242E5F3F4F281739070CF49C01A9
:10EA400080E8821B8093DE114093DF11DD20C1F04E
:10EA50006FEF7FEFC7010E94DC712C960FB6F89420
:10EA6000DEBF0FBECDBFDF91CF911F910F91FF9001
:10EA7000EF90DF90CF90BF90AF909F908F900895D0
:10EA8000C7010E940274E9CFCF93DF93DB01F90144
:10EA90009C919130C1F0943080F094509C938830D8
:10EAA000D1F480819181009771F0019791838083E7
:10EAB000480F591FEA01188206C08C3539F49C5F53
:10EAC0009C93943041F4DF91CF9108958B3339F7C3
:10EAD00081E08C93F8CF20813181B9016F5F7F4F46
:10EAE00071836083420F531FEA0188838081918183
:10EAF0008F3591056CF7E7CF0F931F9381E000915D
:10EB0000F5121091F6122091F7123091F8124091FF
:10EB1000F1125091F2126091F3127091F4120417F5
:10EB200015072607370708F480E01F910F91089515
:10EB30008F929F92AF92BF92CF92DF92EF92FF920D
:10EB40000F931F93CF93DF931092CC041092CB04BA
:10EB50002FE32093CF041092CE041092CD04109294
:10EB6000C7041092C8041092C9041092CA049C01F0
:10EB7000F90190812F5F3F4F9032D1F39E34C9F459
:10EB8000818190ED980F9A3020F08D3211F08B3208
:10EB900081F432969F012F5F3F4F808180538A30EE
:10EBA00008F46BC09F012F5F3F4F8081803209F4D2
:10EBB00066C0F093D205E093D1058F010F5F1F4F20
:10EBC000C0816AE270E0C8010E948EDD009731F0DA
:10EBD000FC01319780818032E1F31182CD3421F044
:10EBE000C43511F0C734E1F5F80180810F5F1F4F84
:10EBF0008032D1F380538A3098F5C093CF0430E04F
:10EC000020E06AE0AF014F5F5F4F629FC001639FEA
:10EC1000900D11249C01205331098081280F311D52
:10EC200087FD3A95FA01808180538A3058F33093FA
:10EC3000CE042093CD04DF0131968C918032D9F33C
:10EC4000CD3449F52E31310539F0D8F4273131056D
:10EC500019F02C313105F9F4B093CC04A093CB0416
:10EC6000DF91CF911F910F91FF90EF90DF90CF90A8
:10EC7000BF90AF909F908F900895F9018BCFF901CD
:10EC800091CF2537310538F02737310528F3203A61
:10EC900083E0380709F3D091D10540E050E0BA0194
:10ECA00010E000E0C12CD12C7601C394FD01319617
:10ECB0008C91882309F47FC08132E1F4CD34D1F402
:10ECC00020323105B9F44093C7045093C8046093CF
:10ECD000C9047093CA04F093CC04E093CB0463E2BC
:10ECE00070E0CF010E948EDD009709F4B9CFFC01DE
:10ECF0001082B6CF81548A3108F058C0DF019D914F
:10ED0000903291F0A0EDA90FAA30E8F09E3271F494
:10ED1000918190539A30B8F00115110519F48F01C3
:10ED20000150110990E013C0FD01E8CF9D3211F0B0
:10ED30009B3291F79181A0EDA90FAA3020F09E326D
:10ED400059F79281E6CF9E2F9D1B309759F3A82F3C
:10ED5000B0E04601570104C0880C991CAA1CBB1CDA
:10ED60008A95D2F7482959296A297B29A355BB4F8F
:10ED70009C9380818154DF018A3108F497CFDF01B1
:10ED80008191882309F492CF90ED980F9A30B8F3CF
:10ED900093ED980F923098F38B3289F3CD01019661
:10EDA000EC91E03209F082CFDC01F8CF01151105BA
:10EDB00001F78D01DECF1093CC040093CB04409378
:10EDC000C7045093C8046093C9047093CA0448CF21
:10EDD000CF92DF92EF92FF926B017C0183E3C81622
:10EDE000D104E104F10470F082E3C81AD108E1080B
:10EDF000F10862E370E080E090E00E949DA00E9434
:10EE0000E128ECCFC701B6010E949DA0FF90EF90D2
:10EE1000DF90CF900C94E1289091F91294FB882711
:10EE200080F994FF06C081E090912111911101C0F9
:10EE300080E008954F925F926F927F928F929F929F
:10EE4000AF92BF92CF92DF92EF92FF920F931F93F8
:10EE5000CF93DF93CDB7DEB72C970FB6F894DEBF14
:10EE60000FBECDBF1092940580917305109273056B
:10EE70008823F9F020E040E070E060E087E690E66B
:10EE80000E9479422C960FB6F894DEBF0FBECDBF1C
:10EE9000DF91CF911F910F91FF90EF90DF90CF9076
:10EEA000BF90AF909F908F907F906F905F904F90AA
:10EEB0000895209106013091070140917F055091FE
:10EEC0008005CA01820F931F2436310509F0EDC376
:10EED0004730510544F006978A3091050CF0F4C391
:10EEE0008AE090E0FBC306964A3F5F4FACF3809107
:10EEF0005F02882309F4D3C16091C1057091C205F6
:10EF0000072E000C880B990B0E9447D411E020912A
:10EF1000BD053091BE054091BF055091C0050E94CE
:10EF2000CCDC18160CF010E01093150580906A01E7
:10EF300090906B01A0906C01B0906D0120E030E0EA
:10EF4000A901C501B4010E9440D4C12CD12CE0EA32
:10EF5000EE2EE0ECFE2E87FD06C0C12CD12C70EA0F
:10EF6000E72E70E4F72E20E030E040E251E4C501E6
:10EF7000B4010E94A6D420E030E048EC52E40E94A4
:10EF8000A6D4A70196010E9449DB20E030E040E2D0
:10EF900051E40E94CCDB0E943EDC6B017C0180E2EC
:10EFA000F7FE09C0F094E094D094C094C11CD11C29
:10EFB000E11CF11C8DE24090620150906301609071
:10EFC0006401709065012091660130916701409164
:10EFD00068015091690129873A874B875C87809344
:10EFE000630260E230E1C31637E2D306E104F104C4
:10EFF0008CF0C701B60120E137E240E050E00E940A
:10F0000006DBCA01B9012AE030E040E050E00E948E
:10F0100006DB605D6093640260E248EEC41643E084
:10F02000D406E104F1048CF0C701B60128EE33E008
:10F0300040E050E00E9406DBCA01B9012AE030E05E
:10F0400040E050E00E9406DB605D60936502C7010E
:10F05000B60124E630E040E050E00E9406DB6AE0C2
:10F06000862E912CA12CB12CCA01B901A5019401C5
:10F070000E9406DB605D60936602C701B601A501D0
:10F0800094010E9406DB162FCA01B901A501940163
:10F090000E9406DB112309F431C38EE280936702DC
:10F0A000605D60936802105D1093690263E672E030
:10F0B0008DE095E00E9499DD20E030E0A901C301D8
:10F0C000B2010E9440D420E030E040E05FEB87FDD9
:10F0D00004C020E030E040E05FE3C301B2010E94E1
:10F0E00049DB0E943EDCCB010E94B340BC0188E0BA
:10F0F00095E00E9499DD20E030E0A90169857A85DC
:10F100008B859C850E9440D420E030E040E05FEB9E
:10F1100087FD04C020E030E040E05FE369857A8548
:10F120008B859C850E9449DB0E943EDCCB010E94BE
:10F13000B340BC0183E095E00E9499DD0E94AF5B83
:10F140008C010E941B40D62E6D837E838F8398870F
:10F15000809142018017C1F100934201C80164E629
:10F1600070E00E94DEDA7B0188E48E9DB0018F9D05
:10F17000700D112490E080E00E9445D42AE037ED24
:10F1800043E25CE30E94A6D40E9445DC6093020542
:10F190000115110509F0C4C21092FD041092F30488
:10F1A00080E88093F2048DEF94E0FC010190002050
:10F1B000E9F7CF018D5F9440982F990F890F880F41
:10F1C00090E8981B9093F10480914101D81609F4BE
:10F1D00066C0D092410141E08D819E81AF81B885AA
:10F1E00080389145A140B10508F440E061EE74E03B
:10F1F000CE0105960E94926A982F990F990F891B4C
:10F20000880F80588093E0048D2D837009F047C0EB
:10F210002091DC043091DD044091DE045091DF0444
:10F22000211531054105510509F0A0C20E941B407E
:10F230006B017C010E94AF5BFC01009799F0A0E19B
:10F24000B7E2A81BB90BA70196010E94AADA9F0199
:10F2500050E040E00E9488DA211531054105510552
:10F2600009F084C201151105A9F0A0E1B7E2A01BC5
:10F27000B10B2D813E814F8158850E94AADA9801F9
:10F2800050E040E00E9488DA211531054105510522
:10F2900009F06CC21092F30480E88093F2040E949B
:10F2A0003CA10091D5041091D6042091D70430914F
:10F2B000D8046B017C01C01AD10AE20AF30A970153
:10F2C000860137FD11C02091D40420952093D404E9
:10F2D0006A547C4F8F4F9F4F6093D5047093D60430
:10F2E0008093D7049093D804D090D40411E0D11027
:10F2F00001C010E081E00E94946D8091DB118731A4
:10F3000080F48091DD11843060F036ECE32E3DE135
:10F31000F32E03E126E044E069E087EA91E10E94F0
:10F32000E8A48091DB118431B8F48091DD11823042
:10F3300098F0DD2009F433C28091F905882309F49F
:10F340002EC280E99DE17C0102E123E042E068E613
:10F3500087EA91E10E94E8A48091DB118C3108F0EA
:10F360006EC04090BD055090BE056090BF05709086
:10F37000C005A090C105B090C205843198F4809179
:10F38000DD11883078F08091150580FF0BC282E492
:10F390009DE17C010CE022E048E064E487EA91E131
:10F3A0000E94E8A48091DB11883040F4B7FEFDC1D3
:10F3B00046E25DE167E082E40E9415738091DB1113
:10F3C0008C31B0F48091DD11843190F020E030E098
:10F3D00040E05FE3C301B2010E9449DB0E943EDCD2
:10F3E00077FF0CC246E25DE16CE182E40E94157396
:10F3F0008091DB118C3118F58091DD118431F8F0AA
:10F400008091F9058823D9F024E6829FC001112458
:10F4100081589F4F6FEF70E00E94F2DACB010E949B
:10F42000324127E62093DE112CE12093DF110E9468
:10F43000027465E270E080E090E00E94A56D0E9499
:10F440000C77882379F18091DB11843358F5809112
:10F45000DD118A3238F107E028E04AE26AE287EA01
:10F4600091E10E9470A305E022E04CE262E387EAAA
:10F4700091E10E9470A324E04AE061E38AE20E94E5
:10F4800036A36091A9117091AA1182E38093C311F0
:10F490008BE28093C41123EC31E142E387EA91E1EE
:10F4A0000E94EEA18091DB11853350F48091DD1133
:10F4B000813330F024E04AE461E386E30E9436A31E
:10F4C0008091DB11843368F48091DD11823348F040
:10F4D00002E02091020542E367E387EA91E10E949E
:10F4E00070A38091DB11803358F58091DD11883253
:10F4F00038F18091DB04811751F08091DA04109388
:10F50000DB048F5F833008F0A2C18093DA0480911E
:10F51000DA0481119FC18091FD04882389F08091D4
:10F52000F1048093DE1180E38093DF118DEF94E08E
:10F530000E94027465E270E080E090E00E94A56D98
:10F540008091DB11883208F05DC08091DD118D3132
:10F5500008F458C02BE040E86DE180E00E9436A33B
:10F560008091DB11873208F04DC08091DD118F3121
:10F5700008F448C083E08093DE1106E20093DF11B7
:10F5800068E570E080E090E00E94A56D8BE08093DC
:10F59000DE110093DF11DD2009F48EC188E095E0D3
:10F5A0000E94027488E28093DE1106E20093DF116C
:10F5B00069E570E080E090E00E94A56D80E38093B3
:10F5C000DE110093DF11DD2009F49BC183E095E09B
:10F5D0000E9402748DE48093DE1106E20093DF1135
:10F5E0006AE570E080E090E00E94A56D85E580937B
:10F5F000DE110093DF11DD2009F4A8C18DE095E054
:10F600000E9402748091DB11833348F58091DD11F3
:10F610008B3228F183E00E94946D83E08093DE11A9
:10F6200003E30093DF1166E070E080E090E00E9469
:10F63000A56D81E00E94946D809106019091070173
:10F640000E9432412CE02093DE110093DF110E94D2
:10F65000027465E270E080E090E00E94A56D809108
:10F66000DB11813408F00ECC8091DD11863308F473
:10F6700009CC1092DE118EE38093DF1189EB9EE0BE
:10F680000E949E6C082F863108F085C189EB9EE0B0
:10F690000E940274053109F4F5CB60E270E080E06D
:10F6A00090E00E94A56D0F5FF5CF243631054CF434
:10F6B0008536910504F58A30910534F48AE090E0AE
:10F6C00009C084369105BCF0883EE3E09E0714F043
:10F6D00087EE93E02817390709F409CC90930701C6
:10F6E0008093060110927F0510928005109281058B
:10F6F00010928205FCCB84E690E0F0CF662351F0B7
:10F700008EE280936702605D6093680280E280937E
:10F710006902CCCC80E28093680280936702F6CFC6
:10F720002E2D80E2243628F08E2D64E60E94C4DA65
:10F73000805D8093670290E22A3040F03AE0822FA9
:10F74000632F0E94C4DA0E94C4DA905D909368022D
:10F75000822F6AE00E94C4DA905D9093690267E6A6
:10F7600072E08DEF94E00E9499DD1DCD29833A83EC
:10F770004B835C8381E0203831454140510508F4DA
:10F7800080E0482F63EF74E0CE0101960E94926AF8
:10F79000982F990F990F891B880F80587ECD8AE585
:10F7A0009DE1D1CD8AE29DE1F4CDC5010E943241B7
:10F7B000FC01808193E0803229F4818192E08032E3
:10F7C00009F491E0892F880F880FE92EE81A8E2D11
:10F7D000855B8093DE1187E08093DF1123E030E0CA
:10F7E000291B3109CF01820F931F0E94027469E027
:10F7F00070E080E090E00E94A56DE0CDCB010E941A
:10F800003241FC01808193E0803229F4818192E0D1
:10F81000803209F491E0892F880F880FF92EF81AA9
:10F820008F2D855B8093DE118CE18093DF1123E0C7
:10F8300030E0291B3109CF01820F931F0E9402740F
:10F8400069E070E080E090E00E94A56DD1CD10925B
:10F85000DA045DCE8230B1F48091F304882391F014
:10F8600043E25DE160E386E30E9415738091F20458
:10F870008093DE1180E38093DF1183EF94E00E9498
:10F8800002745ECE8091E104882309F459CE86E3A8
:10F890008093DE1100E30093DF116FEF7FEF80E2D2
:10F8A0009DE10E94DC718091E0048093DE11009361
:10F8B000DF1181EE94E0E3CF87E00E94053D80FFF9
:10F8C00015C028E0E22E25E0F22EF70161917F01BC
:10F8D000662309F467CE6F320CF06FE3062E000C3E
:10F8E000770B880B990B0E94A56DEFCF80912D05AA
:10F8F00080FD54CE6FEF7FEF8BE19DE10E94DC71C4
:10F9000051CE87E00E94053D81FF15C093E0E92EAE
:10F9100095E0F92EF70161917F01662309F45ACE33
:10F920006F320CF06FE3062E000C770B880B990BEF
:10F930000E94A56DEFCF80912D0581FD47CE6FEF21
:10F940007FEF8BE19DE10E94DC7144CE87E00E9455
:10F95000053D82FF15C08DE0E82E85E0F82EF70109
:10F9600061917F01662309F44DCE6F320CF06FE395
:10F97000062E000C770B880B990B0E94A56DEFCF1C
:10F9800080912D0582FD3ACE6FEF7FEF83E19DE1FF
:10F990000E94DC7137CE8091D9041817B1F0009124
:10F9A000B80E1093D90489EB9EE00E949E6C081754
:10F9B00008F050C00F5FE02FF0E0E754F14F808176
:10F9C000807C8038B9F30093B80EE090B80EF12C2B
:10F9D00097012754314F7901C9010E949E6C182F5D
:10F9E00060E870E0C7010E941E73153108F04ACA32
:10F9F00060E270E080E090E00E94A56D143109F4AF
:10FA000041CA60E270E080E090E00E94A56D133191
:10FA100009F438CA60E270E080E090E00E94A56DD1
:10FA2000123109F42FCA212F30E02E5F3F4F4AEFE9
:10FA30004203B001439F700D112460587F4F89EB42
:10FA40009EE00E941E7360E270E080E090E00E9401
:10FA5000A56D18CA1092B80EB8CF8091A805823053
:10FA600061F00E940C77882349F08091F91282FBA3
:10FA7000882780F991E08927089581E008950E9400
:10FA80002D7D811108C01092DC041092DD041092CB
:10FA9000DE041092DF040C94684081E00895909198
:10FAA000C00095FFFCCF8093C6000895CF93DF93ED
:10FAB000EC01FE0184912196882319F00E944F7D6C
:10FAC000F8CFDF91CF9108950F931F93CF938C01BF
:10FAD000C62F8DE49CE10E94567DC8010E94567D90
:10FAE0008AE30E944F7D80E38C0F0E944F7D8AE065
:10FAF000CF911F910F910C944F7DE091F00C81E616
:10FB0000E89FF0011124EE5AF24F8081811107C065
:10FB100082EE9AE20E94567D8AE00C944F7D089511
:10FB2000CF92DF92EF92FF926A017B010E94567D95
:10FB3000C701B601FF90EF90DF90CF900C944D9CE1
:10FB40000E94907D8AE00C944F7D6DE275E10E94E9
:10FB5000A69D6091CD0B7091CE0B8091CF0B9091B3
:10FB6000D00B0E9445D4AB01BC0184E295E10E9418
:10FB7000907D4091FD0B5091FE0B6091FF0B7091B9
:10FB8000000C81E295E10E94907D4091010C509122
:10FB9000020C6091030C7091040C8EE195E10E94BF
:10FBA000907D4091DD055091DE056091DF057091FB
:10FBB000E0058BE195E10C94A07DCF93DF9361ED9F
:10FBC00074E10E94A69DCDEBDBE04CA95DA96EA976
:10FBD0007FA988EC94E10E94907D48AD59AD6AAD53
:10FBE0007BAD85EC94E10E94907D4CAD5DAD6EAD3A
:10FBF0007FAD8EE195E1DF91CF910C94A07DCF9305
:10FC0000DF936DEA74E10E94A69DCDEBDBE04CA191
:10FC10005DA16EA17FA184EA94E10E94907D48A538
:10FC200059A56AA57BA582EF9BE20E94907D4CA519
:10FC30005DA56EA57FA58FEE9BE20E94907D48A9F1
:10FC400059A96AA97BA98CEE9BE2DF91CF910C9414
:10FC5000A07DCF93DF9368E874E10E94A69DCDEB71
:10FC6000DBE0688179818A819B810E9445D4AB0168
:10FC7000BC018FE794E10E94907D6C817D818E8133
:10FC80009F810E9445D4AB01BC0182EF9BE20E94A0
:10FC9000907D688579858A859B850E9445D4AB01D6
:10FCA000BC018FEE9BE20E94907D6C857D858E85E8
:10FCB0009F850E9445D4AB01BC018CEE9BE2DF9195
:10FCC000CF910C94A07D88E794E10C94567D82E757
:10FCD00094E10C94567DCF9384E50E944967C0E07F
:10FCE000882309F10E94626BC82F1816E4F40E9461
:10FCF000677E8DE40E944F7D6091CD047091CE04AB
:10FD000090E080E00E94DF9A8AEB95E10E94567DA8
:10FD10006C2FCC0F770B880B990B0E94499B8AE0C4
:10FD20000E944F7DCFEF8C2FCF9108952F923F925D
:10FD30004F925F926F927F928F929F92AF92BF92FB
:10FD4000CF92DF92EF92FF920F931F93CF93DF93A7
:10FD5000CDB7DEB765970FB6F894DEBF0FBECDBF47
:10FD60009091BC0B93FD7FC0182F0E946B7E8B87F8
:10FD700087FD79C089E40E944967882309F4A4C0FB
:10FD80000E94626B282F30E01216130614F421E053
:10FD900030E0220F331F220F331FF901EF57FD4FC1
:10FDA000808191811C8A0E94382D8091C10590919B
:10FDB000C2058635910574F0112381F00E943F7DC4
:10FDC0000DC082E50E944967882309F485C00E941E
:10FDD0009B6BE9CF0E949E400E94DE9D6091C10511
:10FDE0007091C205072E000C880B990B0E9447D416
:10FDF0002091BD053091BE054091BF055091C005D1
:10FE00000E94CCDC181644F02C8986E59CE1222364
:10FE100029F04C894D8B61C081E69CE19F938F93C3
:10FE20008CE69CE19F938F931F920E94EA5B0F9058
:10FE30000F900F900F900F9031E03D8B4EC060E01F
:10FE400070E0CB0168C0C8010E9440D487FF24C085
:10FE500080915901882321F0109259010E94DE9D62
:10FE60002B812093D00565960FB6F894DEBF0FBEA8
:10FE7000CDBFDF91CF911F910F91FF90EF90DF9059
:10FE8000CF90BF90AF909F908F907F906F905F903A
:10FE90004F903F902F9008953E2C2F2C09831A836A
:10FEA0001C829EC08FE30E944F7DD5C020E030E0D1
:10FEB00040E450E4C301B2010E94CCDC18160CF0FF
:10FEC00019C14601570116C183E50E9449678C8B11
:10FED00081117DCF111175CF1D8A83E50E9449677D
:10FEE000882331F00E949B6B9093570180935601B9
:10FEF00082E40E944967882331F00E949B6B9093B3
:10FF000051018093500186E40E94D166882309F450
:10FF100096CF0E94BE6B6093520170935301809301
:10FF200054019093550151E05B8320E030E0A9013A
:10FF30000E9440D4811101C01B828B818093D00527
:10FF4000112309F490CF9D89992309F48CCF109245
:10FF5000D00581E0809359011D821E821F82188680
:10FF60001C861D861E861F86188AACE3A98BBCE101
:10FF7000BA8B26E42B8B312C212C30E839834FEBC4
:10FF80004A831C82812C912C54016091C10570918F
:10FF9000C205072E000C880B990B0E9447D47B01E9
:10FFA0008C01232D322D49815A810E9440D488230F
:10FFB000B9F02091BD053091BE054091BF0550912B
:10FFC000C0058C89B70181113ECFC8010E9440D481
:10FFD000881F8827881F8C833E2C2F2C09831A8327
:10FFE0000E943CA16B017C01DC01CB012C853D858D
:10FFF0004E855F85821B930BA40BB50BB7FD2EC0FE
:020000021000EC
:10000000D701C60188519C4FAF4FBF4F8C879D874A
:10001000AE87BF878B850E94AD2782E59CE10E9459
:10002000567D81149104A104B10409F43BCFC501AC
:10003000B401605F784D8F4F9F4F6C197D098E0919
:100040009F0928EE33E040E050E00E9488DACA01C0
:10005000B9010E94499B8AE00E944F7D0E9444B1F1
:100060000E943CA16093D8057093D9058093DA056E
:100070009093DB059091BD059987A091BE05AA8755
:100080000091BF051091C005292F3A2FA801632DBB
:10009000722D89819A810E9448DB2B013C0120E06E
:1000A00030E0A9010E94CCDC87FF04C077FA70948D
:1000B00077F8709481149104A104B10409F0F6CE8C
:1000C00020E030E040E85FE3C301B2010E9440D489
:1000D00087FF10C0BD8985E0882E8DE0982EA12C69
:1000E000B12CB11103C0812C912C54018C0C9D1C9E
:1000F000AE1CBF1C2C812223A9F18D819E81AF8172
:10010000B885892B8A2B8B2B61F0D701C6012D81F5
:100110003E814F815885821B930BA40BB50BB7FD15
:1001200021C029853A85A801688979898A899B89AE
:100130000E9448DB20E030E040EC5FE30E9440D4C6
:1001400087FD86CED701C601805A9541AF4FBF4F7C
:100150008D839E83AF83B8879985988BAA85A98B59
:100160000A8B1B8B80915901882309F471CE81146D
:100170009104A104B10461F0B0E1CB1AB7E2DB0A4B
:10018000E108F108C818D908EA08FB08F7FE60CEB4
:100190001D8AFBCECF93C82F61E975E10E948D9D2A
:1001A000C11102C00E94677E4091C4055091C505EF
:1001B0006091C6057091C70588E895E10E94907D21
:1001C0002CEA35EC47E25EE36091C8057091C90501
:1001D0008091CA059091CB050E94CCDBAB01BC019C
:1001E00085E895E10E94907D2CEA35EC47E25EE3DC
:1001F0006091CC057091CD058091CE059091CF0591
:100200000E94A6D4AB01BC0182E895E10E94907DDA
:100210008AE0CF910C944F7DCF93DF93EB010E9446
:10022000567DBE01DD0F880B990BDF91CF910C94A9
:10023000499BCF93DF93EB010E94567DBE0190E076
:1002400080E00E94DF9A8AE0DF91CF910C944F7D8D
:10025000EC018B01F42E0E943528209709F47EC012
:100260000E94677ECE010E94567D8AE00E944F7DEB
:100270000115110511F402E41BE20E941E6C1F938C
:100280000F93DF93CF9382E494E19F938F9381E068
:100290008F930E94EA5B0E94E143C091A811C6952A
:1002A000C69583EA91E10E94E86EDC2FDD0F1D2FD9
:1002B0001C0F8DB79EB707960FB6F8949EBF0FBE62
:1002C0008DBF83E00E94946D1092DE11C093DF1108
:1002D00089EB9EE00E9402741092DE11D093DF1130
:1002E0006FEF7FEF83E394E10E94DC711092DE11E7
:1002F0001093DF116FEF7FEF86E294E10E94DC71D3
:1003000087EA91E10E94CBA38111DBCF0E94637E3B
:1003100082E594E10E94567D89EE93E0019739F0E1
:1003200000C00000EEE5F9E03197F0F7F7CFF89460
:1003300089EE93E0019739F000C00000E6EEF3E0AB
:100340003197F0F7F7CF0E943528FF2021F00E9467
:100350009F2CA895FECF0E945A2CFBCF01151105AA
:1003600011F402E41BE2C9E4D4E187CF8091060CCA
:100370009091070C2FEF3FEF981751F0E92FF0E025
:10038000EA5FF34F228130E09F5F9F779093070CE5
:10039000C90108951F920F920FB60F9211240F906A
:1003A0000FBE0F901F9018951F920F920FB60F92CD
:1003B00011240BB60F922F938F939F93EF93FF937C
:1003C0009091C6002091070CE091060C81E08E0F01
:1003D0008F77281729F0F0E0EA5FF34F9283E82F38
:1003E000E093060CFF91EF919F918F912F910F90C9
:1003F0000BBE0F900FBE0F901F9018958EBD0DB4C1
:1004000007FEFDCF08958FEF8EBD0DB407FEFDCF23
:100410008EB50895909164009B7F90936400982F0F
:10042000906A96959CBD80FD03C091E0863009F4EA
:1004300090E09DBD0895CF93DF93EB010E94567D20
:10044000CE01DF91CF910C9438A52F923F924F921D
:100450005F926F927F928F929F92AF92BF92CF9254
:10046000DF92EF92FF920F931F93CF93DF93CDB75D
:10047000DEB7C157D1090FB6F894DEBF0FBECDBFAE
:10048000A2968FAFA2972091B4052F962FAF2F97EA
:1004900021E02093B4058091CF048D3409F450C439
:1004A000843511F40C940796873481F48091CD043F
:1004B0009091CE048531910509F4DAC350F482306D
:1004C000910508F4D5C1049709F4DFC30E94CCAEAE
:1004D000CFC38A35910509F424C408F074C14C9740
:1004E000A9F787E00E94053D811111C08091C704E2
:1004F0009091C804A091C904B091CA04FEE0B695D9
:10050000A79597958795FA95D1F780FDB1C30E947D
:10051000E72D10920B010E943CA16093D8057093C7
:10052000D9058093DA059093DB0580913501909190
:100530003601A0913701B09138018093A8049093BF
:10054000A904A093AA04B093AB04809106019091F2
:1005500007019093A7048093A60484E690E090930B
:1005600007018093060181E080932C050E944B3F98
:100570008091C7049091C804A091C904B091CA04A5
:10058000A7FB992490F82B2F2170B1FB882780F9C5
:10059000921203C0891509F4B1C3222E382E82E5C8
:1005A0000E944967882309F4B0C30E94BE6B762E6F
:1005B000C72ED82EE92E20E030E0A9010E9440D4B9
:1005C000882309F44BC0911003C0222009F4D0C045
:1005D00080906A01F0906B0100916C0110916D01A7
:1005E000282D3F2DA801672D7C2D8D2D9E2D0E943D
:1005F00040D487FD04C0872CFC2C0D2D1E2D80E0DF
:1006000090E0A0E8B0E489839A83AB83BC8320E0C8
:1006100030E04AE753E4682D7F2DC8010E9440D4A2
:1006200087FD04C0812CF12C0AE713E420916601B8
:1006300030916701409168015091690160916201B8
:10064000709163018091640190916501DE011196C2
:100650006D01482C5F2C72010E941F3D992009F406
:1006600082C0222009F47CC01092620110926301C2
:100670001092640110926501109266011092670158
:1006800010926801109269010E94D73DE2E8F6E0FD
:10069000C590D590E590F490E6E8F6E04590559049
:1006A00065907490A7019601C301B2010E9440D4E5
:1006B00087FF32C3A7019601C301B2010E94CCDBC0
:1006C0009B01AC010E94A6D420E030E040E85FE34B
:1006D0000E9449DB0E940ADD20E030E048E452E459
:1006E0000E94A6D469837A838B839C8380906A015D
:1006F00090906B01A0906C01B0906D0120E030E013
:1007000040EC5FE3C301B2010E94A6D42B013C017F
:1007100077FA709477F8709420E030E040EC5FE373
:10072000C701B6010E94A6D49058FE0131966F0110
:1007300085017401A30192010E941F3D0E940D409A
:10074000109262011092630110926401109265018F
:10075000109266011092670110926801109269016F
:1007600080E00E94D93D222019F081E00E94D93D0D
:10077000332019F082E00E94D93D0E94D73D80913C
:100780002B0580932C058091A8049091A904A09139
:10079000AA04B091AB048093350190933601A093E5
:1007A0003701B09338018091A6049091A7049093EB
:1007B00007018093060183E080934E010E94B09C64
:1007C0000E94AE3055C28B35910509F4ADC28C350F
:1007D000910509F07BCE59E0252E52E0352E62E6D8
:1007E000E62E61E0F62EC12CD12C10E0D1018D91C6
:1007F0001D010E944967082F882351F10E94BE6B9A
:100800002B013C01F70120813181428153810E94FB
:1008100048DB4B015C012DEB37E346E855EB0E94CA
:10082000CCDC87FD0AC02DEB37E346E855E3C50174
:10083000B4010E9440D418165CF4133011F0C02E9D
:100840000D2DD7014D925D926D927C921397D02E13
:100850001F5FB4E0EB0EF11C143041F6CC2009F41C
:1008600067C20E94D73D0E94B09C0E94AE3000C279
:100870008091DC05833008F4FBC1A0E7CA2EA2E01A
:10088000DA2EB2E6EB2EB1E0FB2E10E088E5810F08
:100890000E944967882309F499C10E94BE6B4B01ED
:1008A0005C01812F0E94AA66882359F0D7012D91FF
:1008B0003D914D915C91C501B4010E9449DB4B0112
:1008C0005C01F60180829182A282B3821F5FF4E014
:1008D000CF0ED11C24E0E20EF11C1330B9F685E4F2
:1008E0000E944967882309F47CC10E94BE6B6B019A
:1008F0007C0183E00E94AA66882371F020916E013A
:1009000030916F014091700150917101C701B601A2
:100910000E9449DB6B017C01C0927C02D0927D0277
:10092000E0927E02F0927F0286E40E94496788236B
:10093000C9F00E94BE6B20E030E0A9010E94CCDC2F
:10094000181684F40E94BE6B20E030E040E752E4C9
:100950000E94CCDB609335017093360180933701A0
:100960009093380180910A01882309F4BDC08091D9
:100970006F02082F80FF3CC0C0900C01D0900D0189
:10098000E0900E01F0900F01209170023091710201
:100990004091720250917302C701B6010E94CCDCF3
:1009A000181644F4C0927002D0927102E092720262
:1009B000F0927302C0901801D0901901E0901A01D2
:1009C000F0901B01209170023091710240917202EF
:1009D00050917302C701B6010E9440D487FF08C03E
:1009E000C0927002D0927102E0927202F092730291
:1009F00001FF3CC0C0901001D0901101E0901201A5
:100A0000F0901301209174023091750240917602AA
:100A100050917702C701B6010E94CCDC181644F44D
:100A2000C0927402D0927502E0927602F092770240
:100A3000C0901C01D0901D01E0901E01F0901F019C
:100A400020917402309175024091760250917702A4
:100A5000C701B6010E9440D487FF08C0C09274024B
:100A6000D0927502E0927602F092770202FF3CC0CB
:100A7000C0901401D0901501E0901601F09017017C
:100A8000209178023091790240917A0250917B0254
:100A9000C701B6010E94CCDC181644F4C09278025B
:100AA000D0927902E0927A02F0927B02C09020010B
:100AB000D0902101E0902201F09023012091780252
:100AC0003091790240917A0250917B02C701B601C0
:100AD0000E9440D487FF08C0C0927802D092790269
:100AE000E0927A02F0927B028091BC0B83FD8CC075
:100AF00020916E0130916F01409170015091710110
:100B000060917C0270917D0280917E0290917F02C3
:100B10000E9440D4882309F477C00E94492D182FE1
:100B2000882331F00E94677E8CEE95E10E94567D0D
:100B300020916E0130916F014091700150917101CF
:100B400060917C0270917D0280917E0290917F0283
:100B50000E9448DB6B017C0120E030E0A9010E948B
:100B6000CCDC87FF04C0F7FAF094F7F8F0942091FA
:100B70005E0130915F014091600150916101C701B8
:100B8000B6010E94A6D420E030E046E154E40E9481
:100B9000CCDC1816BCF50E94677E8DEC95E10E94B6
:100BA000567D80917C0290917D02A0917E02B09151
:100BB0007F0280936E0190936F01A0937001B093B8
:100BC00071018CE792E00E94C43B1EC0F701808156
:100BD0009181A281B381F60180839183A283B38343
:100BE00075CE80916E0190916F01A0917001B091CE
:100BF000710180937C0290937D02A0937E02B0935A
:100C00007F0292CE1111CDCF2AE037ED43E25CE3B3
:100C100060913501709136018091370190913801D2
:100C20000E94A6D46B017C016091060170910701BE
:100C3000072E000C880B990B0E9447D49B01AC0136
:100C4000C701B6010E94A6D469837A838B839C83F3
:100C5000BE016F5F7F4F80E792E00E94CCC680E1CB
:100C6000E0E7F2E0A2E6B1E001900D928A95E1F7AB
:100C7000A2963FADA297311102C00E947D7D2F96B2
:100C80004FAD2F974093B40539C680E50E94496760
:100C9000C12CD12C7601882321F00E94AE6B6B0110
:100CA0007C0183E50E944967882361F00E94BE6B46
:100CB00020E030E04AE754E40E94A6D40E9445DCDC
:100CC0006B017C010E94E72D8091B90E811105C056
:100CD00060E087E096E10E94055C0E943CA1C60EA0
:100CE000D71EE81EF91E0E943CA16C197D098E09D1
:100CF0009F0997FFBDCF0E9444B1F5CF22242394D2
:100D000099249394332433944ACC712CC12C70EAE7
:100D1000D72EE0E4EE2E57CCA3019201C701B60115
:100D2000CDCC1092AC04A4CF8FE08093AC04A0CFC4
:100D3000DD2009F498CD8EE691E00E94C43B93CD6E
:100D40008091CD049091CE048F36910509F432C67E
:100D500008F036C28032910509F416C508F040C18A
:100D60008731910509F416C408F0A5C082319105B8
:100D700009F4A0C108F06EC08230910508F485C363
:100D8000419709F0A3CB0E94C066882309F4D8C319
:100D90000E941F6700918A02102F1095182309F4F2
:100DA00067CFF12CE12CD12CA12EB12CC5010E2C3A
:100DB00002C0959587950A94E2F780FF08C08E2DB2
:100DC0000E94AA2CF701E952FE4F8081D82A4FEFEA
:100DD000E41AF40A53E0E516F10441F713FF05C0E5
:100DE0000E94682C8D2D8360D82E102B10951D210C
:100DF00009F43ECF88E20E944F7DF12CE12CC12EF8
:100E0000D12CC6010E2C02C0959587950A94E2F765
:100E100080FF09C0F701E75FFD4F80810E944F7D91
:100E200080E20E944F7D9FEFE91AF90AA3E0EA16DB
:100E3000F10439F713FF09C085E40E944F7D80E378
:100E40000E944F7D80E20E944F7D83E296E10E94E6
:100E5000567D0ECF8531910509F48AC308F08BC306
:100E6000449709F033CB8091F91284FF7AC38AE466
:100E700096E10E94567D8091F91284FF17C084E5A7
:100E800091E10E94DC248BE1E4E5F1E1DE011196C1
:100E900001900D928A95E1F770E060E0CE01019635
:100EA0000E9443AFCE0101960E94AF268BE396E1EC
:100EB0000E94567DDDCE8B31910509F4A7C308F55C
:100EC0008931910509F487C308F47AC38091F91236
:100ED00084FFCECE83E50E944967882309F4C8CEFB
:100EE0000E94526BAB01BC014093F5125093F61275
:100EF0006093F7127093F8128EE191E10E948BA932
:100F0000B7CE8D31910509F4E2C308F4D9C38E310F
:100F1000910509F4E2C34F9709F0D8CA0E941B401B
:100F20007B018C0120E831E541E050E00E9488DA45
:100F3000C9016DE671E00E94DEDA4B015C01C80177
:100F4000B70120E13EE040E050E00E9488DACA01AB
:100F5000B90128E130E040E050E00E9488DA762EC6
:100F6000672EC62ED72E3CE3232E312C412C512C3C
:100F7000C801B701A20191010E9488DAF62EE72E7E
:100F8000CA01B901A20191010E9488DACB018E0148
:100F90000F5F1F4F8114910409F436C4EF92FF9242
:100FA0007F936F936F927F92BF92AF929F928F9237
:100FB00082EF96E19F938F931F930F930E94D7D355
:100FC0000FB6F894DEBF0FBECDBFC8010E94F09CE3
:100FD0000E94677EB80186E097E10E94DAAE48CEB3
:100FE0008535910509F41AC608F087C08D3491053E
:100FF00009F465C4D0F58B34910509F44AC408F0AE
:101000004BC48934910509F061CA80E50E944967A3
:101010008823A1F00E94BE6B20E030E048EC52E44F
:101020000E94A6D40E9445DC6031B7E27B0710F035
:1010300060E177E270935D0260935C0282E50E945A
:101040004967882309F414CE0E94AE6B9B01AC0162
:10105000ACE3B0E00E94AADA6093DC047093DD0494
:101060008093DE049093DF0403CE8235910509F46A
:1010700055C5C0F48135910509F028CA0E94F72DA5
:101080001092F9050E9435280E949E4068EE73E098
:1010900080E090E00E94E87660E082E397E10E94C1
:1010A000055CE6CD8335910509F43FC5843591058E
:1010B00009F00CCA83E50E944967882309F43CC5FE
:1010C0000E943CA16093D8057093D9058093DA05FE
:1010D0009093DB050E94BE6B20E030E04AE754E4C9
:1010E0000E94A6D40E9445DC60935A0170935B0174
:1010F00080935C0190935D01BBCD8A36910509F424
:1011000017C408F03EC08836910509F4DBC308F027
:10111000E1C38C35910509F0D9C90E946B7E87FD2A
:10112000A7CD8091C70484FD09C08091C90487FDC3
:1011300005C08091CA04837009F4E3C5B9E0CB2EE1
:10114000B2E0DB2E1DEBE12E1BE0F12E10E0D6010C
:101150008D916D010E944967882351F0133009F485
:1011600081C50E94BE6BF701648B758B868B978B54
:101170001F5FF4E0EF0EF11C143049F70E94BB2D05
:1011800077CD8C36910509F451C408F406C48D3628
:10119000910509F49BC38E36910509F097C98EE439
:1011A0000E944967882309F463CD0E94526B6093C3
:1011B000880C7093890C80938A0C90938B0C58CD7B
:1011C0008C3D910511F40C947C9108F08DC0893709
:1011D000910509F48FC6D0F58337910509F496C5BA
:1011E00068F48137910509F42DC408F424C40E94E1
:1011F000B09C8DE791E10E94A12B3ACD86379105F5
:1012000009F435C698F48537910509F05FC98091D6
:10121000CB049091CC04009709F4DAC1DC012C9145
:10122000222309F4D5C10E94F09C22CD8737910575
:1012300009F45CC68837910509F048C981E08093BC
:101240002C0580932B050E944B3F12CD893C9105C4
:1012500009F49EC6D8F48A39910509F415C48B396E
:10126000910509F436C48139910509F02FC970E060
:1012700060E083E50E949F6B823008F443C60E94C1
:10128000637E88EC99E10E94567DF2CC8C3C9105FE
:1012900009F4DCC6B0F48B3C910509F017C98091C4
:1012A000C70484FDB0C68091C904887809F0ABC634
:1012B0008091CA04837009F0A6C681E00E94FF7D78
:1012C000D7CC8D3C910509F416C7833D910509F0F3
:1012D000FDC883E50E94D166882309F479C70E947E
:1012E000766B80930A01C4CC843FE1E09E0711F441
:1012F0000C94CA9508F060C08D3221E0920711F479
:101300000C94639208F042C0823241E0940711F4D9
:101310000C94D9918C3251E0950711F40C944492BD
:101320008D3D910509F0D2C80E946B7E082F87FD84
:101330009FCC83E50E944967002E000C110B7801B9
:10134000EE0CFF1C882311F40C94BF910E949B6B40
:10135000F701EC5DFE4F91838083000F111F000F9A
:10136000111F025A1E4FBC01990F880B990B0E9446
:1013700047D42AE037ED43E25CE30E94A6D4D801CB
:101380006D937D938D939C93139772CC8F32A1E0D4
:101390009A0711F40C94F39210F40C94AD928039E6
:1013A000E1E09E0711F40C94C6958A39914009F04A
:1013B0008DC80E94AE3E5CCC883F31E0930711F4AB
:1013C0000C94D69590F4863F51E0950711F40C9457
:1013D000D29510F40C94CE9561E083E50E94866B63
:1013E00091E089270E94BF2C43CC803AB3E09B0751
:1013F00009F4FDC1A8F48C30924009F067C810913F
:10140000F91212FD02C00C94E89517FF02C00C946B
:10141000E8950E940C7780FB17F91093F91228CCFD
:10142000873E23E0920711F40C94F095893E934097
:1014300009F04CC80E94E72D8091F912877F8B7FBD
:101440008093F9128091F01281110C9400960E9401
:101450001B406D3371058105910520F087E39CE108
:101460000E94AC9783E39CE10E94AC9780E197EAED
:1014700090935D0280935C028FE19CE10E94567D17
:101480008BE19CE10E94AC97F3CB80E50E94496719
:10149000C12CD12C7601882321F00E94AE6B6B0108
:1014A0007C0183E50E944967882361F00E94BE6B3E
:1014B00020E030E04AE754E40E94A6D40E9445DCD4
:1014C0006B017C010E94E72D8091CB049091CC04AC
:1014D000009709F10E94F09C1091B40583E080937D
:1014E000B40581E08093D305C114D104E104F10473
:1014F00031F00E943CA1C60ED71EE81EF91E809155
:10150000D3058823B1F0C114D104E104F10449F4F6
:101510000E9444B1F4CF60E080E196E10E94055C56
:10152000DBCF0E943CA16C197D098E099F0997FDB4
:10153000EFCF1092D3051093B4050E94DE9D98CB97
:1015400060E082E396E10E94055C80E00E94AA2CA4
:1015500081E00E94AA2C82E00E94AA2C0E94682CA2
:1015600087CB0E94677E8BE596E10E94567D80CBFB
:101570000E94F2AC7DCB8091F91282FF02C087FFFE
:1015800077CB0E9444A58091F9128F7E806480936E
:10159000F9126ECB8091CB049091CC04FC01219187
:1015A000222331F02032D9F7DF0111971C92F7CFB7
:1015B00060E00E9416B010925D0210925C0258CB5F
:1015C0000E940C77882321F00E9452A50E943F7D43
:1015D0000E94DE9D4DCB8091F91282FF05C087FDF0
:1015E00003C08B7F8093F9128091A805813081F729
:1015F00082E08093A8050E943CA160936B027093E7
:101600006C0280936D0290936E02E2CF8091C704CA
:101610009091C804A091C904B091CA0442E0B69563
:10162000A795979587954A95D1F780FF1CC08FE6BF
:1016300096E10E94567D80912111882379F0BE01A8
:101640006F5F7F4F8EE191E10E94A723CE0101964B
:101650000E9438A58AE00E944F7D0ACB85E696E17C
:101660000E94567DF7CF8091F91282FF24C0C0906E
:10167000F512D090F612E090F712F090F8128EE783
:1016800096E10E94567DC701B6010E94DF9A8FE263
:101690000E944F7D6091F1127091F2128091F312CD
:1016A0009091F4120E94DF9A8DE00E944F7D8AE0B3
:1016B0000E944F7DDDCA80E996E10E94567DD8CA1E
:1016C0008091CB049091CC040E94FAAED1CA809153
:1016D000F9128E7F8093F912CBCA8091F91284FFA0
:1016E000C7CA0E9474A98091F91284FFC1CA4091AF
:1016F000CB045091CC04BE01645E7F4F80E00E9419
:1017000056AD8C01009709F4B3CA6C8D7D8D19829A
:101710001C8222E0AC01CE0101960E94B526811107
:1017200015C0F12CCE0101960E94AF26B801FF2012
:1017300011F18CEB96E10E94DAAE1092F512109244
:10174000F6121092F7121092F81292CACE01019678
:101750000E941FAA882329F361E0CE0101960E940E
:101760008D230097F1F225EEFC0120831C820E945C
:10177000E6A5F82ED7CF84EA96E10E941B8281EA83
:1017800096E10E94567D74CA8091F91282FF03C0CF
:1017900087FF0E94E72D8091F91284FF69CA60E0FB
:1017A00080E50E94866B182F682F8091CB04909162
:1017B000CC040E9416B083E50E944967882381F01B
:1017C0000E94526BAB01BC014093F5125093F6128C
:1017D0006093F7127093F8128EE191E10E948BA949
:1017E0000E9452A5111144CA0E943F7D41CA209116
:1017F000CB043091CC049091F91292609093F9123D
:10180000C9010E94FAAE34CAA114B10489F0EF9262
:10181000FF927F936F936F927F92BF92AF9282EE0F
:1018200096E19F938F931F930F930E94D7D3C8CBBA
:10183000CD2879F0EF92FF927F936F936F927F9212
:1018400086ED96E19F938F931F930F930E94D7D3BA
:10185000B7CB892B69F0EF92FF927F936F938EEC59
:1018600096E19F938F931F930F930E94D7D3A8CB9A
:10187000EF92FF928AEC96E19F938F931F930F93C1
:101880000E94D7D30F900F900F900F900F900F9052
:101890009CCB0E943F7DECC98091A805813009F066
:1018A000E7C982E08093A8050E943CA160936B0287
:1018B00070936C0280936D0290936E02D9C90E945E
:1018C0009E40D6C980E00E94967ED2C981E00E94E7
:1018D000967ECEC90E946B7E182F87FD0AC083E1D9
:1018E00097E10E94567D812F0E94AD278AE00E94D9
:1018F0004F7D2F96EFAD2F97E093B405CF58DF4F74
:101900000FB6F894DEBF0FBECDBFDF91CF911F9110
:101910000F91FF90EF90DF90CF90BF90AF909F908E
:101920008F907F906F905F904F903F902F90089591
:1019300080E50E94496781112BC08091C7040FEF99
:1019400010E080FF04C06091F905062F10E089E4E3
:101950000E944967882311F40C942B960E94626BB5
:1019600090E01816190614F481E090E0880F991F92
:10197000880F991FFC01EF57FD4F028113810F3F24
:10198000110519F010F00FEF10E00093F90570C980
:101990000E94626B81116CC9D0CF80E50E944967BB
:1019A000811103C01092F90563C90E94626B811115
:1019B0005FC9F8CF83E50E944967882321F00E9420
:1019C000626B8093BC0B0E94677E84E297E10E9469
:1019D000567D8091BC0B882331F110E000E020E0BF
:1019E0008091BC0B90E0002E02C0959587950A94DB
:1019F000E2F780FF12C0FF24F394F20E222319F0C5
:101A00008CE20E944F7DF801EE0FFF1FE65EF84E5C
:101A1000859194910E94567D2F2D0F5F1F4F0530A9
:101A20001105F1F617CE86E197E11ACE1092D30593
:101A3000109259011DC941E070E060E08CEB9CE21E
:101A40000E94288183E50E944967882359F00E94FB
:101A5000626B8D3318F480934D010AC98CE3809337
:101A60004D0106C90E94677E10914D018BE297E1FE
:101A70000E94567D612F70E090E080E00E94DF9A26
:101A80008AE00E944F7DF4C883E50E94496788235D
:101A900009F4EEC80E94626B182F8C3308F08CE3B7
:101AA0008093AE050E943CA16B017C01212F30E0A8
:101AB000A8EEB3E00E94B5DAC60ED71EE81EF91EE6
:101AC000C092AA05D092AB05E092AC05F092AD05AC
:101AD000CFC883E50E944967882309F4C9C80E94DA
:101AE000626B182F8C3308F08CE38093B3050E944F
:101AF0003CA16B017C01212F30E0A8EEB3E00E94F5
:101B0000B5DAC60ED71EE81EF91EC092AF05D092F8
:101B1000B005E092B105F092B205AAC88091AC047C
:101B20008F7D80618093AC04A3C88091AC048F7ECC
:101B300080628093AC049CC80E94C066882309F42C
:101B40006AC00E94E72D0E941F67082F10918A0229
:101B5000182309F48DC8F12CE12CC82ED12CAA240D
:101B6000A394B12CC6010E2C02C0959587950A94BA
:101B7000E2F780FF12C08E2D0E946F2C882369F03F
:101B800095010E2C01C0220F0A94EAF7F701E952E1
:101B9000FE4F8081822B80951823FFEFEF1AFF0AFA
:101BA00023E0E216F104F1F603FF04C00E945A2C70
:101BB0008111147FF12CE12CC12ED12CC6010E2CE9
:101BC00002C0959587950A94E2F780FF0FC0F70150
:101BD000E75FFD4F80810E944F7DF701E952FE4F84
:101BE000908180918A0289230E941CC93FEFE31AE9
:101BF000F30A43E0E416F10409F713FF39C885E45A
:101C00000E944F7D80E30E944F7D80918A02837005
